:100000000C942A110C9423140C944E140C9479140F
:100010000C94A4140C94CF140C94FA140C9425157D
:100020000C9450150C945A110C945A110C945A11AA
:100030000C945A110C945A110C945A110C945A1194
:100040000C945A110C94E92F0C945A110C945A11D7
:100050000C945A110C945A110C9425240C945C1194
:100060000C945A110C947B170C9427180C945A1169
:100070000C945A110C945A110C945A110C945A1154
:100080000C945A110C945A110C945A110C945A1144
:100090000C945A110C945A110C945A110C945A1134
:1000A0000C945A110C945A110C945A110C945A1124
:1000B0000C945A110C945A110C945A110C945A1114
:1000C0000C945A110C945A110C945A110C945A1104
:1000D0000C945A110C945A110C945A110C945A11F4
:1000E0000C945A1199129E12A312AD12B71230132A
:1000F000C112C912D112DB12E512EF12FE1208135F
:10010000301312131C1326135413571346134A1398
:1001100050138E135B135F13651369136D13731301
:1001200077137B138E13811385138913AE17B417BE
:10013000C517D017D817ED17DC17ED17E017E41720
:10014000ED17EA17691F691F701F701F701F771F57
:10015000771F771F841F7E1F7E1F7E1F084AD73B95
:100160003BCE016E84BCBFFDC12F3D6C74319ABD86
:1001700056833DDA3D00C77F11BED9E4BB4C3E91AA
:100180006BAAAABE000000803F05A84CCDB2D44E99
:10019000B93836A9020C50B9918688083CA6AAAA9B
:1001A0002ABE000000803F004E414E494E4954593E
:1001B000494E46CDCCCC3D0AD7233C17B7D1387732
:1001C000CC2B329595E6241FB14F0A000020410048
:1001D00000C84200401C4620BCBE4CCA1B0E5AAE92
:1001E000C59D7400000A0B02090C0D0E08070304DC
:1001F00001000000000000000000000000000000FE
:1002000000000000000000000000000000000012DC
:1002100011100000000000000000000000000000BD
:10022000000000000000000000010210202008086B
:100230001020401020408002010201080402010148
:100240000204081020408080402010080402018031
:100250000402018040201008040201080402010188
:10026000020408102040800102040810204080058C
:10027000050505070508080808020202020A0A081F
:100280000804040404010101010101010103030345
:100290000303030303040707070C0C0C0C0C0C0CE2
:1002A0000C0202020206060606060606060B0B0BE9
:1002B0000B0B0B0B0B000020002300260029002C49
:1002C000002F0032000001000003010601090100B7
:1002D000002200250028002B002E003100340002EF
:1002E000010000050108010B010000210024002786
:1002F000002A002D00300033000101000004010736
:10030000010A014F4646004F4E006563686F3A0090
:100310004572726F723A004572726F72207772691D
:1003200074696E6720746F20454550524F4D210A05
:100330000063616E63656C00706F7765726F6666EF
:10034000002F2F616374696F6E3A0020573A0020C6
:10035000573A00202F002042403A0020403A0054F3
:100360006865726D616C2052756E617761790045C8
:100370003120544845524D414C2052554E41574131
:10038000590042454420544845524D414C20525555
:100390004E4157415900202D20496E76616C6964A9
:1003A000206578747275646572206E756D62657211
:1003B00020210A0048656174696E67206661696C76
:1003C0006564004265642068656174696E672066D3
:1003D00061696C65640048656174696E6720666177
:1003E000696C65640045312048656174696E6720F9
:1003F0006661696C6564004D494E54454D502074EA
:100400007269676765726564004531204572723AAA
:10041000204D494E54454D50004572723A204D4989
:100420004E54454D5020424544004D415854454D91
:1004300050207472696767657265640045312045B4
:1004400072723A204D415854454D50004572723AEF
:10045000204D415854454D5020424544006265644A
:100460000A002C2073797374656D2073746F70703B
:10047000656421204865617465725F49443A2000D3
:1004800023646566696E652044454641554C545F5A
:10049000004B6420004B6920004B70200000626517
:1004A0006400504944204175746F74756E65206610
:1004B000696E69736865642120507574207468657D
:1004C000206C617374204B702C204B6920616E642A
:1004D000204B6420636F6E7374616E747320667258
:1004E0006F6D2062656C6F7720696E746F20436F4B
:1004F0006E66696775726174696F6E2E680A005066
:100500004944204175746F74756E65206661696C2D
:100510006564212074696D656F75740A005468659F
:10052000726D616C2052756E617761790045312082
:10053000544845524D414C2052554E415741590067
:1005400042454420544845524D414C2052554E415D
:100550005741590048656174696E67206661696C2E
:1005600065640045312048656174696E6720666185
:10057000696C6564004265642068656174696E67D2
:10058000206661696C656400504944204175746F50
:1005900074756E65206661696C6564212054656DB3
:1005A000706572617475726520746F6F2068696719
:1005B000680A00204B643A2000204B693A20002052
:1005C0004B703A20000A20436C61737369632050BA
:1005D0004944200A002054753A2000204B753A20E7
:1005E00000206D61783A2000206D696E3A2000206D
:1005F000643A200020626961733A20005049442027
:100600004175746F74756E652073746172740A003D
:10061000504944204175746F74756E652066616938
:100620006C6564212054656D7065726174757265C6
:1006300020746F6F20686967680A001000AD03308E
:10064000016A0150022B0170030A019004F500B009
:1006500005E500D006D800F007CE001009C500302F
:100660000ABE00500BB700700CB100900DAB00B08B
:100670000EA600D00FA200F0109D001012990030BD
:100680001395005014920070158E0090168B00B0D8
:10069000178700D0188400F0198100101B7E0030ED
:1006A0001C7B00501D7900701E7600901F7300B0F7
:1006B000207000D0216E00F0226B00102469003001
:1006C000256600502663007027610090285E00B008
:1006D000295C00D02A5900F02B5600102D54003010
:1006E0002E5100502F4E0070304B0090314800B01A
:1006F000324500D0334200F0343E0010363B00302B
:100700003737005038330070392E00903A2900B046
:100710003B2300D03C1B00F03D1100103F0100F0D6
:100720003F00001000C90210012C0140012201709D
:10073000011801B0010E01F00104015002FA00B0ED
:1007400002F0003003E600D003DC009004D2007019
:1007500005C800A006BE000008B400B009AA00D079
:100760000BA000600E960060118C00001582002026
:10077000197800C01D6E00A0226400B0275A0090B6
:100780002C500000314600E0343C0010383200901C
:100790003A2800603C1E00A03D1400803E0A002064
:1007A0003F00006F70656E005452494747455245FF
:1007B00044003A20007A5F6D6178007A5F6D696E5F
:1007C00000795F6D617800795F6D696E00785F6DAB
:1007D000617800785F6D696E005265706F72746940
:1007E0006E6720656E6473746F70207374617475C6
:1007F000730A00205A3A0020593A0020583A0065FE
:100800006E6473746F7073206869743A2000486F67
:100810006D696E67206661696C656400496E76611A
:100820006C69642065787472756465720A0045307D
:100830003A20005A3A2000593A20004D53312C4DAD
:1008400053322C4D53332050696E730A583A2000AE
:100850004D6963726F737465707320756E61766134
:10086000696C61626C650A00205A3A0020593A00AE
:1008700020436F756E7420583A00C23100001C2668
:100880000000F4190000D80F0000EB080000C004BD
:100890000000750200004001000024F4D43050C371
:1008A0008E20C2A24017828B7011127A910D816C3A
:1008B000D90AA861E108C7586607615143061E4B73
:1008C0005D05C145A7041A411104093D980371391A
:1008D00031034036DB0265339102D4305402802E5E
:1008E0001D02632CEE01752AC501B028A001102756
:1008F00081018F2564012B244B01E0223401AC21BE
:100900001F018D200D01801FFC00841EED00971D2E
:10091000DF00B81CD200E61BC600201BBC00641A16
:10092000B200B219A8000A19A0006A189900D117DC
:10093000910040178B00B516840031167E00B31568
:1009400079003A157300C7146F0058146A00EE134B
:1009500066008813630025135E00C7125B006C12EB
:10096000570015125400C111510070114F00211190
:100970004B00D61049008D1047004610440002106D
:100980004200C00F4000800F3E00420F3C00060FA7
:100990003B00CB0E3800930E37005C0E3500270E5F
:1009A0003400F30D3200C10D3100900D3000600DA8
:1009B0002E00320D2D00050D2C00D90C2B00AE0C95
:1009C0002900850C29005C0C2700350C27000E0C33
:1009D0002600E80B2400C40B2400A00B23007D0B91
:1009E00023005A0B2100390B2100180B2000F80AB4
:1009F0001F00D90A1E00BB0A1E009D0A1D00800AA6
:100A00001D00630A1C00470A1B002C0A1B00110A68
:100A10001A00F7091A00DD091900C4091900AB0909
:100A20001900920917007B091800630917004C0987
:100A3000160036091600200916000A091500F508E7
:100A40001500E0081400CC081400B8081400A4082D
:100A50001400900813007D0812006B08130058085A
:100A60001200460812003408110023081100120871
:100A7000110001081100F0071000E0071000D00776
:100A80001000C0071000B0070F00A1071000910769
:100A90000E0083070F0074070F0065070E0057074D
:100AA0000E0049070E003B070D002E070E00200721
:100AB0000D0013070D0006070D00F9060C00ED06EA
:100AC0000D00E0060C00D4060C00C8060C00BC06A5
:100AD0000C00B0060C00A4060B0099060C008D0655
:100AE0000B0082060B0077060B006C060B006106FC
:100AF0000A0057060B004C060A0042060A00380698
:100B00000A002E060A0024060A001A060A00100629
:100B1000090007060A00FD050900F4050900EB05B8
:100B20000900E2050900D9050900D0050900C7053B
:100B30000900BE050900B5050800AD050800A505BA
:100B400009009C050800940508008C050800840530
:100B500008007C050800740508006C0507006505A1
:100B600008005D050700560508004E05070047050B
:100B700007004005080038050700310507002A0571
:100B80000700230507001C050600160507000F05D2
:100B900007000805060002050700FB040600F5042F
:100BA0000700EE040600E8040600E2040700DB0488
:100BB0000600D5040600CF040600C9040600C304DD
:100BC0000600BD040600B7040600B1040500AC042D
:100BD0000600A6040600A00405009B040600950478
:100BE0000500900406008A040500850405008004C1
:100BF00006007A04050075040500700405006B0406
:100C0000050066040500610405005C040500570446
:100C10000500520405004D04050048040500430486
:100C200005003E0404003A040500350405003004C4
:100C300004002C04050027040400230405001E04FE
:100C400004001A04040016040500110404000D0435
:100C50000400090405000404040000040400FC036B
:100C60000400F8030400F4030400F0030400EC03A0
:100C70000400E8030400E4030400E0030400DC03D0
:100C80000400D8030400D4030400D0030400CC0300
:100C90000400C8030300C503030024F404D9201B87
:100CA000C40C5C0E9804C4095F0265077101F40569
:100CB000F900FB04B30048048700C103690058032E
:100CC000550003034500BE023A008402310053027E
:100CD0002A002902250004022000E4011C00C801AA
:100CE0001900AF011700980114008401130071016D
:100CF00010006101100051010E0043010D0036018A
:100D00000B002B010B0020010B00150109000C0149
:100D1000090003010800FB000800F3000800EB00D5
:100D20000700E4000600DE000600D8000600D2003E
:100D30000600CC000500C7000500C2000500BD008C
:100D40000400B9000400B5000400B1000400AD00C7
:100D50000400A9000400A5000300A20003009F00F6
:100D600004009B000300980003009500020093001C
:100D70000300900003008D0002008B000300880038
:100D800002008600020084000300810002007F0050
:100D900002007D0002007B00020079000200770063
:100DA0000100760002007400020072000100710070
:100DB00002006F0002006D0001006C0002006A007A
:100DC0000100690002006700010066000100650083
:100DD0000100640002006200010061000100600087
:100DE00001005F0002005D0001005C0001005B008B
:100DF00001005A000100590001005800010057008D
:100E0000010056000100550001005400010053008C
:100E10000000530001005200010051000100500089
:100E200001004F0001004E0000004E0001004D0087
:100E300001004C0001004B0000004B0001004A0083
:100E4000010049000100480000004800010047007F
:100E5000010046000000460001004500000045007A
:100E60000100440001004300000043000100420073
:100E7000000042000100410000004100010040006C
:100E800001003F0000003F0001003E0000003E0066
:100E900001003D0000003D0001003C0000003C005E
:100EA00000003C0001003B0000003B0001003A0054
:100EB00000003A000100390000003900010038004C
:100EC0000000380000003800010037000000370043
:100ED0000100360000003600000036000100350039
:100EE000000035000000350001003400000034002F
:100EF0000000340001003300000033000000330024
:100F00000100320000003200000032000100310018
:100F1000000031000000310001003000000030000E
:100F20000000300001002F0000002F0000002F0003
:100F300000002F0001002E0000002E0000002E00F7
:100F400001002D0000002D0000002D0000002D00EC
:100F500001002C0000002C0000002C0000002C00E0
:100F600001002B0000002B0000002B0000002B00D4
:100F700001002A0000002A0000002A0000002A00C8
:100F800001002900000029000000290000002900BC
:100F900000002900010028000000280000002800AF
:100FA00000002800000028000100270000002700A2
:100FB0000000270000002700000027000100260095
:100FC0000000260000002600000026000000260089
:100FD000010025000000250000002500000025007C
:100FE000000025000000250001002400000024006E
:100FF0000000240000002400000024000100230061
:101000000000230000002300000023000000230054
:101010000000230000002300010022000000220045
:101020000000220000002200000022000000220038
:10103000010021000000210000002100000021002B
:10104000000021000000210000002100010020001C
:101050000000200000002000000020000000200010
:1010600000002000000020000000200001001F0000
:1010700000001F0000001F0000001F0000001F00F4
:1010800000001F0000001F0001001E0000001E00E5
:1010900000001E0000001E0000003A0A0020286D1B
:1010A0006D2900204500205A0020204D393037207E
:1010B000580053746570706572206D6F746F722084
:1010C00063757272656E74733A0A0020204D393070
:1010D00030204B004C696E65617220416476616E10
:1010E00063653A0A0020204D383531205A005A2DC8
:1010F00050726F6265204F6666736574002044000D
:1011000020490020204D333034205000204400205E
:10111000490020204D333031205000504944207385
:10112000657474696E67733A0A0020204D3432305A
:101130002053004175746F20426564204C657665CC
:101140006C696E673A0A00205A0020590020204D31
:10115000323036205800486F6D65206F66667365C3
:10116000743A0A00204500205A00205900205800F7
:1011700020540020530020204D32303520420020E2
:10118000453C6D61785F655F6A65726B3E00205813
:101190003C6D61785F785F6A65726B3E20593C6D8B
:1011A00061785F795F6A65726B3E205A3C6D617849
:1011B0005F7A5F6A65726B3E00416476616E63655B
:1011C000643A20423C6D696E5F7365676D656E744D
:1011D0005F74696D655F75733E20533C6D696E5F2A
:1011E00066656564726174653E20543C6D696E5F2E
:1011F00074726176656C5F66656564726174653E84
:101200000020540020520020204D32303420500065
:10121000416363656C65726174696F6E2028756ED9
:101220006974732F7332293A20503C7072696E745E
:101230005F616363656C3E20523C726574726163EA
:10124000745F616363656C3E20543C7472617665C3
:101250006C5F616363656C3E0A00204500205A00A4
:1012600020590020204D3230312058004D617869DE
:101270006D756D20416363656C65726174696F6E35
:101280002028756E6974732F7332293A0A0020453D
:1012900000205A0020590020204D323033205800C1
:1012A0004D6178696D756D20666565647261746500
:1012B000732028756E6974732F73293A0A0053746A
:1012C0006570732070657220756E69743A0A00202B
:1012D00020473231202020203B20556E6974732036
:1012E000696E206D6D0048617264636F646564208F
:1012F00044656661756C742053657474696E6773B8
:10130000204C6F616465640A0028230000282300D4
:101310000064000000E8030000000096430000960F
:101320004300000041000020420000C9420000C903
:10133000420000C8440000D243290A0020627974A8
:1013400065733B2063726320002073746F72656461
:101350002073657474696E67732072657472696551
:10136000766564202800202863616C63756C617465
:10137000656429210A0020213D2000454550524F37
:101380004D20435243206D69736D61746368202D55
:10139000202873746F7265642920002053697A6570
:1013A0003A2000496E6465783A2000204D61726CE5
:1013B000696E3D563634290A0028454550524F4D36
:1013C0003D00454550524F4D2076657273696F6EF2
:1013D000206D69736D617463682000290A002062C2
:1013E000797465733B20637263200053657474697C
:1013F0006E67732053746F726564202800454550F2
:10140000524F4D206461746173697A652065727210
:101410006F722E0A0050726F62696E672066616992
:101420006C65640A005761726E696E673A20486F96
:101430006D696E672042756D702044697669736FBF
:1014400072203C20310A0002020420666972737423
:101450000A005A0059005800486F6D65200020743A
:101460006F6F206C6F6E6720657874727573696F2B
:101470006E2070726576656E7465640A0020636F15
:101480006C6420657874727573696F6E2070726514
:1014900076656E7465640A0020453A00205A3A0069
:1014A00020593A00583A000000F0410000F0410095
:1014B000000041FF01010000A0400000A04000002A
:1014C0000040000025430000454300002143000088
:1014D00040C000003E4300001F43000022430000C4
:1014E0003E4300001F43000040C00000E0C0000079
:1014F00000C020746F6F206C6F6E67206578747207
:101500007573696F6E2070726576656E7465640AB6
:101510000020636F6C6420657874727573696F6EF8
:101520002070726576656E7465640A006275737901
:101530003A2070617573656420666F7220696E7001
:1015400075740A00627573793A2070617573656409
:1015500020666F7220757365720A00627573793A3E
:101560002070726F63657373696E670A004D313165
:10157000372050726F62652073756363657373669D
:10158000756C0A0020496E76616C69642065787418
:1015900072756465722000205A3A200020593A2062
:1015A0000042656420583A200050726F6265205AEC
:1015B000204F66667365743A20003F5A206F757439
:1015C000206F662072616E676520282D3220746F4F
:1015D0002035290A00556E6B6E6F776E20636F6D34
:1015E0006D616E643A202200454550524F4D204FA8
:1015F0004B0A004543484F00494E464F0045525262
:101600004F52530044525952554E00434F4D4D5581
:101610004E49434154494F4E006F666600F315F83A
:1016200015FD1504160B1644454255473A00205A3D
:1016300000205900580020204D61783A2000205A9F
:1016400000205900580020204D696E3A2000536F49
:10165000667420656E6473746F70733A2000256938
:10166000730025696D202569730025696820256947
:101670006D20256973002569642025696820256926
:101680006D20256973002569792025696420256905
:10169000682025696D20256973005072696E742079
:1016A00074696D653A20004D3131332053002F2F7E
:1016B00020004361703A004D4F54494F4E5F4D4FEB
:1016C00044455300544845524D414C5F50524F548D
:1016D000454354494F4E004155544F5245504F5287
:1016E000545F53445F5354415455530050524F4D2F
:1016F00050545F535550504F525400454D4552473A
:10170000454E43595F504152534552004341534562
:101710005F4C494748545F4252494748544E4553ED
:101720005300544F47474C455F4C4947485453007A
:10173000534F4654574152455F504F574552004210
:1017400055494C445F50455243454E54004C455614
:10175000454C494E475F44415441005A5F50524FF7
:101760004245004155544F4C4556454C0050524956
:101770004E545F4A4F420050524F47524553530018
:101780004155544F5245504F52545F54454D5000AF
:10179000564F4C554D455452494300454550524FC4
:1017A0004D0053455249414C5F584F4E5F584F468C
:1017B00046004649524D574152455F4E414D453ACC
:1017C0004D61726C696E20204649524D5741524519
:1017D0005F56455253494F4E3A322E302E302E39F5
:1017E000312045585452554445525F545950453A5A
:1017F00048617264656E6564537465656C20534F0F
:10180000555243455F434F44455F55524C3A6874C7
:101810007470733A2F2F636F64652E616C65706806
:101820006F626A656374732E636F6D2F6469666699
:101830007573696F6E2F4D41524C494E2050524F77
:10184000544F434F4C5F56455253494F4E3A312EF9
:1018500030204D414348494E455F545950453A4C1C
:10186000756C7A426F74204D696E692045585452E8
:10187000554445525F434F554E543A3120555549D2
:10188000443A33353134383762362D636139612D4E
:10189000346331612D383736352D64363638623150
:1018A0006461363538350A00546F6F2066617220E6
:1018B00066726F6D207265666572656E6365207015
:1018C0006F696E740A0020284E6F74207965742049
:1018D0006D656173757265642900202041766572BB
:1018E000616765206D65617375726564206261630F
:1018F0006B6C61736820286D6D293A002020536D50
:101900006F6F7468696E6720286D6D293A202020FA
:1019100020202020202020202020202020205300B4
:1019200020204261636B6C61736820446973746149
:101930006E636520286D6D293A202020202020200C
:10194000200020202020202846312E30203D2066F7
:10195000756C6C2C2046302E30203D206E6F6E65ED
:10196000290A002020436F7272656374696F6E20CC
:10197000416D6F756E742F466164652D6F75743A95
:10198000202020202046006163746976653A0A00B1
:10199000696E004261636B6C61736820636F727281
:1019A000656374696F6E2069732000205A002050AF
:1019B0006F736974696F6E616C204572726F723AF1
:1019C0000A004E6F7A7A6C6520546970204F7574E6
:1019D00065722044696D656E73696F6E733A0A00B3
:1019E0002020546F703A2000202046726F6E743AA7
:1019F000200020204C6566743A20004261636B6CC5
:101A00006173683A0A00205A0043656E7465723A41
:101A10000A00202046726F6E743A200020204C6528
:101A200066743A20002020546F703A200053696495
:101A300065733A0A00426564204C6576656C696E90
:101A40006720004661696C656420746F20656E6173
:101A5000626C6520426564204C6576656C696E67D2
:101A60000A00426564204C6576656C20436F727293
:101A7000656374696F6E204D61747269783A000A0B
:101A80000A426564204C6576656C20436F7272650E
:101A90006374696F6E204D61747269783A00202B0F
:101AA000000A436F72726563746564204265642046
:101AB0004865696768742076732E204265642054F7
:101AC0006F706F6C6F67793A0A00202B000A4265CD
:101AD000642048656967687420546F706F6772612D
:101AE0007068793A0A2020202B2D2D2D2042414369
:101AF0004B202D2D2B0A2020207C20202020202050
:101B000020202020207C0A204C207C2020202028FF
:101B10002B29202020207C20520A2045207C2020B8
:101B20002020202020202020207C20490A20462020
:101B30007C20282D29204E20282B29207C20470A74
:101B40002054207C20202020202020202020207CA9
:101B500020480A2020207C20202020282D292020F9
:101B600020207C20540A2020207C2020202020209F
:101B700020202020207C0A2020204F2D2D2046527E
:101B80004F4E54202D2D2B0A2028302C30290A00AE
:101B90003474682070726F626520706F696E742C87
:101BA0002064697374616E63652066726F6D207066
:101BB0006C616E653A2000202844525952554E29D6
:101BC00000473239204175746F20426564204C65AE
:101BD00076656C696E67003F20284C2C522C462C91
:101BE0004229206F7574206F6620626F756E647372
:101BF0002E0A003F50726F626520706F696E7473B9
:101C00002028592920697320696D706C617573698A
:101C1000626C652028322D32292E0A003F50726FE7
:101C2000626520706F696E7473202858292069736B
:101C300020696D706C61757369626C652028322D46
:101C400032292E0A003F2856296572626F7365207B
:101C50006C6576656C20697320696D706C61757355
:101C600069626C652028302D34292E0A0041647683
:101C7000616E6365204B3D003F4B2076616C75655E
:101C8000206F7574206F662072616E676520283042
:101C90002D3130292E0A004D31313720486F742004
:101CA000456E642048656174696E672E2E2E0A4D5C
:101CB00031303420533137302054300A4732382005
:101CC0004F310A473120593235205A3130204635BC
:101CD0003030300A4D3130392052313730205430D5
:101CE0000A4D313137205265776970696E67206E11
:101CF0006F7A7A6C650A54300A473120583435209F
:101D0000593137322046353030300A4731205A3188
:101D10000A4D31303920523137300A47312058349A
:101D20003520593137322046343030300A4731209F
:101D300058343520593137322046343030300A4754
:101D40003120583435205931373220463430303044
:101D50000A47312058343520593137322046343043
:101D600030300A4731205834352059313732204637
:101D7000343030300A473120583435205931373229
:101D80002046343030300A4731205834352059311C
:101D900037322046343030300A473120583435202D
:101DA000593137322046343030300A4731205834E8
:101DB0003520593137322046343030300A4731200F
:101DC00058343520593137322046343030300A47C4
:101DD00031205834352059313732204634303030B4
:101DE0000A473120583435205931373220463430B3
:101DF00030300A4731205A31350A4D3130362053C0
:101E0000323535200A47302058302059300A4D31BC
:101E1000303920523136302054300A4D3130370AB3
:101E20000020466C6F773A200020643A0020693A1F
:101E30000020703A00204500205A00205900204D13
:101E4000393220580043290A0061626C65642028F9
:101E50006D696E2074656D70200064697300656E35
:101E600000436F6C642065787472756465732061DB
:101E700072652000205400205200416363656C6548
:101E8000726174696F6E3A205000496E76616C69B8
:101E9000642065787472756465720A0020643A0083
:101EA00020693A0020703A0047322F4733206261A0
:101EB0006420706172616D65746572730A0050729E
:101EC000696E7465722073746F70706564206475D8
:101ED0006520746F206572726F72732E2046697868
:101EE00020746865206572726F7220616E6420755F
:101EF0007365204D39393920746F207265737461B0
:101F000072742E202854656D7065726174757265E7
:101F10002069732072657365742E2053657420697F
:101F2000742061667465722072657374617274697D
:101F30006E67290A004E6F20436865636B73756D89
:101F40002077697468206C696E65206E756D6265B6
:101F5000722C204C617374204C696E653A200063CA
:101F60006865636B73756D206D69736D617463680B
:101F70002C204C617374204C696E653A20004C69CA
:101F80006E65204E756D626572206973206E6F7488
:101F9000204C617374204C696E65204E756D6265CE
:101FA000722B312C204C617374204C696E653A2081
:101FB000004D31313000526573656E643A20002067
:101FC00042002050006F6B00656E71756575656924
:101FD0006E67202200504944204175746F74756EFD
:101FE00065206661696C65642120426164206578C2
:101FF000747275646572206E756D6265720A006F29
:102000006B002020506C616E6E657242756666656D
:102010007242797465733A20002046726565204DDE
:10202000656D6F72793A2000436F6D70696C6564FD
:102030003A2046656220313920323031390A002099
:102040007C20417574686F723A2028416C65706815
:10205000204F626A6563747320496E632E2C204C96
:10206000756C7A426F7420476974205265706F7383
:1020700069746F7279290A0000204C6173742055CD
:102080007064617465643A2000322E302E302E392F
:10209000310A004D61726C696E0020536F6674776F
:1020A0006172652052657365740A0020576174631C
:1020B00068646F672052657365740A002042726F0E
:1020C000776E206F75742052657365740A00204521
:1020D000787465726E616C2052657365740A005085
:1020E0006F77657255700A0073746172740A0050DC
:1020F00072696E7465722068616C7465642E206B01
:10210000696C6C28292063616C6C6564210A004B42
:10211000494C4C2063617573656420627920746F4B
:102120006F206D75636820696E61637469766520E0
:1021300074696D65202D2063757272656E742063FD
:102140006F6D6D616E643A20004D3132310A473057
:10215000205A31300A4732382058302059300A4747
:1021600031320A4D31303920523136300A4D313159
:10217000372050726F62696E67206265640070720A
:102180006F62655F7265776970650050726F626932
:102190006E67206661696C6564004D31313720429D
:1021A0006564206C6576656C696E67206661696C34
:1021B00065642E0A4730205A31300A4730204530B6
:1021C0000A4D3330302050323520533838300A4DE4
:1021D000333030205035302053300A4D33303020EA
:1021E00050323520533838300A4D33303020503596
:1021F000302053300A4D33303020503235205338A0
:1022000038300A47342053310070726F62655F6660
:1022100061696C65640050726F74656374656420F5
:1022200050696E0A0025301D0C1E282924311C0B14
:10223000184527232F1B0A174443222B1A41420417
:102240003803FF36040806060001CB15CE15AB1A7D
:10225000FC691A9211241FBECFEFD1E2DEBFCDBFC1
:1022600000E00CBF13E0A0E0B2E0E4E3FFE601E031
:102270000BBF02C007900D92A038B107D9F72FE02D
:10228000A0E8B3E001C01D92A831B207E1F711E167
:10229000CAE2D1E100E006C021970109802FFE01CA
:1022A0000E942FB0C532D10780E00807A9F766D495
:1022B0000C9498B70C9400001F920F920FB60F92D7
:1022C00011242F933F938F939F93AF93BF9380914C
:1022D000810390918203A0918303B0918403309194
:1022E000800323E0230F2D3720F40196A11DB11D9B
:1022F00005C026E8230F0296A11DB11D209380037F
:102300008093810390938203A0938303B09384030B
:102310008091850390918603A0918703B0918803F3
:102320000196A11DB11D8093850390938603A09310
:102330008703B0938803BF91AF919F918F913F9195
:102340002F910F900FBE0F901F9018952FB7F894F4
:102350006091810370918203809183039091840343
:102360002FBF08953FB7F89480918503909186031D
:10237000A0918703B091880326B5A89B05C02F3F85
:1023800019F00196A11DB11D3FBFBA2FA92F982F9B
:102390008827820F911DA11DB11DBC01CD0142E016
:1023A000660F771F881F991F4A95D1F708958F925E
:1023B0009F92AF92BF92CF92DF92EF92FF926B010A
:1023C0007C01D0DF4B015C01C114D104E104F104B4
:1023D000F1F091D3C7DFDC01CB0188199909AA0973
:1023E000BB09883E9340A105B10570F321E0C21AF4
:1023F000D108E108F10888EE880E83E0981EA11C40
:10240000B11CC114D104E104F10421F7DDCFFF9028
:10241000EF90DF90CF90BF90AF909F908F900895F6
:10242000789484B5826084BD84B5816084BD85B5AF
:10243000826085BD85B5816085BDEEE6F0E0808176
:1024400081608083E1E8F0E0108280818260808397
:10245000808181608083E0E8F0E08081816080831A
:10246000E1EBF0E0808184608083E0EBF0E080814C
:1024700081608083E1E9F0E08081826080838081F7
:1024800081608083E0E9F0E0808181608083E1EA1F
:10249000F0E0808182608083808181608083E0EAD7
:1024A000F0E0808181608083E1E2F1E08081826000
:1024B0008083808181608083E0E2F1E080818160BF
:1024C0008083EAE7F0E0808184608083808182609D
:1024D0008083808181608083808180688083109286
:1024E000C10008951F93CF93DF93182FEB0161E094
:1024F00016D1209711F460E004C0CF3FD10531F42C
:1025000061E0812FDF91CF911F9145C1E12FF0E074
:10251000ED51FE4FE4914E2F50E0FA013197E23138
:10252000F10508F09DC08827EE58FF4F8F4F0C949F
:102530002FB084B5806884BDC7BD97C084B5806264
:1025400084BDC8BD92C08091800080688093800067
:10255000D0938900C093880088C0809180008062F9
:1025600080938000D0938B00C0938A007EC08091BE
:102570008000886080938000D0938D00C0938C0091
:1025800074C08091B00080688093B000C093B300A5
:102590006CC08091B00080628093B000C093B400A2
:1025A00064C080919000806880939000D0939900DF
:1025B000C09398005AC080919000806280939000F0
:1025C000D0939B00C0939A0050C080919000886087
:1025D00080939000D0939D00C0939C0046C0809152
:1025E000A00080688093A0008091A0008F7B8093E2
:1025F000A000D093A900C093A80037C08091A0008C
:1026000080628093A000D093AB00C093AA002DC03D
:102610008091A00088608093A000D093AD00C0930B
:10262000AC0023C080912001806880932001D0936A
:102630002901C093280119C08091200180628093F4
:102640002001D0932B01C0932A010FC0809120015B
:10265000886080932001D0932D01C0932C0105C088
:10266000C038D1050CF04CCF46CFDF91CF911F91F0
:10267000089590E0FC013197E231F10508F04EC079
:102680008827EC57FF4F8F4F0C942FB0809180001C
:102690008F7703C0809180008F7D809380000895A4
:1026A00080918000877FF9CF84B58F7702C084B591
:1026B0008F7D84BD08958091B0008F7703C0809195
:1026C000B0008F7D8093B0000895809190008F7747
:1026D00007C0809190008F7D03C080919000877F1C
:1026E0008093900008958091A0008F7707C080911B
:1026F000A0008F7D03C08091A000877F8093A00001
:102700000895809120018F7707C0809120018F7DEF
:1027100003C080912001877F809320010895CF938B
:10272000DF9390E0FC01E75DFD4F2491FC01E1594E
:10273000FD4F8491882361F190E0880F991FFC017F
:10274000E751FD4FC591D491FC01E153FD4FA59197
:10275000B491611109C09FB7F894888120958223B4
:102760008883EC912E230BC0623061F49FB7F894FC
:102770003881822F809583238883EC912E2B2C9394
:102780009FBF06C08FB7F894E8812E2B28838FBF98
:10279000DF91CF9108951F93CF93DF93282F30E0DF
:1027A000F901ED51FE4F8491F901E75DFD4FD491A0
:1027B000F901E159FD4FC491CC23C1F0162F8111CD
:1027C00058DFEC2FF0E0EE0FFF1FE153FD4FA59116
:1027D000B4918FB7F894111105C09C91ED2FE0953D
:1027E000E92302C0EC91ED2BEC938FBFDF91CF91E9
:1027F0001F910895CF93DF93282F30E0F901ED5119
:10280000FE4F8491F901E75DFD4FD491F901E15943
:10281000FD4FC491CC2389F081112BDFEC2FF0E028
:10282000EE0FFF1FEB54FD4FA591B491EC91ED23FA
:1028300081E090E021F480E002C080E090E0DF9150
:10284000CF91089508951F920F920FB60F92112401
:102850000BB60F922F933F934F935F936F937F939A
:102860008F939F93AF93BF93EF93FF93E0910402F5
:10287000F09105021995FF91EF91BF91AF919F9152
:102880008F917F916F915F914F913F912F910F9019
:102890000BBE0F900FBE0F901F9018951F920F92B6
:1028A0000FB60F9211240BB60F922F933F934F93B5
:1028B0005F936F937F938F939F93AF93BF93EF93A8
:1028C000FF93E0910602F09107021995FF91EF91B5
:1028D000BF91AF919F918F917F916F915F914F9138
:1028E0003F912F910F900BBE0F900FBE0F901F9036
:1028F00018951F920F920FB60F9211240BB60F92DC
:102900002F933F934F935F936F937F938F939F93F7
:10291000AF93BF93EF93FF93E0910802F091090208
:102920001995FF91EF91BF91AF919F918F917F91F9
:102930006F915F914F913F912F910F900BBE0F9030
:102940000FBE0F901F9018951F920F920FB60F9207
:1029500011240BB60F922F933F934F935F936F9376
:102960007F938F939F93AF93BF93EF93FF93E091E8
:102970000A02F0910B021995FF91EF91BF91AF916F
:102980009F918F917F916F915F914F913F912F9187
:102990000F900BBE0F900FBE0F901F9018951F92B7
:1029A0000F920FB60F9211240BB60F922F933F93F5
:1029B0004F935F936F937F938F939F93AF93BF9347
:1029C000EF93FF93E0910002F09101021995FF91BE
:1029D000EF91BF91AF919F918F917F916F915F9197
:1029E0004F913F912F910F900BBE0F900FBE0F9004
:1029F0001F9018951F920F920FB60F9211240BB6CD
:102A00000F922F933F934F935F936F937F938F9387
:102A10009F93AF93BF93EF93FF93E0910202F091E6
:102A200003021995FF91EF91BF91AF919F918F9103
:102A30007F916F915F914F913F912F910F900BBEBE
:102A40000F900FBE0F901F9018951F920F920FB608
:102A50000F9211240BB60F922F933F934F935F93D6
:102A60006F937F938F939F93AF93BF93EF93FF9356
:102A7000E0910C02F0910D021995FF91EF91BF9139
:102A8000AF919F918F917F916F915F914F913F9106
:102A90002F910F900BBE0F900FBE0F901F901895A7
:102AA0001F920F920FB60F9211240BB60F922F9315
:102AB0003F934F935F936F937F938F939F93AF93C6
:102AC000BF93EF93FF93E0910E02F0910F021995DF
:102AD000FF91EF91BF91AF919F918F917F916F91F6
:102AE0005F914F913F912F910F900BBE0F900FBEB2
:102AF0000F901F90189508954F925F926F927F925A
:102B0000AF92BF92CF92DF92EF92FF920F931F93FB
:102B1000CF93DF93CDB7DEB729013A019B01AC011A
:102B200024193509460957098A899B89AC89BD89C9
:102B3000BC01CD016A197B098C099D090E94CEAFA9
:102B4000A801970124193509460957090E9413B0B5
:102B5000CA01B9016A0D7B1D8C1D9D1DDF91CF91AE
:102B60001F910F91FF90EF90DF90CF90BF90AF90AB
:102B70007F906F905F904F900895089551DCFDDF36
:102B80000E9458ABC0E0D0E00E94E0AB2097E1F398
:102B90000E940000F9CF109289030895EEE8F3E057
:102BA000108214820895CF93C82F0E94002ECC2348
:102BB00049F024982C9A65E070E080E090E0F7DB23
:102BC000149A03C0249A2C981498CF91089580E009
:102BD000EACFCF92DF92EF92FF926B017C0183E309
:102BE000C816D104E104F10468F082E3C81AD108E0
:102BF000E108F10862E370E080E090E0D8DB0E9439
:102C00003C22EDCFC701B601D2DBFF90EF90DF9001
:102C1000CF900C943C22DC01FB01460F571FE417B8
:102C2000F507C1F081912D913C911197382798E0DB
:102C3000B901660F771F37FF06C09B0181E2282785
:102C400080E1382701C09B01915091F711963C9388
:102C50002E93E5CF0895CF93DF93FC018491EF018C
:102C60002196882319F087D2FE01F8CFDF91CF910A
:102C700008958AE093E0EFCF80E193E0ECCF0F93EB
:102C80001F93CF93DF931F921F92CDB7DEB7698357
:102C90007A83E1DF6981062F7A81172FF80181910C
:102CA0008F01882311F067D2F9CF0F900F90DF9139
:102CB000CF911F910F910895CF93DF93EB01CBDF5D
:102CC0006AE070E0CE01DF91CF9148C3CF92DF92EE
:102CD000EF92FF926A017B01BEDF4AE050E0C7013C
:102CE000B601FF90EF90DF90CF9027C3CF92DF9295
:102CF000EF92FF926A017B01AEDF42E050E0C70134
:102D0000B601FF90EF90DF90CF90B3C3CF92DF92E8
:102D1000EF92FF926A017B019EDF42E050E0C70123
:102D2000B601FF90EF90DF90CF90A3C3CF93DF93D6
:102D3000EB0191DF6AE070E0CE01DF91CF9123C318
:102D4000CF92DF92EF92FF926A017B0184DF4AE02B
:102D500050E0C701B601FF90EF90DF90CF900DC318
:102D6000811103C083E093E002C087E093E073CF5A
:102D7000F7DF8AE000C2CF93DF931F921F92CDB797
:102D8000DEB72091120F3091130FCE01019621155D
:102D9000310519F488519F4002C0821B930B9A831E
:102DA000898389819A810F900F90DF91CF91089547
:102DB00081E0089581E008958F929F92AF92BF9233
:102DC000CF92DF92EF92FF920F931F93CF93DF93F7
:102DD0001F921F92CDB7DEB76C0159018B017B01A9
:102DE000E40EF51E0E151F0561F1F601808091803D
:102DF000F80161918F016983C4016A830E9482B7DF
:102E00006A81681779F0C4010E948AB7C4010E94E0
:102E100082B79981891731F02CDF87E193E01BDFBE
:102E200081E010C041E050E0BE016F5F7F4FC501FF
:102E3000F2DEF601408151814F5F5F4F5183408345
:102E4000D1CF80E00F900F90DF91CF911F910F9124
:102E5000FF90EF90DF90CF90BF90AF909F908F90BA
:102E600008958F929F92AF92BF92CF92DF92EF928E
:102E7000FF920F93CF93DF931F92CDB7DEB75C0124
:102E80006B017A014901F501808191810E9482B72D
:102E90008983002311F0F601808341E050E0BE01F8
:102EA0006F5F7F4FC401B7DEF501408151814F5FF5
:102EB0005F4F51834083FFEFCF1ADF0A81E0E81AAA
:102EC000F10809F780E00F90DF91CF910F91FF900B
:102ED000EF90DF90CF90BF90AF909F908F9008952C
:102EE00098E288E10FB6F894A895809360000FBE31
:102EF0009093600008951F920F920FB60F921124C5
:102F00000BB60F920F931F932F933F934F935F93A3
:102F10006F937F938F939F93AF93BF93CF93DF93E1
:102F2000EF93FF930091B903D091B80311E01D0F07
:102F30001F77C091C60090919403492F092E000C71
:102F4000550B660B770B4C30510508F046C0FA0163
:102F50008827EA56FF4F8F4F0C942FB0CD3441F0A5
:102F6000CE34B9F481E005C0CA3330F0CD3471F508
:102F700082E0809394034AC0C03308F047C0C03257
:102F800009F444C0CD3211F541C0C13329F0C43336
:102F900029F0C032D9F43AC083E0EBCF88E0E9CF22
:102FA000C03321F0C13391F486E0E3CF84E0E1CF78
:102FB000C83361F485E0DDCFC23341F487E0D9CF77
:102FC000C13321F489E0D5CFC03311F08BE0D1CFEC
:102FD0008AE0CFCFCA30D1F417C0CA30B9F480919B
:102FE0004304882389F0973049F09A3059F095309E
:102FF00059F410925B021092110F06C081E0809389
:10300000440402C00E9412AA10929403101731F0D7
:10301000ED2FF0E0E854FC4FC283D12FD093B803DA
:10302000FF91EF91DF91CF91BF91AF919F918F91E0
:103030007F916F915F914F913F912F911F910F91D0
:103040000F900BBE0F900FBE0F901F9018951F9200
:103050000F920FB60F9211240BB60F922F938F93EE
:103060009F93EF93FF9380919703209196032817E6
:1030700091F0E82FF0E0EA56FC4F92818F5F8F715C
:103080009093C600809397039091C00090649093B2
:10309000C000281305C08091C1008F7D8093C100BE
:1030A000FF91EF919F918F912F910F900BBE0F90F9
:1030B0000FBE0F901F9018959B01AC011092C0009D
:1030C000211581EE380741055105C1F08091C000FE
:1030D00082608093C00060E079E08DE390E00E9420
:1030E00013B0CA01B901615071098109910922E047
:1030F00030E040E050E00E9413B002C020E130E038
:103100003093C5002093C4008091C10080618093FA
:10311000C1008091C10088608093C1008091C1008E
:1031200080688093C1008091C1008F7D8093C10031
:103130001092950308958091B8039091B90389176F
:1031400059F0E92FF0E0E854FC4F82819F5F9F77B0
:103150009093B90390E008958FEF9FEF0895E8EB07
:10316000F3E0808181830895E8EBF3E08081918131
:10317000891B8F77089591E0909395039091C100FA
:1031800095FD04C09091C00095FD40C0209196032C
:103190002F5F2F710FB607FC34C09091970329134E
:1031A00022C09091C00095FF1DC09091970340915F
:1031B0009603491791F0E92FF0E0EA56FC4F32816F
:1031C0009F5F9F713093C600909397033091C0002A
:1031D00030643093C000491305C09091C1009F7DB9
:1031E0009093C100DACFE0919603F0E0EA56FC4FED
:1031F0008283209396038091C10080628093C100F6
:103200000895909197032913EECFFBCF8093C600CA
:103210008091C00080648093C00008958DE0ABDF92
:103220008AE0A9CFCF93DF93EC018991882311F035
:10323000A2DFFBCFDF91CF91F1CF8F929F92AF9220
:10324000BF92EF92FF921F93CF93DF93CDB7DEB77C
:10325000A0970FB6F894DEBF0FBECDBF6115710504
:103260008105910579F110E0842E912CA12CB12CCF
:10327000EE24E394F12CEC0EFD1EE10EF11C17FD83
:10328000FA94A50194010E94F1AFF7016083B9019E
:10329000CA011F5F611571058105910549F711503C
:1032A00010F1E1E0F0E0EC0FFD1FE10FF11D17FD63
:1032B000FA9580818A3010F097E301C090E3890F7E
:1032C0005ADFEDCF80E3A0960FB6F894DEBF0FBEB5
:1032D000CDBFDF91CF911F91FF90EF90BF90AF9046
:1032E0009F908F9048CFA0960FB6F894DEBF0FBE88
:1032F000CDBFDF91CF911F91FF90EF90BF90AF9026
:103300009F908F900895CF92DF92EF92FF926B0182
:103310007C0197FF0AC08DE22EDFF094E094D094F8
:10332000C094C11CD11CE11CF11C4AE0C701B601CC
:10333000FF90EF90DF90CF9080CF4115510511F4B1
:10334000862F19CF4A30510509F4DDCF76CFAB0176
:10335000682F880F770B880B990BEFCFAB01BC015F
:10336000990F880B990BE9CFAB01BC01990F880B22
:10337000990BE3DF53CFE1DF51CF4115510511F434
:10338000862FF9CE5ACFAB01BC0180E090E0F5CF9B
:103390008F929F92AF92BF92CF92DF92EF92FF9265
:1033A000CF936B017C01B42E20E030E0A9010E9494
:1033B000C6AC87FF06C08DE2DEDEF7FAF094F7F8C0
:1033C000F094C0E060E070E080E09FE3CB1541F056
:1033D0002DEC3CEC4CEC5DE30E9404AFCF5FF6CFEC
:1033E0009B01AC01C701B6010E94EDAB6B017C01F2
:1033F0000E943AAD4B015C014AE01FDFCC2379F11A
:10340000C501B4010E9466AD9B01AC01C701B601C4
:103410000E94ECAB6B017C018EE2ADDE20E030E07F
:1034200040E251E4C701B6010E9404AF4B015C01C8
:103430000E9435AD6B01770FEE08FF08C701B6019A
:1034400062DFC701B6010E9468AD9B01AC01C501F6
:10345000B4010E94ECAB6B017C01C150F9F6CF9135
:10346000FF90EF90DF90CF90BF90AF909F908F90A4
:1034700008958ECFCF92DF92EF92FF920F931F931A
:103480000E94A61100913E0410913F042091400437
:10349000309141046B017C01C01AD10AE20AF30A9F
:1034A000F7FC52C08B019C010C53164F2F4F3F4F1E
:1034B00000933E0410933F04209340043093410452
:1034C000079B39C0069B37C0059B35C02091C504BA
:1034D000211131C0049B2FC000913A0410913B048C
:1034E00020913C0430913D04011511052105310561
:1034F00071F0DC01CB01801B910BA20BB30B80564A
:103500009A4EA109B109B7FF02C068E701C060E0A7
:1035100060934204809102016111809588708093CC
:10352000000170E086E01F910F91FF90EF90DF9017
:10353000CF900C94721260933A0470933B04809382
:103540003C0490933D04C8CF1F910F91FF90EF90E2
:10355000DF90CF90089581E0809343040895909187
:1035600040068917D1F00E941459809140068823A3
:1035700059F043EB55E06FEA75E08BEA95E00E9465
:10358000D7571092400607C081E0809340068BEA2F
:1035900095E00E9445580C94B04C089580E0DFDF20
:1035A0008CE196E00C947FA50F931F93CF93DF934C
:1035B0001F92CDB7DEB78C0181E493E069834BDBCA
:1035C000C80149DB6981662339F08AE00F90DF91F9
:1035D000CF911F910F91CFCD0F90DF91CF911F9180
:1035E0000F91089561E088E393E0DECF61E081E32D
:1035F00093E0DACFEF92FF920F931F93CF93DF9375
:103600001F92CDB7DEB78C017B0180E24983B3DD29
:1036100049814F3F11F084E501C082E4ACDD8AE3CB
:10362000AADDF801608171818281938142E050E0DE
:1036300020DFF701408151816281738183E593E04E
:1036400055DB62E070E080E090E00F90DF91CF9179
:103650001F910F91FF90EF900C94D711811109C029
:10366000CB016F3F710519F010F08FEF90E0809360
:10367000CE04089597FF03C08091C50404C0FC01E7
:10368000E657FB4F808190E008952F923F924F9232
:103690005F926F927F928F929F92AF92BF92CF92E2
:1036A000DF92EF92FF92CF93DF9300D01F92CDB7BE
:1036B000DEB76090CF047090D0048090D3049090D7
:1036C000D404A090D504B090D604B301072C000C0C
:1036D000880B990B0E9468ADA50194010E94ECAB88
:1036E0006B017C0120ED3CEC4CE45DE36091AB04AC
:1036F0007091AC048091AD049091AE040E9404AF2F
:103700001B012C01209176043091770440917804BC
:1037100050917904C501B4010E94ECAB9B01AC014E
:10372000C201B1010E9404AF1B012C0123E333E36A
:1037300043E75FE3609172047091730480917404B5
:10374000909175040E9404AF9B01AC01C201B101CC
:103750000E94EDAB69837A838B839C8360937204B0
:10376000709373048093740490937504809276042C
:1037700090927704A0927804B092790420E030E02F
:1037800040E251E4C701B6010E94C9AE181654F4D4
:1037900081E080936904412C512C2FE7622E23E4B1
:1037A000722EC0C020E030E040E251ECC701B6010B
:1037B0000E94C6AC87FD02C0672839F481E080937F
:1037C0006904412C512C3201ADC0809169048823D9
:1037D00051F01092650410926604109267041092E2
:1037E0006804109269042091650430916604409148
:1037F000670450916804C701B6010E94EDAB4B010C
:103800005C016093650470936604809367049093F1
:1038100068042091A3043091A4044091A504509120
:10382000A604C701B6010E9404AF2B013C016093BE
:103830006A0470936B0480936C0490936D042091E0
:10384000A7043091A8044091A9045091AA04C5018D
:10385000B4010E9404AF9B01AC0160936E047093AD
:103860006F048093700490937104C301B2010E94AD
:10387000EDAB29813A814B815C810E94ECAB2B013D
:103880003C0120E030E04FE753E40E94C9AE20E065
:1038900030E0A9011816DCF4C701B6010E94C9AED8
:1038A0001816B4F5A7019601C501B4010E94ECAB4E
:1038B0006093650470936604809367049093680432
:1038C000412C512C9FE7692E93E4792E2BC0C30124
:1038D000B2010E94C6AC87FF25C020E030E0A901FC
:1038E000C701B6010E94C6AC87FF19C0A7019601A7
:1038F000C501B4010E94ECAB60936504709366044B
:103900008093670490936804412C512C32010AC0C3
:10391000412C512C8FE7682E83E4782E03C0412C74
:10392000512C3201C301B2010F900F900F900F90F4
:10393000DF91CF91FF90EF90DF90CF90BF90AF904D
:103940009F908F907F906F905F904F903F902F90BF
:1039500008954F925F926F927F928F929F92AF9253
:10396000BF92CF92DF92EF92FF92CF93DF93CDB7CA
:10397000DEB72C970FB6F894DEBF0FBECDBF809197
:10398000CA049091CB04A091CC04B091CD0489835A
:103990009A83AB83BC836091C6047091C704072EE1
:1039A000000C880B990B0E9468AD29813A814B81EC
:1039B0005C810E94ECAB6B017C0120916104309131
:1039C000620440916304509164040E94EDAB4B018A
:1039D0005C0160936104709362048093630490932C
:1039E00064042091B1043091B2044091B304509129
:1039F000B404C701B6010E9404AF6D837E838F8338
:103A0000988760935504709356048093570490935D
:103A100058042091B5043091B6044091B7045091F8
:103A2000B804C501B4010E9404AF69877A878B8707
:103A30009C876093590470935A0480935B0490931D
:103A40005C0420ED3CEC4CE45DE36091B9047091C2
:103A5000BA048091BB049091BC040E9404AF2B0176
:103A60003C012091510430915204409153045091F3
:103A7000540469817A818B819C810E94ECAB9B010B
:103A8000AC01C301B2010E9404AF2B013C0123E34E
:103A900033E343E75FE360915D0470915E048091DE
:103AA0005F04909160040E9404AF9B01AC01C301CC
:103AB000B2010E94EDAB2B013C0160935D04709359
:103AC0005E0480935F049093600489819A81AB8146
:103AD000BC818093510490935204A0935304B093FB
:103AE000540429853A854B855C856D817E818F8163
:103AF00098850E94EDABA30192010E94ECAB2B01D3
:103B00003C0120E030E04FE753E40E94C9AE20E0E2
:103B100030E0A9011816DCF4C701B6010E94C9AE55
:103B20001816B4F5A7019601C501B4010E94ECABCB
:103B300060936104709362048093630490936404BF
:103B4000412C512C9FE7692E93E4792E2BC0C301A1
:103B5000B2010E94C6AC87FF25C020E030E0A90179
:103B6000C701B6010E94C6AC87FF19C0A701960124
:103B7000C501B4010E94ECAB6093610470936204D0
:103B80008093630490936404412C512C32010AC049
:103B9000412C512C8FE7682E83E4782E03C0412CF2
:103BA000512C3201C301B2012C960FB6F894DEBF3E
:103BB0000FBECDBFDF91CF91FF90EF90DF90CF9000
:103BC000BF90AF909F908F907F906F905F904F903D
:103BD00008954F925F926F927F928F929F92AF92D1
:103BE000BF92CF92DF92EF92FF920F931F93CF93EA
:103BF000DF933C01C62F662389F03ED86AE070E06F
:103C00008C2F90E0ABDB86E993E025D880E090E054
:103C10000E9457AA60E070E0CB017AC0B0E2A0E059
:103C20006A2F70E0AB014B0F511D559547954A1710
:103C300011F04B130BC0E1EAF7E065917491072E88
:103C4000000C880B990B0E9468AD62C0CA010197F5
:103C5000880F991F880F991FFC01ED5DF84F0591A2
:103C600014919A01220F331F220F331FF901ED5DCA
:103C7000F84FC591D4916016710614F4B42FD2CFC9
:103C8000A42FC615D7050CF4CBCF8B5D984FFC0144
:103C9000E590F490F901EB5DF84FC590D490B70131
:103CA0000F2C000C880B990B0E9468AD4B015C0136
:103CB000B301601B710B072E000C880B990B0E943F
:103CC00068AD2B013C01B6016E197F09072E000C6F
:103CD000880B990B0E9468AD9B01AC01C301B20136
:103CE0000E9404AF6B017C01C01BD10BBE01DD0F34
:103CF000880B990B0E9468AD9B01AC01C701B6010E
:103D00000E94CDAC9B01AC01C501B4010E94EDAB9A
:103D1000DF91CF911F910F91FF90EF90DF90CF90A7
:103D2000BF90AF909F908F907F906F905F904F90DB
:103D300008954F925F926F927F928F929F92AF926F
:103D4000BF92CF92DF92EF92FF920F931F93CF9388
:103D5000DF933C01BAE3A0E06A2F70E0AB014B0FA8
:103D6000511D559547954A1711F04B130BC0E1E2D1
:103D7000F7E065917491072E000C880B990B0E9457
:103D800068AD62C0CA010197880F991F880F991FFB
:103D9000FC01E55CF94F059114919A01220F331F44
:103DA000220F331FF901E55CF94FC591D4916016DC
:103DB000710614F4B42FD2CFA42FC615D7050CF476
:103DC000CBCF835C994FFC01E590F490F901E35C63
:103DD000F94FC590D490B7010F2C000C880B990BAC
:103DE0000E9468AD4B015C01B301601B710B072E93
:103DF000000C880B990B0E9468AD2B013C01B601A9
:103E00006E197F09072E000C880B990B0E9468AD74
:103E10009B01AC01C301B2010E9404AF6B017C01A4
:103E2000C01BD10BBE01DD0F880B990B0E9468AD42
:103E30009B01AC01C701B6010E94CDAC9B01AC0156
:103E4000C501B4010E94EDABDF91CF911F910F919D
:103E5000FF90EF90DF90CF90BF90AF909F908F90AA
:103E60007F906F905F904F90089560E08091D104B3
:103E70009091D204AEDE6093D3047093D404809307
:103E8000D5049093D6048091C8049091C90451DF61
:103E90006093CA047093CB048093CC049093CD04B8
:103EA000A89510929B04089567707727E82F880FD4
:103EB000FF0BED51FE4FE4918E2F90E0FC01379700
:103EC000EC30F10508F58827EE55FF4F8F4F0C9425
:103ED0002FB08091B100887F682B6093B100089566
:103EE00080919100887F682B609391000895809164
:103EF000A100887F682B6093A10008958091210123
:103F0000887F682B6093210108956D9A7598809140
:103F10000101806180930101809102018071809391
:103F2000000180910101886080930101809102016C
:103F30008870809300019D9AA5988091010180620C
:103F40008093010164E070E088E0AEDF80910101C0
:103F500088608093010164E070E086E0A5DF87ED72
:103F600080937A0010927E0010927D0080917E00F6
:103F7000816080937E0080917E00846080937E00CB
:103F800080E888BD80916E00846080936E006AEF47
:103F900070E080E090E00E94D71185E090E090937F
:103FA0008C0480938B0460E080911702909118023A
:103FB00010DE20E030E040EA50E40E94C6AC87FF0B
:103FC0000AC08091170290911802409790931802AE
:103FD00080931702E8CF81E391E0909316028093DB
:103FE000150260E080918D0490918E04F2DD20E056
:103FF00030E848E953E40E94C9AE181654F48091A1
:104000008D0490918E04409690938E0480938D043D
:10401000E8CF80911B0290911C028BDE20E030E003
:1040200040EA50E40E94C6AC87FF0AC080911B02A0
:1040300090911C02409790931C0280931B02E9CF41
:104040008091C3049091C40474DE20E030E046E126
:1040500053E40E94C9AE181654F48091C3049091A1
:10406000C40440969093C4048093C304E9CF089598
:10407000CF92DF92EF92FF928091CF049091D00483
:104080000097B9F0C090D304D090D404E090D50448
:10409000F090D6040D97BC01990F880B990B0E94E4
:1040A00068AD9B01AC01C701B6010E94C6AC87FD9B
:1040B00009C010929D0410929E0410929F041092C9
:1040C000A0041EC020E030E040E050E4C701B6018B
:1040D0000E94EDAB0E943AAD7093A2046093A104DC
:1040E0000E94A611DC01CB01805E914BAF4FBF4F08
:1040F00080939D0490939E04A0939F04B093A0048A
:10410000FF90EF90DF90CF900895CF92DF92EF92E3
:10411000FF928091C6049091C7040097B9F0C090B7
:10412000CA04D090CB04E090CC04F090CD04089762
:10413000BC01990F880B990B0E9468AD9B01AC01E3
:10414000C701B6010E94C6AC87FD09C01092BD042C
:104150001092BE041092BF041092C0041EC020E052
:1041600030E040E050E4C701B6010E94EDAB0E9490
:104170003AAD7093C2046093C1040E94A611DC01A1
:10418000CB01805A9541AF4FBF4F8093BD049093B0
:10419000BE04A093BF04B093C004FF90EF90DF90E3
:1041A000CF90089580911502909116020F971816DE
:1041B000190614F480E090E09093D0048093CF042B
:1041C00080E056DF1092C7041092C6049EDF8091F3
:1041D0001502909116020F971816190614F480E034
:1041E00090E09093D0048093CF0480E041DF109260
:1041F0008A0475981092C7041092C6041092C504E0
:10420000A5980895EF92FF920F931F93CF93C82F15
:104210007B018A0180915C028823B1F00E943C16E8
:10422000C7010E942B1682E694E00E942B16C7FD60
:1042300007C06AE070E08C2FCC0F990B95D804C0B2
:104240008DE594E00E942B1680917A0481110DC0B7
:1042500010925C0281E080937A04C801CF911F9193
:104260000F91FF90EF900C9457AACF911F910F914F
:10427000FF90EF9097CF8F3F19F04CE354E002C0CE
:104280004CE454E06AE274E0BDCF8F3F19F049E09E
:1042900054E002C049E154E067EF73E0B3CF2F92DE
:1042A0003F924F925F926F927F928F929F92AF92C6
:1042B000BF92CF92DF92EF92FF920F931F93CF9313
:1042C000DF9300D01F92CDB7DEB75C017A8369839C
:1042D0004A01170107FD05C0802F002E000C990B25
:1042E00002C081E090E0F9014080518062807380DB
:1042F0009C01220F331F220F331F3C832B83275B2C
:104300003B4F7901A3019201F701608171818281A4
:1043100093810E94C6AC882391F0F70140825182BC
:104320006282738211E020E030E0A901C301B20192
:104330000E94C9AE18160CF010E0F5011083F501CB
:1043400080818230D1F0833009F45EC0813009F081
:104350007CC0EB81FC81E75BFB4F20813181428196
:104360005381F40160817181828193810E94C6AC86
:1043700087FD6BC082E0F50180832B813C81275B48
:104380003B4F7901B60180E090E00E9466AD9B0151
:10439000AC01F70160817181828193810E94ECAB55
:1043A0009B01AC01F40160817181828193810E9443
:1043B000C9AE87FD16C00E94A6116B017C01910158
:1043C000A8EEB3E00E9437B0DC01CB018C0D9D1D3F
:1043D000AE1DBF1DE981FA8180839183A283B383DF
:1043E00034C00E94A611E981FA81C080D180E280A8
:1043F000F380DC01CB018C199D09AE09BF09B7FD23
:1044000024C083E0F50180830F3F19F04FE653E0AD
:1044100002C042E853E06FE573E0802F0F900F90E9
:104420000F900F90DF91CF911F910F91FF90EF9020
:10443000DF90CF90BF90AF909F908F907F906F90C4
:104440005F904F903F902F90DDCE0F900F900F9088
:104450000F90DF91CF911F910F91FF90EF90DF9020
:10446000CF90BF90AF909F908F907F906F905F9014
:104470004F903F902F9008958F929F92AF92BF924E
:10448000CF92DF92EF92FF920F93CF93DF9300D002
:104490001F92CDB7DEB78091440481111DC1809178
:1044A0009B04811110C00F900F900F900F90DF911F
:1044B000CF910F91FF90EF90DF90CF90BF90AF9092
:1044C0009F908F900895D1DC0E94A6114B015C0152
:1044D0008091130290911402181619060CF001C174
:1044E000019790931402809313026091CF0470910E
:1044F000D004072E000C880B990B0E9468AD6983CD
:104500007A838B839C834EE1C42ED12C5FE0E52E11
:10451000F12C00E09E012F5F3F4F43ED54E065E832
:1045200074E089E894E0BBDEC090D304D090D4045A
:10453000E090D504F090D60480918B0490918C0487
:10454000BC01990F880B990B0E9468AD9B01AC01CF
:10455000C701B6010E94C9AE1816CCF460911502CD
:1045600070911602072E000C880B990B0E9468AD03
:104570009B01AC01C701B6010E94C6AC87FF07C012
:1045800080E083D80E9435AD7595679501C060E0E5
:1045900060938A0480919D0490919E04A0919F0451
:1045A000B091A0040097A105B10521F1A5019401E6
:1045B000281B390B4A0B5B0B57FD1CC06091A104F3
:1045C0007091A20480E090E00E9466AD9B01AC0176
:1045D0006091D3047091D4048091D5049091D60455
:1045E0000E94C6AC87FF9EC045EE53E066ED73E0C7
:1045F00080E008DE8091BD049091BE04A091BF04CC
:10460000B091C0040097A105B10509F1881A990A73
:10461000AA0ABB0AB7FC1BC06091C1047091C20416
:1046200080E090E00E9466AD2091CA043091CB04F6
:104630004091CC045091CD040E94C9AE18160CF0E4
:104640006FC043EC53E064EB73E08FEFDBDD609110
:10465000C6047091C704072E000C880B990B0E94AA
:1046600068AD69837A838B839C839AE0C92ED12CB1
:104670002FE0E22EF12C0FEF9E012F5F3F4F4AEC0F
:1046800054E060E874E084E894E009DE8090CA04B5
:104690009090CB04A090CC04B090CD0420E030E00A
:1046A00040EA50E4C501B4010E94C9AE87FD10C0C4
:1046B00020E030E046E153E4C501B4010E94C6ACFD
:1046C000181634F046D90E9435AD7595679501C02E
:1046D00060E06093C504E7CE80E090E00E9457AAB6
:1046E000DECEC090D304D090D404E090D504F090F6
:1046F000D60420E030E848E953E4C701B6010E943F
:10470000C9AE181694F020E030E040EA50E4C7014A
:10471000B6010E94C6AC87FFE8CE80E0B6DDE5CEEC
:10472000F4DC95CF80E0A4DC65CF80E0A4DDC09010
:10473000D304D090D404E090D504F090D604E3CF15
:1047400080918F04909190049093D2048093D1042F
:104750008091AF049091B0049093C9048093C804F1
:1047600081E080939B0408951F93CF93DF93809102
:104770009B04811101C0E4DF8CE0EFE8F4E0DF018D
:104780001D928A95E9F71092B0041092AF04C0917F
:10479000D104D091D204D195C195D1098091CF0493
:1047A0009091D00411E0181619062CF080918A041B
:1047B000811101C010E080918D0490918E0491953B
:1047C000819591098C179D0714F480E054DD809148
:1047D000170290911802919581959109C817D907F0
:1047E00024F4112311F080E050DD8091C6049091F3
:1047F000C704C1E0181619062CF08091C504811178
:1048000001C0C0E02091C8043091C9048091C30464
:104810009091C4048217930714F08FEF2CDD209140
:104820001B0230911C028091C8049091C904821728
:1048300093073CF0CC2329F08FEFDF91CF911F91AC
:1048400024CDDF91CF911F9108950F930FB70F9350
:1048500000916E000B7F00936E0078940F930BB75E
:104860000F930CB70F921F922F933F934F935F9329
:104870006F937F938F939F93AF93BF93EF93FF9328
:104880001124C7D0FF91EF91BF91AF919F918F916C
:104890007F916F915F914F913F912F911F900F905A
:1048A0000CBF0F910BBF0F910460F89400936E0042
:1048B0000F910FBF0F911895CF93809112028F37F0
:1048C00090F08F5790918A0490934804992311F0A7
:1048D000759A01C075989091C504909347049923E7
:1048E00059F0A59A0AC090914804891708F0759864
:1048F00090914704891708F0A598805F8093120271
:104900009091460481E089278093460480911102AA
:1049100085301CF4C1E0C80F01C0C0E08230A1F1B5
:1049200084F4882329F1813009F062C010927B0061
:1049300080E480937C0080917A00806480937A0088
:1049400057C0843009F43EC094F1853009F050C05E
:1049500090914504911102C08093450480914504D3
:10496000815080934504882309F442C0C5E040C0CB
:10497000809110028F5F80311CF48093100238C048
:1049800010921002F1DE34C080917A0086FD2DC0B5
:10499000809178009091790020918F04309190045B
:1049A000820F931F9093900480938F0421C01092E4
:1049B0007B0082E480937C0080917A008064809305
:1049C0007A0016C080917A0086FD11C0809178002F
:1049D000909179002091AF043091B004820F931F21
:1049E0009093B0048093AF0403C0C2E001C0C4E060
:1049F000C09311020E944B2F8091BA069091BB0682
:104A0000009729F001979093BB068093BA06CF9147
:104A1000089552CF1F93CF93DF93CDB7DEB728977A
:104A20000FB6F894DEBF0FBECDBF182F6091CF0434
:104A30007091D004072E000C880B990B0E9468AD72
:104A400069837A838B839C838091D3049091D4046F
:104A5000A091D504B091D6048D839E83AF83B8878F
:104A60004DEFBE016F5F7F4FCE0105960E94FA1A8F
:104A70006091C6047091C704072E000C880B990B37
:104A80000E9468AD69837A838B839C838091CA047A
:104A90009091CB04A091CC04B091CD048D839E83E2
:104AA000AF83B8874FEFBE016F5F7F4FCE01059692
:104AB0000E94FA1A8BE593E00E942B16812F90E05A
:104AC0000E943A1B6AE070E00E94AE1986E593E00E
:104AD0000E942B168091C5046AE070E090E00E946D
:104AE000AE1928960FB6F894DEBF0FBECDBFDF918A
:104AF000CF911F9108952F923F924F925F926F92A4
:104B00007F928F929F92AF92BF92CF92DF92EF925D
:104B1000FF920F931F93CF93DF93CDB7DEB7C155AD
:104B2000D1090FB6F894DEBF0FBECDBF62969FAF1E
:104B30008EAF6297162F4BAB2C962FAF2C970E94FF
:104B4000A611688B798B8A8B9B8B17FD04C0B4E10F
:104B5000CB2ED12C03C0ACE3CA2ED12C6296AEADC5
:104B6000BFAD62972D913D914D915C912FA738ABD0
:104B700049AB5AAB17FDB3C4E12E012E000CFF0860
:104B8000F701EE0FFF1FEB5EFD4F608171816F50EB
:104B90007109072E000C880B990B0E9468AD9B01D0
:104BA000AC016FA578A989A99AA90E94C9AE181667
:104BB000ECF480E196E0CF5ADF4F0FB6F894DEBFF9
:104BC0000FBECDBFDF91CF911F910F91FF90EF905E
:104BD000DF90CF90BF90AF909F908F907F906F901D
:104BE0005F904F903F902F900C942B168CEF95E098
:104BF0000E942B16D7DAF701E657FB4F8FE7808329
:104C000080E090E0A0E5B1E425968CAF9DAFAEAF1B
:104C1000BFAF25979601A8EEB3E00E9437B021966A
:104C20006CAF7DAF8EAF9FAF21979B01AC018889A0
:104C30009989AA89BB89280F391F4A1F5B1F2DAB91
:104C40003EAB4FAB58AF81E080935B022889398936
:104C50004A895B892EA33FA348A759A72AA33BA350
:104C60004CA35DA3812C912C54018C8A9D8AAE8A21
:104C7000BF8A75016401188E30E4398F4CE14A8F88
:104C800056E45B8F1C8E1D8E1E8E1F8E1EA689AE57
:104C90009AAEABAEBCAE8FE790E0A0E0B0E08E8302
:104CA0009F83A887B987EFE74E2E512C612C712C7A
:104CB0001AA61BA61CA61DA691E09A871F861E8613
:104CC0001982212C312C00E0812F012E000C990B30
:104CD000DC01A657BB4F2796BFAFAEAF2797880F13
:104CE000991F880F991FFC01ED52FB4FF9A3E8A310
:104CF0002BA9022E000C330B3CAB2BAB80915B023B
:104D0000882309F4C1C20E94A6116A837B838C8325
:104D10009D8380919B04882309F424C1A6D817FFA2
:104D20000AC03091CA0439832090CB043090CC045F
:104D30000091CD0409C0A8A1B9A1BC91B983E8A193
:104D4000F9A12180328003812981322D432D502FFA
:104D50006C8D7D8D8E8D9F8D0E94C6AC87FF05C0AA
:104D6000F981FC8F2D8E3E8E0F8F2981322D432DA0
:104D7000502F688D798D8A8D9B8D0E94C9AE181633
:104D80002CF42981288F298E3A8E0B8F3A85332374
:104D900009F486C06296AEADBFAD6297BC9128960D
:104DA000BFAF28976296EEADFFAD6297F18129966D
:104DB000FFAF29976296AEADBFAD62971296BC91D8
:104DC0002A96BFAF2A976296EEADFFAD6297F38148
:104DD0002B96FFAF2B9728962FAD289729963FAD9E
:104DE00029974B2F5F2F6981722D832D902F0E9461
:104DF000C9AE18160CF0B6C02A813B814C815D818A
:104E00008EA19FA1A8A5B9A5281B390B4A0B5B0B46
:104E100060962CAF3DAF4EAF5FAF6097DA01C9012E
:104E200088589341A109B109B7FD9CC0D301C201C3
:104E30002E813F8148855985821B930BA40BB50BAE
:104E4000B595A7959795879517FF03C08093C504DF
:104E500005C02796EEADFFAD2797808360962CADF9
:104E60003DAD4EAD5FAD60972AA73BA74CA75DA7B0
:104E700028963FAD28973C8F29964FAD29974D8FA7
:104E80002A965FAD2A975E8F2B968FAD2B978F8FCB
:104E90002A813B814C815D812AA33BA34CA35DA366
:104EA0006296AEADBFAD62972D913D914D915C91F3
:104EB0006981722D832D902F0E94C6AC87FF0DC390
:104EC0008A819B81AC81BD812AA13BA14CA15DA1BE
:104ED000821B930BA40BB50BAC01BD014858534189
:104EE0006109710977FDF9C24E855F85452B09F08F
:104EF000E6C18E819F81A885B985840D951DA61D6B
:104F0000B71DB595A7959795879517FFE0C2809334
:104F1000C5042E853F852F5F3F4F3F872E876296C2
:104F2000AEADBFAD6297BC91B88F6296EEADFFADEE
:104F30006297F181F98F6296AEADBFAD629712961E
:104F4000BC91BA8F6296EEADFFAD6297F381FB8F95
:104F50002A813B814C815D812EA33FA348A759A79D
:104F600031E03A8720E030E040EA51E46296AEADAD
:104F7000BFAD62976D917D918D919C910E94EDAB3B
:104F80009B01AC016981722D832D902F0E94C9AEC7
:104F900018162CF488E895E00E942B1675C18A81BA
:104FA0009B81AC81BD81288939894A895B89821BB3
:104FB000930BA40BB50BB7FD9AC0812F17FD80E0B2
:104FC00029DD8AE00E94BB188A819B81AC81BD816A
:104FD0008053984FAF4FBF4F888B998BAA8BBB8B59
:104FE0009EA5911161C029AD3AAD4BAD5CAD698113
:104FF000722D832D902F0E94C9AE1816DCF520E08B
:1050000030E040E050E46981722D832D902F0E94A2
:10501000EDAB69AF7AAF8BAF9CAF2A813B814C81FE
:105020005D8121968CAD9DADAEADBFAD2197280FB2
:10503000391F4A1F5B1F2DAB3EAB4FAB58AF2596B8
:105040002CAD3DAD4EAD5FAD25976FA578A989A973
:105050009AA90E94ECAB9B01AC0191E09EA76981EB
:10506000722D832D902F0E94C9AE18160CF43FC0EC
:105070001EA63DC08A819B81AC81BD812DA93EA920
:105080004FA958AD821B930BA40BB50BB7FD2FC0D6
:105090001F3F19F043E655E002C045E755E064E5DF
:1050A00075E0812FAFD823C020E030E040EA51E422
:1050B0006296AEADBFAD62976D917D918D919C91E1
:1050C0000E94ECAB9B01AC016981722D832D902F66
:1050D0000E94C6AC87FF0BC01F3F19F04DE255E0A0
:1050E00002C040E455E06DE175E0812F8BD88A81E4
:1050F0009B81AC81BD81880F991FAA1FBB1F2AA16C
:105100003BA14CA15DA1821B930BA40BB50B2EA15F
:105110003FA148A559A5821B930BA40BB50B813861
:105120009F44A241B10528F08FEF94E00E942B1616
:10513000ABC04E855F858BA99CA9841795070CF0A1
:10514000DDCD433051050CF4D9CD82EA94E00E94C4
:105150002B1617FD05C02DE9622E24E0722E04C027
:105160009EE9692E94E0792E80E894E00E942B1647
:10517000C3010E942B16B701A60189E994E00E94A1
:1051800076168AE00E94BB1880E894E00E942B16F5
:10519000C3010E942B164C895D896E897F8985E940
:1051A00094E00E9476168AE00E94BB1880E894E0A2
:1051B0000E942B16C3010E942B16B501A40181E9A0
:1051C00094E00E9476168AE00E94BB182C969FAD50
:1051D0002C97992309F4A4C117FF2BC0C092B104E6
:1051E000D092B204E092B304F092B4042CEA35EC0D
:1051F00047E25EE36C897D898E899F890E9404AFB6
:105200006093B5047093B6048093B7049093B80488
:105210002CEA35EC47E25EE3C501B4010E94CDAC57
:105220006093B9047093BA048093BB049093BC0458
:1052300077C1ACE01A029001112489010D551B4F72
:10524000F801C082D182E282F3822CEA35EC47E297
:105250005EE36C897D898E899F890E9404AFD801A5
:1052600014966D937D938D939C9317972CEA35EC50
:1052700047E25EE3C501B4010E94CDACF80160874E
:105280007187828793874CC1CF5ADF4F0FB6F8944E
:10529000DEBF0FBECDBFDF91CF911F910F91FF9069
:1052A000EF90DF90CF90BF90AF909F908F907F90C6
:1052B0006F905F904F903F902F900C94D2202AA532
:1052C0003BA54CA55DA5280F391F4A1F5B1F2A87E8
:1052D0003B874C875D872AA53BA54CA55DA5281B70
:1052E000390B4A0B5B0BCA01B9012E813F814885FE
:1052F00059850E94CEAF2A853B854C855D850E94ED
:1053000013B0D301C201820F931FA41FB51F8431B4
:105310009105A105B105FCF02C013D018C3E9105E4
:10532000A105B1052CF06BEE462E512C612C712C91
:1053300040E84416510461047104DCF08EEF90E003
:10534000A0E0B0E084199509A609B7098E839F8370
:10535000A887B98712C054E1452E512C612C712CBD
:1053600024E130E040E050E02E833F8348875987B6
:1053700004C04E825F8268867986B301A20184EF01
:1053800095E00E9466164E815F81688579858FEE73
:1053900095E00E946616488D598D6A8D7B8D88EE4A
:1053A00095E00E9476164C8D5D8D6E8D7F8D81EE21
:1053B00095E00E9476164E855F85433051050CF4CA
:1053C00098CD6E817F81888599850E9468AD20E0A7
:1053D00030E040E850E40E9404AF6B017C01288D6E
:1053E000398D4A8D5B8D6C8D7D8D8E8D9F8D0E944C
:1053F000ECAB2BED3FE049E450E40E9404AF20E029
:1054000030E040E05FE30E9404AF9B01AC01C701C4
:10541000B6010E94CDAC6B017C016A857B858C85D1
:105420009D850E9468AD2FE632E143E85AE30E9471
:1054300004AF4B015C01B701A6018BED95E00E9422
:105440007616B501A40185ED95E00E9476162AE94D
:1054500039E949E15FE3C701B6010E9404AF6B017E
:105460007C019B01AC010E94EDABA50194010E945F
:10547000CDAC6C8B7D8B8E8B9F8BA5019401C7016E
:10548000B6010E9404AF20E030E040E05EE30E94FD
:1054900004AF4B015C0185EC95E00E942B16B7012F
:1054A000A6018FEB95E00E9476164C895D896E8986
:1054B0007F8989EB95E00E947616B501A40183EB04
:1054C00095E00E9476168AE00E94BB1812CD2796BE
:1054D000EEADFFAD279780831CCD1A8643CD20E02B
:1054E00030E047E053E46FA578A989A99AA90E9402
:1054F000C9AE18160CF45DCB8CEF95E00E942B160C
:105500000E94D2208FE78093C50420E030E040E085
:1055100051E425962CAF3DAF4EAF5FAF25977ACBC8
:10552000CF5ADF4F0FB6F894DEBF0FBECDBFDF916D
:10553000CF911F910F91FF90EF90DF90CF90BF9090
:10554000AF909F908F907F906F905F904F903F9023
:105550002F900895CF92DF92EF92FF9280917F0477
:105560008823A1F10E94A611C0907B04D0907C04F6
:10557000E0907D04F0907E04DC01CB018C199D0944
:10558000AE09BF09B7FD22C00E94A6116B017C01C4
:1055900020917F0430E0A8EEB3E00E9437B0DC0138
:1055A000CB018C0D9D1DAE1DBF1D80937B04909380
:1055B0007C04A0937D04B0937E0480E02BDA8AE023
:1055C000FF90EF90DF90CF900C94BB18FF90EF907E
:1055D000DF90CF9008952F923F924F925F926F92FB
:1055E0007F928F929F92AF92BF92CF92DF92EF9273
:1055F000FF920F931F93CF93DF93CDB7DEB76397DF
:105600000FB6F894DEBF0FBECDBF888B698B81E0EB
:1056100080935B021A821B821C821D821886198667
:105620001A861B8619821C862CE32D873CE13E8757
:1056300046E44F87C12CD12C80E8E82E9FEBF92E51
:10564000812C912C54016091CF047091D004072ECD
:10565000000C880B990B0E9468AD6A8B7B8B182F0E
:10566000092F9B01482F592FB601C7010E94C6ACD4
:105670008823A1F12091D3043091D4044091D50422
:105680005091D6046A897B89812F902F0E94C6ACE5
:10569000881F8827881F89835989552319F18823F2
:1056A00009F180915B0280915B0263960FB6F894DA
:1056B000DEBF0FBECDBFDF91CF911F910F91FF9045
:1056C000EF90DF90CF90BF90AF909F908F907F90A2
:1056D0006F905F904F903F902F900895CA8ADB8A19
:1056E0001E2D0F2D0E94A6116B017C01DC01CB0148
:1056F000288539854A855B85821B930BA40BB50BE6
:10570000B7FD34C0D701C60188519C4FAF4FBF4F82
:1057100088879987AA87BB8788897CD98FE493E09B
:105720000E942B1681149104A104B104C9F0D50183
:10573000C40188519C4FAF4FBF4FBC01CD016C19C4
:105740007D098E099F0928EE33E040E050E00E9479
:10575000F1AFCA01B9014AE050E00E949D1903C0AF
:105760008FE30E94BB188AE00E94BB180E944BABDB
:105770000E94A61160932A0C70932B0C80932C0C22
:1057800090932D0C2090D3043090D4049091D504A4
:105790009E83A091D604AF839101492F5A2F6A8925
:1057A0007B89812F902F0E94ECAB2B013C0120E0E4
:1057B00030E0A9010E94C9AE87FF04C0C301B20155
:1057C000905802C0C301B20120E030E040E251E451
:1057D00081149104A104B10429F40E94C6AC87FF8E
:1057E00007C004C00E94C9AE181614F44601570140
:1057F000B981BB2391F12A813B814C815D812115C7
:1058000031054105510541F0D701C601821B930BBB
:10581000A40BB50BB7FD21C091014E815F816C8552
:105820007D858E859F850E94ECAB20E030E040ECCA
:105830005FE30E94C6AC87FD34CFD701C601805A12
:105840009541AF4FBF4F8A839B83AC83BD832C862A
:105850003D869E819E87AF81AF8780915B028823C2
:1058600009F41FCF81149104A104B10429F4CA885A
:10587000DB88E12EF02EE7CEB8EECB1AB3E0DB0AE0
:10588000E108F108C818D908EA08FB08F7FE09CFB3
:10589000EECF2F923F924F925F926F927F928F92B4
:1058A0009F92AF92BF92CF92DF92EF92FF920F93AF
:1058B0001F93CF93DF93CDB7DEB762970FB6F894FF
:1058C000DEBF0FBECDBF888B81E080935B021A8262
:1058D0001B821C821D82188619861A861B861982D5
:1058E0001C862CE32D873CE13E8746E44F87C12C84
:1058F000D12C80E8E82E9FEBF92E812C912C5401BD
:105900006091C6047091C704072E000C880B990B98
:105910000E9468AD698B7A8B182F092F9B01482F45
:10592000592FB601C7010E94C6AC8823A1F120916E
:10593000CA043091CB044091CC045091CD046989C4
:105940007A89812F902F0E94C6AC881F8827881FD4
:1059500089835889552319F1882309F180915B02C5
:1059600080915B0262960FB6F894DEBF0FBECDBF8A
:10597000DF91CF911F910F91FF90EF90DF90CF902B
:10598000BF90AF909F908F907F906F905F904F905F
:105990003F902F900895C98ADA8A1E2D0F2D0E94FC
:1059A000A6116B017C01DC01CB01288539854A8574
:1059B0005B85821B930BA40BB50BB7FD34C0D701DD
:1059C000C60188519C4FAF4FBF4F88879987AA87E0
:1059D000BB8780E01FD88BE493E00E942B168114D4
:1059E0009104A104B104C9F0D501C40188519C4FB0
:1059F000AF4FBF4FBC01CD016C197D098E099F09C6
:105A000028EE33E040E050E00E94F1AFCA01B90156
:105A10004AE050E00E949D1903C08FE30E94BB182A
:105A20008AE00E94BB180E944BAB0E94A6116093B3
:105A30002A0C70932B0C80932C0C90932D0C90912E
:105A4000CA049E83A091CB04AF832090CC043090F5
:105A5000CD04292F3A2FA10169897A89812F902FAE
:105A60000E94ECAB2B013C0120E030E0A9010E9438
:105A7000C9AE87FF04C0C301B201905802C0C30180
:105A8000B20120E030E040EA50E481149104A10426
:105A9000B10429F40E94C6AC87FF07C004C00E946D
:105AA000C9AE181614F446015701B981BB2391F110
:105AB0002A813B814C815D812115310541055105CC
:105AC00041F0D701C601821B930BA40BB50BB7FDA8
:105AD00021C02E813F81A1016C857D858E859F85AA
:105AE0000E94ECAB20E030E040EC5FE30E94C6ACEB
:105AF00087FD34CFD701C601805A9541AF4FBF4FC4
:105B00008A839B83AC83BD839E819C87AF81AD8755
:105B10002E863F8680915B02882309F41FCF811473
:105B20009104A104B10429F4C988DA88E12EF02E89
:105B3000E7CEB8EECB1AB3E0DB0AE108F108C818EB
:105B4000D908EA08FB08F7FE09CFEECFCF93C82F9C
:105B50006115710519F0CB010E942B1682EB97E0BD
:105B60000E942B16C11103C083EA97E002C088EAA5
:105B700097E00E942B168AE0CF910C94BB1880917D
:105B8000DF048093E00408958091DE04882319F0F7
:105B90001092DE0408958EE098E00C9457AA80914C
:105BA000E004811105C08091DA04811101C00895DB
:105BB00062E070E080E090E00E94E9158091DB04F3
:105BC000882339F061E070E080E090E00E94E91500
:105BD000F5CF08958093E0048093DF04E0CF26980A
:105BE0002E9A25982D9A24982C9A3F98479A0A988D
:105BF000129A0998119A81E0EDCF8093E004CFCFFB
:105C00008093DA04CCCF8091DE04882339F190911F
:105C1000DE048091D904981709F10E9439168FEF9C
:105C200097E00E942B168091DE0480FD1CC08091BD
:105C3000DE0484FD18C08091DE0481FD1EC08091C9
:105C4000DE0485FD1AC08091DE0482FD20C08091B3
:105C5000DE0486FD1CC08AE00E94BB188091DE0431
:105C60008093D904089580E00E94DB58AB01BC0109
:105C70008BEF97E00E947616DECF81E00E94DB5822
:105C8000AB01BC0187EF97E00E947616DCCF82E083
:105C90000E94DB58AB01BC0183EF97E00E947616AF
:105CA000DACFCF9389ED97E00E942B1683B1C1E044
:105CB00086FB882780F963ED77E08C2747DF86B184
:105CC0006DEC77E0881F8827881F40DF83B185FB54
:105CD000882780F967EC77E08C2738DF80B182FB7A
:105CE000882780F961EC77E08C2730DF83B18295DB
:105CF00081706BEB77E08C2729DF80B1869581700E
:105D000065EB77E08C27CF9121CF8091DD041E9940
:105D100004C081608093DD0403C08E7F8093DD0426
:105D20008091DD04379B4DC080618093DD048091BC
:105D3000DD041D9904C082608093DD0403C08D7F63
:105D40008093DD048091DD04029904C08062809319
:105D5000DD0403C08F7D8093DD048091DD041C99F8
:105D600004C084608093DD0403C08B7F8093DD04D6
:105D70008091DD04019904C080648093DD0403C038
:105D80008F7B8093DD049091D8048091DD04981777
:105D900031F092E09093DB048093D80409C08091A5
:105DA000DB04882329F081508093DB04882369F089
:105DB0008091E00481110CC08091DA04811108C047
:105DC00008958F7E8093DD04B2CF9093DC04F0CFF2
:105DD00080914F0580FF1BC0909150058091DC049D
:105DE00090FF0BC080FF13C08091DE048160809320
:105DF000DE0480E00E94D9580AC084FF08C0809168
:105E0000DE0480618093DE0480E00E94D958809196
:105E10004F0581FF1BC0909150058091DC0491FFDC
:105E20000BC081FF13C08091DE0482608093DE048A
:105E300081E00E94D9580AC085FF08C08091DE0425
:105E400080628093DE0481E00E94D95880914F05E2
:105E500082FF20C08091500582FF10C08091DA043B
:105E60008823C1F08091DC0482FF14C08091DE049D
:105E700084608093DE0482E00C94D9588091DC0425
:105E800086FF08C08091DE0480648093DE0482E097
:105E90000C94D958089539CFCF938823A1F0C82FF7
:105EA0000E94391684E50E94BB186AE070E08C2FCE
:105EB00090E00E94AE1980E20E94BB188CE198E04D
:105EC000CF910C942B16CF91089508958091BF0621
:105ED0009091BC06891B8F7019F480E090E00895C2
:105EE0009091B906992351F0833030F48FEF890FE8
:105EF00019F08093B906F1CF1092B906E091BC0673
:105F000086E5E89FF0011124E054F94F808180FD7F
:105F1000E4CF8091BC068F5F8F708093BE06909116
:105F2000BC068091BD06981306C08091BE06809382
:105F3000BD06CF010895CF010895EFE6F0E080811E
:105F40008260808308958091500580FF09C0809110
:105F50000B018270809309018FEF8093E10409C0E7
:105F600080910B01809582708093090181E080937C
:105F7000E1048091500581FF0AC080910B0180955A
:105F80008170809309018FEF8093E20408C08091B3
:105F90000B0181708093090181E08093E20480917C
:105FA000500582FF09C080910B0184708093090124
:105FB0008FEF8093E30409C080910B01809584707A
:105FC0008093090181E08093E30400000000000059
:105FD00008950F930FB70F9300916E000F930B7FEF
:105FE00000936E0000916F000D7F00936F000F9380
:105FF0000BB70F930CB70F921F922F933F934F93B2
:106000005F936F937F938F939F93AF93BF93EF9320
:10601000FF9311240E94C938FF91EF91BF91AF9176
:106020009F918F917F916F915F914F913F912F91B0
:106030001F900F900CBF0F910BBF0F910260F8944F
:1060400000936F000F9100936E000F910FBF0F919F
:106050001895CF92DF92EF92FF920F931F9380914A
:106060004E058823D1F010924E05809151059091F4
:106070005205892B91F010924F0510925205109203
:1060800051059091BF068091BC06981731F0809120
:10609000BC068F5F8F708093BC06809151059091F4
:1060A0005205892B09F4AAC140911D0550911E0586
:1060B00060911F0570912005909145050091110593
:1060C000109112052091130530911405041B150B36
:1060D000260B370B892F90E0A0E0B0E008171907D6
:1060E0002A073B0710F4D901C801E82F840F951F38
:1060F000A61FB71F80931D0590931E05A0931F0533
:10610000B09320052091840030918500225E3F4F9E
:1061100040913505509136056091370570913805ED
:106120008091250590912605A0912705B09128051D
:10613000840F951FA61FB71F8093350590933605D2
:10614000A0933705B0933805B7FD1CC0409A409125
:10615000E5045091E6046091E7047091E8048091B1
:10616000E104082E000C990BAA0BBB0B840F951FA2
:10617000A61FB71F8093E5049093E604A093E7045D
:10618000B093E8044091390550913A0560913B0580
:1061900070913C058091290590912A05A0912B05CD
:1061A000B0912C05840F951FA61FB71F809339054A
:1061B00090933A05A0933B05B0933C05B7FD1CC0F6
:1061C000419A4091E9045091EA046091EB04709186
:1061D000EC048091E204082E000C990BAA0BBB0B77
:1061E000840F951FA61FB71F8093E9049093EA04BC
:1061F000A093EB04B093EC0440913D0550913E0513
:1062000060913F057091400580912D0590912E057C
:10621000A0912F05B0913005840F951FA61FB71FC1
:1062200080933D0590933E05A0933F05B0934005B4
:10623000B7FD1CC0429A4091ED045091EE0460916C
:10624000EF047091F0048091E304082E000C990B88
:10625000AA0BBB0B840F951FA61FB71F8093ED04DD
:106260009093EE04A093EF04B093F00440914105A5
:10627000509142056091430570914405809131052C
:1062800090913205A0913305B0913405840F951F8C
:10629000A61FB71F8093410590934205A093430525
:1062A000B0934405B7FD3CC0C090F104D090F20417
:1062B000E090F304F090F4044091E404042E000C08
:1062C000550B660B770B4C0D5D1D6E1D7F1D4093AE
:1062D000F1045093F2046093F3047093F40440913A
:1062E0002105509122056091230570912405841B9E
:1062F000950BA60BB70B8093410590934205A09395
:106300004305B0934405909150058091060593FF95
:1063100004C081508093060503C08F5F80930605FB
:10632000809184009091850082179307C8F3809133
:10633000350590913605A0913705B0913805B7FD28
:1063400015C040912105509122056091230570915F
:106350002405841B950BA60BB70B809335059093F2
:106360003605A0933705B0933805409880913905DC
:1063700090913A05A0913B05B0913C05B7FD15C041
:1063800040912105509122056091230570912405CB
:10639000841B950BA60BB70B8093390590933A0598
:1063A000A0933B05B0933C05419880913D059091A9
:1063B0003E05A0913F05B0914005B7FD15C0409145
:1063C0002105509122056091230570912405841BBD
:1063D000950BA60BB70B80933D0590933E05A093BC
:1063E0003F05B09340054298E15041F08091840010
:1063F0009091850082179307C8F388CE1F910F9163
:10640000FF90EF90DF90CF900895CF92DF92EF92C0
:10641000FF9280910505882309F465C0C0901D0591
:10642000D0901E05E0901F05F090200540911505C5
:106430005091160560911705709118058091060519
:106440004C155D056E057F05E8F420910B05309134
:106450000C05E0910905F0910A05E217F30790F4A5
:106460008150809306052150310930930C0520930B
:106470000B054091210250912202609123027091FC
:10648000240234C0C416D506E606F706E8F42091C7
:106490000B0530910C054091070550910805241714
:1064A000350790F48F5F809306052F5F3F4F309341
:1064B0000C0520930B05409121025091220260911E
:1064C00023027091240212C08FEF9FEFDC018093B2
:1064D000210290932202A0932302B09324024FEF53
:1064E0005FEFBA0103C04FEF5FEFBA01809106057D
:1064F00087FD06C080910B0180748093090106C05E
:1065000080910B0180958074809309012091840013
:1065100030918500225E3F4F80910605882311F15E
:10652000439A809184009091850082179307C8F365
:106530008091060587FF04C08F5F8093060503C026
:10654000815080930605439880910605882321F3A6
:10655000809184009091850082179307C8F3225E92
:106560003F4FDACFCB01BA01FF90EF90DF90CF9091
:106570000895BC012091510530915205409151057B
:10658000509152052417350711F09A01F7CF81E099
:106590006217730709F080E00895CF93DF93EC0151
:1065A00088819981AA81BB81E5EEF4E080839183A3
:1065B000A283B383EB0188819981AA81BB81848303
:1065C0009583A683B783EA0188819981AA81BB81DB
:1065D00080879187A287B387E90188819981AA8101
:1065E000BB8184879587A687B787DF91CF91089570
:1065F0003F924F925F926F927F928F929F92AF9253
:10660000BF92CF92DF92EF92FF920F931F93CF939F
:10661000DF93CDB7DEB728970FB6F894DEBF0FBE75
:10662000CDBFA0915105B0915205109739F18090DE
:106630001D0590901E05A0901F05B090200540916B
:10664000110550911205609113057091140584167F
:106650009506A606B706C8F010924F05109252058F
:10666000109251059091BF068091BC06981731F0A9
:106670008091BC068F5F8F708093BC0670EDC72E33
:1066800077E0D72EE12CF12C97C14091190550915C
:106690001A0560911B0570911C05481559056A057E
:1066A0007B0508F46EC000914A0510914B052091BE
:1066B0004C0530914D05D1964D915D916D917C9138
:1066C000D497EE27059FF12D169FC001269F900DB0
:1066D000259F800D911D069FF00D811D9E1F159F0A
:1066E000F00D811D9E1F249FF00D811D9E1F149F84
:1066F000F10D8E1F9E1FF6958E1F9E1F709F800DA1
:10670000911D719F900D1124FD01EB5BFF4F4081A6
:10671000518162817381480F591F611D711D409322
:1067200001055093020560930305709304053497A7
:10673000C080D180E280F380C416D506E606F70655
:1067400040F4C0920105D0920205E0920305F09258
:106750000405409101055091020560910305709177
:1067600004058AE798E0BB24B394FC01C590D5905A
:10677000E590F490C416D506E606F70608F475C24F
:106780007FC24090150550901605609017057090D7
:106790001805481459046A047B0408F080C020914D
:1067A00046053091470540914805509149052D8394
:1067B0003E834F835887D1960D911D912D913C9129
:1067C000D4974D815E816F817885EE27419FF12DB1
:1067D000529FC001629F900D619F800D911D429F4D
:1067E000F00D811D9E1F519FF00D811D9E1F609F0A
:1067F000F00D811D9E1F509FF10D8E1F9E1FF6955F
:106800008E1F9E1F349F800D911D359F900D11246A
:106810008C0120E030E0C0900105D0900205E090AE
:106820000305F0900405CD01875B9F4FFC010C151B
:106830001D052E053F05C0F44081518162817381A1
:1068400049835A836B837C83C01AD10AE20AF30A14
:10685000C416D506E606F70610F46A017B018AE73E
:1068600098E03324339410C0C080D180E280F3805C
:10687000F6CFF694E794D794C794330C049628E0A7
:106880008639920709F480C2FC0105911591259182
:1068900034910C151D052E053F0558F375C28091E6
:1068A00006058823D9F0D7964D915C91D89760E082
:1068B00070E0009121021091220220912302309178
:1068C0002402041715072607370741F01092250206
:1068D00010922602109227021092280240911D0267
:1068E00050911E0260911F027091200277FF5CC0E0
:1068F000AF5BBF4F8D919D910D90BC91A02D2AE76C
:1069000038E041E0F901C590D590E590F490C816C3
:10691000D906EA06FB0658F4B695A795979587958C
:10692000440F2C5F3F4F58E02639350759F7409305
:10693000450580329105A105B10520F480E290E083
:10694000A0E0B0E08097A109B109811578E0970730
:10695000A105B10508F4CEC224E0929FF0011124F4
:106960009F012656334FF901329665917491EE27B7
:10697000879FA001869F410D5E1F06944E1F5E1FDC
:10698000112460E070E0F90185919491A0E0B0E0FD
:10699000841B950BA60BB70B80931D0290931E02D0
:1069A000A0931F02B0932002C0901D02D0901E023F
:1069B000E0901F02F09020028091510590915205C5
:1069C000892B09F01DC382DA9093520580935105FB
:1069D000892B09F415C3E0915105F091520580818E
:1069E00083FF19C09F012F5D3F4FAF01435E5F4F93
:1069F000BF01675E7F4FCF014596CFDD9091BF0607
:106A00008091BC069817F9F28091BC068F5F8F7059
:106A10008093BC06D8CFC588D688E788F08C81E003
:106A2000C114D104E104F10409F480E0018D128D58
:106A3000238D348D011511052105310509F0826082
:106A4000458D568D678D70A1411551056105710504
:106A500009F0846080934F05109246051092470517
:106A6000109248051092490510924A0510924B0564
:106A700010924C0510924D0585A196A1A7A1B0A535
:106A80008093110590931205A0931305B0931405FC
:106A9000882499245401881A990AAA0ABB0A809268
:106AA000410590924205A0924305B0924405809220
:106AB0003D0590923E05A0923F05B0924005809220
:106AC000390590923A05A0923B05B0923C05809220
:106AD000350590923605A0923705B0923805CC0C5A
:106AE000DD1CEE1CFF1CC0922505D0922605E0920D
:106AF0002705F0922805000F111F221F331F009356
:106B0000290510932A0520932B0530932C05440F5B
:106B1000551F661F771F40932D0550932E056093D8
:106B20002F057093300541A152A163A174A1440FB8
:106B3000551F661F771F40933105509332056093B0
:106B4000330570933405880F991FAA1FBB1F8093CC
:106B5000210590932205A0932305B093240510925C
:106B60001D0510921E0510921F051092200581A58B
:106B700092A5A3A5B4A58093190590931A05A09397
:106B80001B05B0931C0585A596A5A7A5B0A9809364
:106B9000150590931605A0931705B093180586A9BF
:106BA00080930505882309F183AD94AD90930A0580
:106BB0008093090581AD92AD9093080580930705F8
:106BC000109225021092260210922702109228029B
:106BD00087A990ADA0E0B0E08093210290932202BB
:106BE000A0932302B09324020BC08FEF9FEFDC0130
:106BF0008093210290932202A0932302B093240257
:106C000085A990915005891719F0809350059BD95B
:106C10007CD88FEF9FEFDC0180931D0290931E02C2
:106C2000A0931F02B0932002E0915105F09152050C
:106C3000EB5BFF4F80819181A281B381809301053D
:106C400090930205A0930305B09304052AE738E06A
:106C500041E0F901C590D590E590F490C816D906A9
:106C6000EA06FB0608F46BC176C1769567955795E1
:106C70004795BB0C0496E8E086399E0709F075CD70
:106C8000B0924505403251056105710520F440E29E
:106C900050E060E070E0405251096109710941150E
:106CA00088E058076105710500F194E0599FF001F3
:106CB0001124CF018656934FFC013296E590F49053
:106CC000F701DD244F9F50014E9FA10CBD1C06947F
:106CD000AD1CBD1C1124FC01C590D490E12CF12CFD
:106CE000CA18DB08E108F10824C06A017B01F694A8
:106CF000E794D794C794F601EC7FCF018656974F5F
:106D00007C01FC0185919491F7013296E590F49015
:106D100047704E9DB0014F9D700D1124AB0163E093
:106D2000569547956A95E1F76C01C41AD50AE12C8E
:106D3000F12C0C0D1D1D2E1D3F1D00934A051093B7
:106D40004B0520934C0530934D059091050580919E
:106D50000605992309F465C0882309F42DCED7963A
:106D60008D919C91D897A0E0B0E040912102509184
:106D700022026091230270912402481759076A0782
:106D80007B0709F051C018CE30924505F0E2CF16CE
:106D9000D104E104F10428F430E2C32ED12CE12C1B
:106DA000F12CF0E2CF1AD108E108F108C11428E073
:106DB000D206E104F10408F440C034E0D39EC001DF
:106DC00011248656934FFC013296059114916C2D37
:106DD0003327619FA001609F410D531F0694431FFD
:106DE000531F1124FC01C590D490E12CF12CC41A3E
:106DF000D50AE108F1084D815E816F8178854C0DDF
:106E00005D1D6E1D7F1D40934605509347056093A1
:106E100048057093490580910505811132C0809124
:106E20000605882309F4C8CD109225021092260287
:106E30001092270210922802BFCD97018601369545
:106E4000279517950795F801EC7FCF018656974F48
:106E5000FC0105911491FC013296459154913C2D11
:106E60003770349FC001359F900D112423E0969513
:106E700087952A95E1F76801C81AD90AE12CF12C07
:106E8000BACF430C511C611C711C481459046A048C
:106E90007B04C8F480910605882309F48DCDD7962C
:106EA0004D915C91D89760E070E0009121021091C3
:106EB000220220912302309124020417150726078D
:106EC000370709F479CD109225021092260210920C
:106ED000270210922802D7968D919C91D897A0E016
:106EE000B0E08093210290932202A0932302B093FA
:106EF000240262CDAC01BD01769567955795479503
:106F0000FA01EC7FAF014656574FFA0125913491B3
:106F1000FA013296659174918770869FA001879FD0
:106F2000500D1124CA01F3E096958795FA95E1F783
:106F3000A901481B590BCA01A0E0B0E02DCDB695C0
:106F4000A79597958795440F2C5F3F4F68E02639AA
:106F5000360709F07ECE4093450580329105A105A4
:106F6000B10520F480E290E0A0E0B0E08097A109B4
:106F7000B109811558E09507A105B105F8F064E065
:106F8000969FF00111249F012656334FF901329646
:106F900065917491EE27879FA001869F410D5E1F2A
:106FA00006944E1F5E1F1124F901C590D490E12C68
:106FB000F12CC41AD50AE108F10822C0AC01BD01C8
:106FC0007695679557954795FA01EC7FAF01465640
:106FD000574FFA01C590D490FA01329645915491D9
:106FE0008770849F9001859F300D1124C901A3E013
:106FF00096958795AA95E1F7C81AD90AE12CF12C44
:10700000C701B60128960FB6F894DEBF0FBECDBFFC
:10701000DF91CF911F910F91FF90EF90DF90CF9074
:10702000BF90AF909F908F907F906F905F904F90A8
:107030003F900895CF92DF92EF92FF921F93CF93EC
:10704000DF938FEF9FEF90938900809388001AE081
:10705000C0E0D0E0789480910D0590910E05A0914C
:107060000F05B0911005892B8A2B8B2B11F40E94F0
:1070700029308091250290912602A0912702B0919B
:107080002802892B8A2B8B2B49F4BFD960932502C8
:1070900070932602809327029093280280910D0519
:1070A00090910E05A0910F05B0911005892B8A2BA8
:1070B0008B2B49F49DDA60930D0570930E05809338
:1070C0000F0590931005C0900D05D0900E05E0902F
:1070D0000F05F09010054091250250912602609115
:1070E000270270912802FC2DED2D3E2D2F2D4C15E1
:1070F0005D056E057F0520F4F42FE52F362F272F31
:107100008F2F9E2FA32FB22F009721E0A207B1054A
:1071100020F08FEF9FEFA0E0B0E0C81AD90AEA0A8A
:10712000FB0AC0920D05D0920E05E0920F05F09279
:1071300010054F3F2FEF52076207720761F0481B9F
:10714000590B6A0B7B0B40932502509326026093E8
:10715000270270932802F8942091840030918500D2
:10716000205F3F4F115039F0C80FD91FC217D30706
:1071700008F470CF01C0E901D0938900C093880062
:107180007894DF91CF911F91FF90EF90DF90CF9097
:10719000089550CF90916F0091FB222720F991FF25
:1071A00005C090916F009D7F90936F0094E0899F40
:1071B000F0011124EB51FB4F608171818281938139
:1071C000222329F020916F00226020936F00089500
:1071D00090916F0091FB222720F991FF05C09091BB
:1071E0006F009D7F90936F0034E0839FC001112456
:1071F000FC01EB51FB4F4081518162817381FC01A5
:10720000EB50FB4F408351836283738381E0809313
:107210004E05222329F080916F00826080936F00D9
:10722000089590916F0091FB222720F991FF05C0EE
:1072300090916F009D7F90936F0094E0899FF00183
:107240001124EB50FB4F6081718182819381222355
:1072500029F020916F00226020936F0008954F92D3
:107260005F926F927F928F929F92AF92BF92CF92D6
:10727000DF92EF92FF9280916F0081FB992790F946
:1072800081FF05C080916F008D7F80936F004090DB
:10729000E5045090E6046090E7047090E804809064
:1072A000E9049090EA04A090EB04B090EC04C09044
:1072B000ED04D090EE04E090EF04F090F0049923F8
:1072C00029F080916F00826080936F0080E798E0E2
:1072D0000E942B164AE050E0C301B2010E949D19A2
:1072E0008CE698E00E942B164AE050E0C501B401FC
:1072F0000E949D1988E698E00E942B164AE050E013
:10730000C701B6010E949D198AE0FF90EF90DF90BF
:10731000CF90BF90AF909F908F907F906F905F9035
:107320004F900C94BB18DB01833070F494E0899F7C
:10733000F0011124ED5AFA4FAB01770F660B770B72
:107340004083518362837383813091F018F08230DF
:10735000E9F008952FEF30E00E9446B020ED37E0CD
:1073600040E050E00E9413B0B9018EE20C9472121A
:107370002FEF30E00E9446B020ED37E040E050E0D3
:107380000E9413B0B9018DE20C9472122FEF30E01D
:107390000E9446B020ED37E040E050E00E9413B07C
:1073A000B9018CE20C947212CF93DF93C3E5D5E060
:1073B0006881798180E0B7DF6C817D8181E0B3DF16
:1073C0006885798582E0DF91CF91ADCFEAE0F1E089
:1073D00080818860808380818061808380818062F9
:1073E0008083E2DFE1E2F1E08081887F8160808359
:1073F000089567FD2CC0813061F028F0823099F04B
:107400008330D9F024C0662311F0A19A2AC0A19834
:1074100028C08091080161118095807880930601D1
:1074200047FF27C0089580910801611180958074FD
:107430008093060147FF23C00895809108016111E0
:10744000809588708093060147FF21C0089547FD0D
:1074500026C0813071F038F0823089F08330B9F085
:10746000089547FD1CC0442311F0A09A0895A098E8
:107470000895442311F0A29A0895A2980895809146
:1074800008014111809580728093060108958091D2
:107490000801411180958071809306010895089537
:1074A000643091F040F4613059F06230A9F420E08A
:1074B00040E061E09ECF683059F0603149F00CC087
:1074C00020E040E060E095CF20E041E060E091CF37
:1074D00020E041E061E08DCF0E943C1680E598E01D
:1074E0000C942B160F931F93CF93999A989A80918F
:1074F00007018068809307019A9A80910701806450
:107500008093070180910701806280930701809139
:107510000701886080930701809107018061809353
:1075200007010DE013E0C0E0F80161918F018C2F9D
:10753000B7DFCF5FC630C1F7CF911F910F9108958C
:1075400045DFD0DFEAE0F1E08081826080838081E6
:107550008160808380818460808380818064808377
:107560000F9A179A0E9A169A0D9A159A0C9A149ABF
:10757000389A4098179A8091BC058E7F8093BC05FD
:10758000399A4198169A8091BC058D7F8093BC05ED
:107590003A9A4298159A8091BC058B7F8093BC05DE
:1075A0003B9A4398149AA0E8B0E08C918C7F8C931E
:1075B000E1E8F0E08081877E886080838C918F7322
:1075C0008C938081887F8260808380E090E49093B8
:1075D0008900809388001092850010928400EFE665
:1075E000F0E0808182608083789482E0809350050F
:1075F0000C94A32F8BE398E00E942B16919902C064
:1076000080E301C081E30E94BB18909902C080E32F
:1076100001C081E30E94BB1887E398E00E942B160B
:1076200080910601881F8827881F805D0E94BB18F3
:10763000929902C080E301C081E30E94BB1883E3FA
:1076400098E00E942B168091060186FD02C080E31F
:1076500001C081E30E94BB188091060185FD02C034
:1076600080E301C081E30E94BB188EE298E00E9493
:107670002B168091060183FD02C080E301C081E3E7
:107680000E94BB188091060184FD02C080E301C006
:1076900081E30C94BB181F93CF93DF93CDB7DEB774
:1076A00060970FB6F894DEBF0FBECDBF8091AB05DB
:1076B0009091AC05A091AD05B091AE0589839A83F8
:1076C000AB83BC838091AF059091B005A091B105CB
:1076D000B091B2058D839E83AF83B8878091B30547
:1076E0009091B405A091B505B091B60589879A87A8
:1076F000AB87BC878091B7059091B805A091B9057B
:10770000B091BA058D879E87AF87B88B0E948B6931
:107710006091500270915102072E000C880B990B5A
:107720000E9468AD2AE037ED43E25CE30E9404AFBB
:1077300060934C0270934D0280934E0290934F02DF
:1077400010E0812F0E946F51812F0E94614F1F5FB7
:107750001330B9F729DE0E94D26940E150E06BEAAC
:1077600075E0CE0101960E947EB4892B59F0609697
:107770000FB6F894DEBF0FBECDBFDF91CF911F9142
:107780000C94674C60960FB6F894DEBF0FBECDBF69
:10779000DF91CF911F9108958734924041F00E946C
:1077A0003C168DEF93E10E942B1681E0089580E056
:1077B0000895EF92FF920F931F93CF93DF93CDB76E
:1077C000DEB7C458D1090FB6F894DEBF0FBECDBFE7
:1077D000ED961CAE1DAE1EAE1FAEED9785E492E594
:1077E000A2E5B0E0E9968CAF9DAFAEAFBFAFE99731
:1077F000CF57DF4F19821882C158D04084E690E0FD
:10780000C158DF4F99838883CF57D0400E94D81644
:10781000109260059E012F573F4F44E050E0BE019B
:107820006B587F4FCE0181589F4F0E94DC16C15884
:10783000DF4F88819981CF57D0400296C158DF4FE2
:1078400099838883CF57D040CF57DF4F1982188252
:10785000C158D04081E0CC57DF4F8883C458D04016
:107860009E012F573F4F41E050E0BE016C577F4FC4
:10787000CE0181589F4F0E94DC169E012F573F4F2B
:1078800048E450E061E776E0CE0181589F4F0E94C6
:10789000DC169E012F573F4F40E150E061E476E057
:1078A000CE0181589F4F0E94DC168AE097EDA3EA33
:1078B000BCE3ED968CAF9DAFAEAFBFAFED979E0131
:1078C0002F573F4F44E050E0BE0167587F4FCE0135
:1078D00081589F4F0E94DC169E012F573F4F4CE06E
:1078E00050E067E775E0CE0181589F4F0E94DC169B
:1078F00080E090E0A0E2B1E489839A83AB83BC830B
:107900009E012F573F4F44E050E08E010F5F1F4F05
:10791000B801CE0181589F4F0E94DC16ED961CAE37
:107920001DAE1EAE1FAEED9783E0AE968FAFAE9745
:1079300089839E012F573F4F44E050E0BE016758B6
:107940007F4FCE0181589F4F0E94DC169E012F571A
:107950003F4F41E050E0BE0163597F4FCE01815857
:107960009F4F0E94DC169E012F573F4F41E050E091
:10797000B801CE0181589F4F0E94DC162AE0F22EFA
:10798000FA949E012F573F4F44E050E0FF2049F00A
:10799000BE0167587F4FCE0181589F4F0E94DC1671
:1079A000EFCF61E675E0CE0181589F4F0E94DC1653
:1079B0009E012F573F4F44E250E06CE176E0CE014C
:1079C00081589F4F0E94DC1683E0CD57DF4F88839C
:1079D000C358D040EE968FAFEE97E1961CAE1DAE29
:1079E0001EAE1FAEE19719821A821B821C82ED9691
:1079F0001CAE1DAE1EAE1FAEED979E012F573F4F22
:107A000041E050E0BE016D577F4FCE0181589F4F3E
:107A10000E94DC169E012F573F4F41E050E0BE010F
:107A200063587F4FCE0181589F4F0E94DC169E0104
:107A30002F573F4F44E050E0B801CE0181589F4F8F
:107A40000E94DC169E012F573F4F44E050E0BE01DC
:107A500063597F4FCE0181589F4F0E94DC169AE0F8
:107A6000E92EF12C81E0E81AF10871F09E012F5700
:107A70003F4F44E050E0BE0167587F4FCE01815830
:107A80009F4F0E94DC16EECFAE961FAEAE978FEFE3
:107A900089839E012F573F4F41E050E0BE0163595B
:107AA0007F4FCE0181589F4F0E94DC169E012F57B9
:107AB0003F4F41E050E0B801CE0181589F4F0E94F6
:107AC000DC1680E1F82EF8018F2D11928A95E9F7E6
:107AD0009E012F573F4F40E150E0B801CE01815841
:107AE0009F4F0E94DC1688EC90E0AF969FAF8EAF60
:107AF000AF9780EF90E0E1969FAF8EAFE19786E47D
:107B000090E09A8389838EE690E09C838B83EE9647
:107B10001FAEEE97EF961FAEEF979E012F573F4F88
:107B200044E050E0BE0163597F4FCE0181589F4F22
:107B30000E94DC169E012F573F4F44E050E0B801F1
:107B4000CE0181589F4F0E94DC169E012F573F4F58
:107B500042E050E0BE0163587F4FCE0181589F4FF5
:107B60000E94DC16F8011192FA94E9F780E090E0A7
:107B7000A0E8BFE38D879E87AF87B88B8091A30471
:107B80009091A404A091A504B091A60489839A833E
:107B9000AB83BC838091A7049091A804A091A90411
:107BA000B091AA048D839E83AF83B8878091AB0484
:107BB0009091AC04A091AD04B091AE0489879A87EE
:107BC000AB87BC879E012F573F4F40E150E0B80183
:107BD000CE0181589F4F0E94DC1684E190E09A8389
:107BE00089839E012F573F4F42E050E0B801CE01FC
:107BF00081589F4F0E94DC169E012F573F4F4CE04B
:107C000050E061EB74E0CE0181589F4F0E94DC167A
:107C100080E290E09A8389839E012F573F4F42E094
:107C200050E0B801CE0181589F4F0E94DC1681E0E0
:107C300089839E012F573F4F41E050E0B801CE01AC
:107C400081589F4F0E94DC1680E2EDE5F2E0D801FA
:107C500001900D928A95E1F79E012F573F4F40E228
:107C600050E0B801CE0181589F4F0E94DC16AE96BD
:107C70001FAEAE979E012F573F4F41E050E0BE012F
:107C800063597F4FCE0181589F4F0E94DC161982A5
:107C900080E090E0A0E4B0E4ED968CAF9DAFAEAF95
:107CA000BFAFED979E012F573F4F41E050E0B80125
:107CB000CE0181589F4F0E94DC169E012F573F4FE7
:107CC00044E050E0BE0167587F4FCE0181589F4F7E
:107CD0000E94DC168AE1F80111928A95E9F79E016B
:107CE0002F573F4F4AE150E0B801CE0181589F4FD6
:107CF0000E94DC1684E3EDE7F2E0D80101900D92DA
:107D00008A95E1F79E012F573F4F44E350E0B801B9
:107D1000CE0181589F4F0E94DC161A8219821C8264
:107D20001B821E821D829E012F573F4F46E050E06E
:107D3000B801CE0181589F4F0E94DC168DE0F801FA
:107D400011928A95E9F79E012F573F4F4DE050E081
:107D5000B801CE0181589F4F0E94DC169E012F571B
:107D60003F4F44E050E063EE75E0CE0181589F4FF5
:107D70000E94DC169E012F573F4F4CE050E063E518
:107D800075E0CE0181589F4F0E94DC168CE6F80109
:107D900011928A95E9F79E012F573F4F4CE650E02C
:107DA000B801CE0181589F4F0E94DC169E012F57CB
:107DB0003F4F4CE050E060E176E0CE0181589F4FAC
:107DC0000E94DC16E1961CAE1DAE1EAE1FAEE19702
:107DD000E5961CAE1DAE1EAE1FAEE5979E012F5759
:107DE0003F4F48E050E0BE0163597F4FCE018158BC
:107DF0009F4F0E94DC168091600581114FC0C158D1
:107E0000DF4F08811981CF57D04004561109CF5751
:107E1000DF4F88819981C158D040AF969FAF8EAF18
:107E2000AF9784E690E0C158DF4F99838883CF579E
:107E3000D0409E012F573F4F44E050E063E173E094
:107E4000CE0181589F4F0E94DC169E012F573F4F55
:107E500042E050E0BE0163597F4FCE0181589F4FF1
:107E60000E94DC160E943916B8018BEE93E10E9445
:107E70009616AF964EAD5FADAF9760E070E08EEDB9
:107E800093E10E94A0168BED93E10E942B16C8018E
:107E900083DC90916005892B809360050E94DA163F
:107EA0009091600581E08927CC57DF4F0FB6F89499
:107EB000DEBF0FBECDBFDF91CF911F910F91FF901D
:107EC000EF9008951F93CF93DF93CDB7DEB72C9734
:107ED0000FB6F894DEBF0FBECDBFA1E7B6E020E03D
:107EE00030E0C9012430310510F083E090E0880FC4
:107EF000991F880F991FFC01E75DFC4E4591559134
:107F00006591749154964D935D936D937C935797BF
:107F1000FC01E75EFC4E45915591659174919496F4
:107F20004D935D936D937C939797FC01E75FFC4EB7
:107F300045915591659174914D935D936D937D93AA
:107F40002F5F3F4F2430310509F0CBCF80E29EE414
:107F5000A0E0B0E08093810690938206A093830610
:107F6000B093840680E090E0AAEFB4E48093A50685
:107F70009093A606A093A706B093A80640E050E809
:107F80006BE375E44093A9065093AA066093AB0691
:107F90007093AC068093AD069093AE06A093AF06A7
:107FA000B093B0061092B1061092B2061092B306CA
:107FB0001092B4061092B5061092B6061092B7064B
:107FC0001092B80680E090E0A0E4B1E4809341060E
:107FD00090934206A0934306B093440680934506CF
:107FE00090934606A0934706B09348068DEC9CEC10
:107FF000ACECBEE38093490690934A06A0934B06EF
:10800000B0934C0680E090E0A0E2B1E480934D068E
:1080100090934E06A0934F06B09350061CE0E7E7FE
:10802000F5E0DF01812F1D928A95E9F70E94CE1AB3
:1080300080E090E0A0EBBFEB809361059093620538
:10804000A0936305B093640583E393E3A6E1B2E4F0
:108050008093A3049093A404A093A504B093A604D2
:108060008EEA92E1A2E6BFE38093A7049093A8046E
:10807000A093A904B093AA0480E896E7A7ECB3E420
:108080008093AB049093AC04A093AD04B093AE0482
:1080900080E090E0A3E9B3E48093B1049093B2044C
:1080A000A093B304B093B40483EC94E6AAE2B1E4E1
:1080B0008093B5049093B604A093B704B093B8042A
:1080C00080EB98EBA1E1B5E48093B9049093BA04F6
:1080D000A093BB04B093BC0481E00E94EA2D0E94EF
:1080E000652F1092E3051092E4051092E5051092B9
:1080F000E605E1EBF2E0DE01119601900D921A9592
:10810000E1F713E01150C0F0A4E01A9F9001112490
:10811000E1E0F0E0EC0FFD1FE20FF31F60817181E1
:1081200082819381F901ED5AFA4F608371838283D2
:108130009383812FF8D8E6CFAEDA0E94391686EE07
:1081400092E12C960FB6F894DEBF0FBECDBFDF9143
:10815000CF911F910C942B16CF93C82F811102C081
:108160000E9439168FEC92E10E942B168DE990E166
:108170000E942B168AE00E94BB188AE00E94BB185E
:10818000C11106C00E9439168EEB92E10E942B1697
:108190006FEF81E08C270E94FC93C11108C00E9400
:1081A000391680EA92E10E942B160E9439164091FE
:1081B000950650919606609197067091980687E90A
:1081C00092E10E9476164091990650919A0660912C
:1081D0009B0670919C0684E992E10E94761640917C
:1081E0009D0650919E0660919F067091A00681E9C0
:1081F00092E10E9476164091A1065091A2066091EC
:10820000A3067091A4068EE892E10E9476168AE099
:108210000E94BB18C11108C00E9439168CE692E179
:108220000E942B160E943916609171067091720699
:1082300080917306909174060E9466ADAB01BC01FB
:1082400083E692E10E94761660917506709176063B
:1082500080917706909178060E9466ADAB01BC01D3
:1082600080E692E10E9476166091790670917A0616
:1082700080917B0690917C060E9466ADAB01BC01AB
:108280008DE592E10E94761660917D0670917E06E2
:1082900080917F06909180060E9466ADAB01BC0183
:1082A0008AE592E10E9476168AE00E94BB18C1110D
:1082B00008C00E94391680E192E10E942B160E94AC
:1082C00039164091A5065091A6066091A7067091B7
:1082D000A80687E092E10E9476164091A906509187
:1082E000AA066091AB067091AC0684E092E10E9410
:1082F00076164091AD065091AE066091AF06709132
:10830000B00681E092E10E9476168AE00E94BB18D6
:10831000C11113C00E94391689EB91E10E942B16FE
:108320008EE891E10E942B168FE791E10E942B16B7
:108330008AE00E94BB180E943916609181067091F4
:10834000820680918306909184060E9466ADAB01FF
:10835000BC0186E791E10E9476164091B1065091EA
:10836000B2066091B3067091B40683E791E10E9472
:1083700076164091B5065091B6066091B706709199
:10838000B80680E791E10E9476164091410650912F
:10839000420660914306709144068DE691E10E9489
:1083A00076164091450650914606609147067091B9
:1083B00048068AE691E10E9476164091490650915E
:1083C0004A0660914B0670914C0687E691E10E9447
:1083D000761640914D0650914E0660914F06709171
:1083E000500684E691E10E9476168AE00E94BB184E
:1083F000C11108C00E94391686E591E10E942B1632
:108400000E94391640917705509178056091790561
:1084100070917A058DE491E10E94761640917B057A
:1084200050917C0560917D0570917E058AE491E113
:108430000E94761640917F055091800560918105DC
:108440007091820587E491E10E9476168AE00E948D
:10845000BB18C11108C00E94391683E391E10E9444
:108460002B160E9439166091400670E08AE291E175
:108470000E945C168AE00E94BB18C11108C00E94CD
:1084800039168BE191E10E942B160E94391640911A
:10849000A3045091A4046091A5047091A60482E104
:1084A00091E10E9476162CEA35EC47E25EE360919A
:1084B000A7047091A8048091A9049091AA040E9435
:1084C000CDACAB01BC018FE091E10E9486162CEA95
:1084D00035EC47E25EE36091AB047091AC048091AF
:1084E000AD049091AE040E9404AFAB01BC018CE0DE
:1084F00091E10E9486168AE00E94BB18C11102C059
:108500000E9439164091B1045091B2046091B304B5
:108510007091B40483E091E10E9476162CEA35EC68
:1085200047E25EE36091B5047091B6048091B704B0
:108530009091B8040E94CDACAB01BC0180E091E108
:108540000E9486162CEA35EC47E25EE36091B9049E
:108550007091BA048091BB049091BC040E9404AF56
:10856000AB01BC018DEF90E10E9486168AE00E946B
:10857000BB18C11110C00E9439168EEE90E10E9406
:108580002B168DE990E10E942B168AE990E10E945A
:108590002B160E9439164091610550916205609139
:1085A00063057091640585EE90E10E9476168AE07D
:1085B0000E94BB18C11108C00E94391684ED90E1D9
:1085C0000E942B160E9439164091E3055091E40554
:1085D0006091E5057091E6058BEC90E10E947616BE
:1085E0008AE00E94BB18C11108C00E94391682EBB4
:1085F00090E10E942B160E9439164091530550912C
:108600005405609155057091560589EA90E10E94E4
:10861000A0164091570550915805609159057091E9
:108620005A0586EA90E10E94A01640915B055091A0
:108630005C0560915D0570915E0583EA90E10E94A2
:10864000A0168AE0CF910C94BB182F923F924F92C4
:108650005F926F927F928F929F92AF92BF92CF92D2
:10866000DF92EF92FF920F931F93CF93DF93CDB7DB
:10867000DEB7C45AD1090FB6F894DEBF0FBECDBF26
:108680002DB73EB7CD55DF4F39832883C35AD0402D
:10869000C756DF4F19821882C959D04084E690E04E
:1086A000C956DF4F99838883C759D0400E94D81696
:1086B00001E09E0127563F4F44E050E0BE016F5657
:1086C0007F4FCE0189569F4F0E9431179E0127563A
:1086D0003F4F42E050E0BE016B567F4FCE018956BE
:1086E0009F4F0E94311743E050E0BE016F567F4F0D
:1086F00083E193E00E949DB4892B39F1CC56DF4F82
:108700008881C459D040882359F08FE3CF56DF4F7A
:108710008883C159D040CE56DF4F1882C259D0400D
:108720000E94391682EC93E10E942B16BE016F560F
:108730007F4F89EB93E10E943F168BEA93E10E9401
:108740002B1681E0809360052BC5C357DF4F18823D
:1087500019821A821B82CD58D040C756DF4F19822A
:108760001882C959D04001E09E0127563F4F41E091
:1087700050E0BE0164567F4FCE0189569F4F0E9444
:1087800031178DB79EB7C156DF4F99838883CF5974
:10879000D0406E019DE7C90ED11C80E1EDEBF2E007
:1087A000D60101900D928A95E1F77E01EDE6EE0E7D
:1087B000F11C80E1EDECF2E0D70101900D928A9579
:1087C000E1F780E1EDEDF2E09E012F5F3F4F5901AF
:1087D000D90101900D928A95E1F7C456DF4F488187
:1087E000CC59D04050E04D5F5F4F440F551F440FB0
:1087F000551F8DB79EB7841B950B0FB6F8949EBF7F
:108800000FBE8DBFEDB7FEB731961F0100915F051A
:1088100011E0012728563F4FBF01CE0189569F4FD7
:108820000E94311700915F0501279E0127563F4F97
:1088300044E050E061E876E0CE0189569F4F0E9407
:108840003117C456DF4F8880CC59D040912CF3E0CB
:108850008F0E911C880C991C880C991C2DB73EB763
:10886000281939090FB6F8943EBF0FBE2DBF8DB73A
:108870009EB701962C01EDB7FEB7E819F9090FB6BE
:10888000F894FEBF0FBEEDBF2DB73EB72F5F3F4F31
:10889000390100915F0501279E0127563F4FA40132
:1088A000BC01CE0189569F4F0E94311700915F0590
:1088B00001279E0127563F4FA401B301CE018956DF
:1088C0009F4F0E94311730915F05C256DF4F3883AA
:1088D000CE59D040332309F4CAC011E0C256DF4F4D
:1088E0000881CE59D04001279E0127563F4F44E0D2
:1088F00050E065EA76E0CE0189569F4F0E9431171D
:1089000000915F0501279E0127563F4F44E050E04C
:1089100069EA76E0CE0189569F4F0E943117009197
:108920005F0501279E0127563F4F44E050E06DEA66
:1089300076E0CE0189569F4F0E94311700915F0566
:1089400001279E0127563F4F44E050E061EB76E05F
:10895000CE0189569F4F0E94311700915F05012774
:108960009E0127563F4F44E050E065EB76E0CE0194
:1089700089569F4F0E94311700915F0501279E0184
:1089800027563F4F40E150E061E476E0CE01895642
:108990009F4F0E94311700915F0501279E012756C6
:1089A0003F4F44E050E0BE0163577F4FCE018956F0
:1089B0009F4F0E943117C156DF4F88819981CF594F
:1089C000D0400FB6F8949EBF0FBE8DBF00915F05DB
:1089D00001279E0127563F4F4CE050E067E775E0C6
:1089E000CE0189569F4F0E94311700915F050127E4
:1089F0009E0127563F4F44E050E0BE0163577F4F32
:108A0000CE0189569F4F0E94311700915F050127C3
:108A10009E0127563F4F44E050E0BE0163577F4F11
:108A2000CE0189569F4F0E94311701E09E012756C3
:108A30003F4F41E050E0B701CE0189569F4F0E9461
:108A400031179E0127563F4F41E050E0BE016F5F56
:108A50007F4FCE0189569F4F0E943117F701A080AA
:108A60008981A89E50011124812C912C9DC0C4564F
:108A7000DF4F8881CC59D04090E09C012E5F3F4F62
:108A8000CF55DF4F39832883C15AD040A1E7B6E0E4
:108A900040E050E080E090E04601B70131E0C3568D
:108AA000DF4F3883CD59D040CF55DF4FE881F98172
:108AB000C15AD040E817F90764F4C356DF4F188253
:108AC000CD59D0409C018430910558F023E030E02E
:108AD00008C0F101E40FF51F00811181228133816B
:108AE0000BC0220F331F220F331FF401E20FF31FBD
:108AF00000811181228133810D931D932D933D932C
:108B0000C356DF4FF881CD59D040FF2341F0F20129
:108B1000E40FF51F008111812281338111C09C0176
:108B20008430910510F023E030E0220F331F220F34
:108B3000331FFB01E20FF31F00811181228133817A
:108B400050960D931D932D933C935397C356DF4F2F
:108B50002881CD59D040222341F0F301E40FF51FC5
:108B6000008111812281338111C09C0184309105E3
:108B700010F023E030E0220F331F220F331FF501E6
:108B8000E20FF31F008111812281338190960D93B2
:108B90001D932D933C93939701964C5F5F4F8430C8
:108BA000910509F07BCF99CE00915F058A149B0453
:108BB00091F001279E0127563F4F44E050E0BE014F
:108BC00063577F4FCE0189569F4F0E9431173FEF69
:108BD000831A930AE9CF11E001279E0127563F4FE0
:108BE00044E050E061E675E0CE0189569F4F0E9457
:108BF000311700915F0501279E0127563F4F44E240
:108C000050E06CE176E0CE0189569F4F0E9431170B
:108C100001E09E0127563F4F41E050E0BE016556FE
:108C20007F4FCE0189569F4F0E9431179E012756D4
:108C30003F4F41E050E0B601CE0189569F4F0E9460
:108C4000311700915F0501279E0127563F4F44E0F1
:108C500050E0B701CE0189569F4F0E943117009115
:108C60005F0501279E0127563F4F44E050E0BE01BB
:108C70006F5F7F4FCE0189569F4F0E943117C556B7
:108C8000DF4FA880CB59D040F6018081A89E5001CB
:108C90001124812C912C00915F058A149B0491F082
:108CA00001279E0127563F4F44E050E0BE01635725
:108CB0007F4FCE0189569F4F0E943117FFEF8F1AC9
:108CC0009F0AE9CF11E001279E0127563F4F41E05F
:108CD00050E0B701CE0189569F4F0E943117009195
:108CE0005F0501279E0127563F4F41E050E0BE013E
:108CF0006F5F7F4FCE0189569F4F0E9431170091C1
:108D00005F0501279E0127563F4F40E150E0BE011D
:108D10006F5F7F4FCE0189569F4F0E9431170091A0
:108D20005F0501279E0127563F4F44E050E0B70101
:108D3000CE0189569F4F0E94311700915F05012790
:108D40009E0127563F4F44E050E0BE016F5F7F4FCA
:108D5000CE0189569F4F0E94311700915F05012770
:108D60009E0127563F4F42E050E0B601CE018956A2
:108D70009F4F0E94311700915F0501279E012756E2
:108D80003F4F40E150E0BE016F5F7F4FCE018956FB
:108D90009F4F0E94311700915F0501112EC08980FD
:108DA0009A80AB80BC8020E030E84BE355E4C501FD
:108DB000B4010E94C6AC882301F18092A304909272
:108DC000A404A092A504B092A6048D819E81AF81D7
:108DD000B8858093A7049093A804A093A904B093A6
:108DE000AA0489859A85AB85BC858093AB04909352
:108DF000AC04A093AD04B093AE0411E001279E0132
:108E000027563F4F42E050E0BE016F5F7F4FCE01DB
:108E100089569F4F0E94311700915F0501279E01DF
:108E200027563F4F4CE050E0BE016F5F7F4FCE01B1
:108E300089569F4F0E94311700915F05011115C09F
:108E400020E030E84BE355E469817A818B819C8195
:108E50000E94C6AC882349F08CE0FE013196A1EB5C
:108E6000B4E001900D928A95E1F711E001279E018F
:108E700027563F4F42E050E0BE016F5F7F4FCE016B
:108E800089569F4F0E94311700915F0501279E016F
:108E900027563F4F41E050E0BE016F5F7F4FCE014C
:108EA00089569F4F0E94311700915F0501279E014F
:108EB00027563F4F40E250E0BE016F5F7F4FCE012B
:108EC00089569F4F0E94311700915F0501279E012F
:108ED00027563F4F41E050E0B701CE0189569F4FE2
:108EE0000E94311700915F0501279E0127563F4FD1
:108EF00045E050E0BE016F5F7F4FCE0189569F4F26
:108F00000E94311780915F05811102C00E94652F78
:108F100000915F0511E001279E0127563F4F4AE16E
:108F200050E0BE016F5F7F4FCE0189569F4F0E9478
:108F3000311700915F0501279E0127563F4F44E3FB
:108F400050E0BE016F5F7F4FCE0189569F4F0E9458
:108F5000311700915F0501279E0127563F4F46E0DC
:108F600050E0BE016F5F7F4FCE0189569F4F0E9438
:108F7000311700915F0501279E0127563F4F4DE0B5
:108F800050E0BE016F5F7F4FCE0189569F4F0E9418
:108F9000311700915F0501279E0127563F4F44E09E
:108FA00050E0BE016F5F7F4FCE0189569F4F0E94F8
:108FB000311700915F0501110CC089819A81AB8145
:108FC000BC818093E3059093E405A093E505B093FD
:108FD000E60581E008279E0127563F4F4CE050E010
:108FE000BE016F5F7F4FCE0189569F4F0E943117A0
:108FF00000915F05011109C08CE0FE013196A3E5E7
:10900000B5E001900D928A95E1F711E001279E01EC
:1090100027563F4F4CE650E0BE016F5F7F4FCE01B9
:1090200089569F4F0E94311719821A821B821C8217
:109030001D821E821F82188619861A861B861C8630
:1090400000915F0501279E0127563F4F4CE050E0FD
:10905000BE016F5F7F4FCE0189569F4F0E9431172F
:1090600000915F0501279E0127563F4F48E050E0E1
:10907000BE016F5F7F4FCE0189569F4F0E9431170F
:10908000C956DF4F88819981C759D04084569109CC
:109090000E94CC3B809360058823C1F00E94391662
:1090A000C956DF4F68817981C759D040645671092C
:1090B00083EA93E10E945C1667E472E08BE993E136
:1090C0000E9496168AE00E94BB1860C0C756DF4F08
:1090D00028813981C959D040CB56DF4F8881998189
:1090E000C559D0402817390729F1109360050E940F
:1090F0003C168BE793E10E942B166AE070E0CB569A
:10910000DF4F88819981C559D0400E94C31986E7F5
:1091100093E10E942B166AE070E0C756DF4F88810A
:109120009981C959D0400E94C31986E693E10E94F3
:109130002B162CC080915F05811128C00E94391622
:1091400003E113E0F80181918F01882319F00E9457
:10915000BB18F8CFC956DF4F68817981C759D04015
:109160006456710989E493E10E945C16C756DF4F8B
:1091700048815981C959D04060E070E08CE393E1A7
:109180000E94A01689E393E10E942B1680915F054F
:10919000811106C080916005811102C00E944B3B85
:1091A00080915F05811102C00E94AC400E94DA16D6
:1091B0009091600581E08927CD55DF4F2881398165
:1091C000C35AD0400FB6F8943EBF0FBE2DBFCC554A
:1091D000DF4F0FB6F894DEBF0FBECDBFDF91CF914A
:1091E0001F910F91FF90EF90DF90CF90BF90AF90C5
:1091F0009F908F907F906F905F904F903F902F90B7
:10920000089581E080935F0520DA10925F0508954C
:10921000F8DF81111ACA0E94623F81E00895BF926F
:10922000CF92DF92EF92FF920F931F93CF93DF9332
:10923000CDB7DEB728970FB6F894DEBF0FBECDBF0F
:109240009091DA04981709F47AC0B82E882309F4AB
:1092500053C080E090E0A0EAB0E48D839E83AF83AA
:10926000B887C0906105D0906205E0906305F090EA
:10927000640520E030E0A901C701B6010E94C6AC38
:1092800087FF0CC0A701960160E070E080EA90E4DF
:109290000E94ECAB6D837E838F83988720E030E063
:1092A0004FE153E46D817E818F8198850E94C9AE24
:1092B000181644F480E090E0AFE1B3E48D839E8320
:1092C000AF83B8872091B3053091B4054091B505BF
:1092D0005091B6056D817E818F8198850E94C9AEBF
:1092E000181654F419821A821B821C82BE016F5F09
:1092F0007F4FCE010596F6D46091AB057091AC0519
:109300008091AD059091AE052091AF053091B005EB
:109310004091B1055091B20519821A821B821C82BC
:10932000E090B305F090B4050091B5051091B60535
:10933000FE0131966F01FAD38B2D0E94002E80E042
:1093400028960FB6F894DEBF0FBECDBFDF91CF9148
:109350001F910F91FF90EF90DF90CF90BF900895F5
:109360002F923F924F925F926F927F928F929F9235
:10937000AF92BF92CF92DF92EF92FF920F931F9323
:10938000CF93DF93CDB7DEB7A0970FB6F894DEBFCB
:109390000FBECDBF1C017F8F6E8F498F28A3DC01CC
:1093A0008D909D90AD90BC90FB014080518062807B
:1093B000738022ED30E040EE50ECC301B201002397
:1093C00009F43BC00E94C9AE87FD49C227E030E0E6
:1093D0004EE353E4C301B2010E94C6AC18160CF46C
:1093E0003EC223EA31E040E450ECC501B4010E94E2
:1093F000C9AE87FD34C227E030E042E253E4C50144
:10940000B4010E94C6AC18160CF429C227E030E063
:1094100041E253E4C501B4010E94C6AC18160CF435
:109420001EC227E030E041E253E4C301B2010E94D2
:10943000C6AC18160CF413C224C00E94C9AE87FD36
:109440000EC227E030E04EE353E4C301B2010E94B4
:10945000C6AC18160CF403C223EA31E040E450EC29
:10946000C501B4010E94C9AE87FDF9C127E030E013
:1094700042E253E4C501B4010E94C6AC18160CF4D4
:10948000EEC1E090B305F090B4050091B5051091E0
:10949000B6058091480290914902A0914A02B0918C
:1094A0004B028A8F9B8FAC8FBD8F8091420290912F
:1094B0004302A0914402B0914502809348029093E8
:1094C0004902A0934A02B0934B0219821A821B826E
:1094D0001C82DE0111966D01A3019201C501B40148
:1094E00025D381E09CDE81113EC18091BC0582FFC5
:1094F00011C0209161053091620540916305509142
:10950000640560E070E080E890EC0E94ECAB6B01D9
:109510007C0106C0C12CD12C40E2E42E41ECF42E9B
:10952000CD8ADE8AEF8AF88E812C912CA12C31E431
:10953000B32E898A9A8AAB8ABC8ABE016F5E7F4F3E
:10954000CE014596CFD31091DE041092DE0482E066
:1095500031D206D212FD05C060E070E080EC9FE7DA
:10956000BDC04090B3055090B4056090B5057090B3
:10957000B60589829A82AB82BC8220E030E040EA64
:1095800050E4C301B2010E94EDAB6D837E838F83F3
:1095900098878E010B5F1F4FBE016F5F7F4FC80121
:1095A000A1D3CD86DE86EF86F88A80E090E0A0E841
:1095B000BFE389879A87AB87BC87BE01675F7F4F10
:1095C000CE010D968FD3F090DE041092DE0482E07F
:1095D000F1D1C6D1F2FEC0CF8091580C8F3F09F473
:1095E0005BC0C090B305D090B405E090B505F09095
:1095F000B6058090B3059090B405A090B505B090E5
:10960000B60520E030E040E05FE3C701B6010E940C
:10961000EDAB9B01AC01C501B4010E94C6AC87FF54
:109620001CC01C991AC080E090E0A0E8BFE38983C9
:109630009A83AB83BC832AE037ED43EA5BE3C50141
:10964000B4010E94EDAB6D837E838F839887BE014A
:109650006F5F7F4FC80146D3CCCFA7019601C501EC
:10966000B4010E94ECAB9B01AC016091610C709164
:10967000620C8091630C9091640C0E94EDAB60933E
:10968000610C7093620C8093630C9093640C8091D6
:10969000580C8F5F8093580C20E030E040E450E499
:1096A0006091B3057091B4058091B5059091B605B0
:1096B0000E9404AF6B017C01A3019201C301B201BE
:1096C0000E94EDAB9B01AC01C701B6010E94EDAB5E
:1096D0002DEC3CEC4CE45EE30E9404AF209161056C
:1096E0003091620540916305509164050E94EDAB95
:1096F0007B018C01898D8250823048F580E090E0BA
:10970000A0E0B1E489839A83AB83BC836091B30505
:109710007091B4058091B5059091B605A98DA330DF
:1097200029F020E030E040EA50E404C020E030E0DE
:1097300048EC51E40E94EDAB6D837E838F83988764
:10974000BE016F5F7F4FCE010596CCD207C0B98DA9
:10975000B13021F480E063DD811105C0E8A1E33080
:1097600008F45DC008C098A1933008F481C0E12CD2
:10977000F12C00EC1FE727E1C22E23E0D22ED60108
:109780008D916D01882319F00E94BB18F8CF2091AC
:109790006B0530916C0540916D0550916E05F1019E
:1097A00060817181828193810E94EDAB43E050E042
:1097B0000E94391A9FE1C92E93E0D92ED6018D91CE
:1097C0006D01882319F00E94BB18F8CF20916F0516
:1097D000309170054091710550917205EE8DFF8DAD
:1097E00060817181828193810E94EDAB43E050E002
:1097F0000E94391A84E2C82E83E0D82ED6018D91BA
:109800006D01882319F00E94BB18F8CF43E050E0A7
:10981000B701C8010E94391A8AE00E94BB188A8DDC
:109820009B8DAC8DBD8D8093480290934902A0938F
:109830004A02B0934B029701A801B701C8010E94E8
:10984000B2AF882389F080E0EADC0E943C1685E113
:1098500094E10E942B162E2D7F2DC8011AC020E006
:1098600070E080EC9FE715C02E2D7F2DC80111C040
:109870008A8D9B8DAC8DBD8D80934802909349025B
:10988000A0934A02B0934B02E12CF12C00EC1FE7AD
:10989000DACFC22ED72E7C01C701B601A0960FB633
:1098A000F894DEBF0FBECDBFDF91CF911F910F9116
:1098B000FF90EF90DF90CF90BF90AF909F908F90F0
:1098C0007F906F905F904F903F902F9008950F93EF
:1098D0001F93CF93DF93CBEAD5E00BE615E0F801B9
:1098E0002081318142815381688179818A819B8184
:1098F0000E94EDABAB01BC0184EA94E10E947616B4
:10990000F80124813581468157816C817D818E816A
:109910009F810E94EDABAB01BC0180EA94E10E9403
:109920007616F801208531854285538568857985CD
:109930008A859B850E94EDABAB01BC018CE994E16B
:109940000E9476164C855D856E857F8588E994E159
:109950000E947616DF91CF911F910F910C942F39B1
:1099600027EB35E043EB55E06FEA75E08BEA95E0D5
:109970000C94E26887EB95E00C942F69CF93DF930A
:1099800080E00E940059CFE8D5E0688379838A831C
:109990009B8381E00E9400596C837D838E839F832B
:1099A00082E00E940059688779878A879B87DF91C8
:1099B000CF9108951F93CF93DF93CDB7DEB7609714
:1099C0000FB6F894DEBF0FBECDBF182FD7DF809142
:1099D0008F0590919005A0919105B0919205898392
:1099E0009A83AB83BC838091930590919405A09159
:1099F0009505B09196058D839E83AF83B88780913E
:109A0000970590919805A0919905B0919A0589873D
:109A10009A87AB87BC878091B7059091B805A091D4
:109A2000B905B091BA058D879E87AF87B88BCE01F7
:109A300001960E9445581E3F51F480E1FE01319687
:109A4000ABEAB5E001900D928A95E1F716C024E0EB
:109A5000129FC0011124FC01E555FA4FA1E0B0E0CE
:109A6000AC0FBD1FA80FB91F8D919D910D90BC919A
:109A7000A02D80839183A283B38360960FB6F89460
:109A8000DEBF0FBECDBFDF91CF911F910895AF9282
:109A9000BF92CF92DF92EF920F931F93A12CB12C24
:109AA0006501E12C08E412E027EB35E043EB55E0DB
:109AB0006FEA75E08BEA95E00E94A6671F910F910F
:109AC000EF90DF90CF90BF90AF900895AF92BF928C
:109AD000CF92DF92EF920F931F93CF93DF9300D03B
:109AE0001F92CDB7DEB769837A838B839C83A12CC9
:109AF000B12C6501E12C8E010F5F1F4F27EA35E085
:109B000043EA55E06FE975E08BE995E00E94A667AE
:109B10000F900F900F900F90DF91CF911F910F91A9
:109B2000EF90DF90CF90BF90AF9008954F925F92EB
:109B30006F927F928F929F92AF92BF92CF92DF925D
:109B4000EF92FF920F931F93CF93DF93CDB7DEB7C2
:109B50002C970FB6F894DEBF0FBECDBF6D837E830A
:109B60008F83988729873A874B875C8747015801FD
:109B700036018091480290914902A0914A02B09129
:109B80004B0289839A83AB83BC83D601CD90DD9051
:109B9000ED90FC9020E030E0A901C701B6010E94E1
:109BA000C6AC811106C0EFEAF4E1C590D590E5900E
:109BB000F490A50194016091B3057091B405809172
:109BC000B5059091B6050E94C6AC87FF11C0C09242
:109BD0004802D0924902E0924A02F0924B028092EF
:109BE000B3059092B405A092B505B092B6054FDFCB
:109BF000F301408051806280738020E030E0A90151
:109C0000C301B2010E94C6AC811108C0409042025B
:109C10005090430260904402709045024092480286
:109C20005092490260924A0270924B028D819E814D
:109C3000AF81B8858093AB059093AC05A093AD053B
:109C4000B093AE0589859A85AB85BC858093AF05B9
:109C50009093B005A093B105B093B20518DFA501AC
:109C600094016091B3057091B4058091B505909110
:109C7000B6050E94C9AE18168CF4C0924802D09264
:109C80004902E0924A02F0924B028092B305909210
:109C9000B405A092B505B092B605F9DE89819A8126
:109CA000AB81BC818093480290934902A0934A0201
:109CB000B0934B022C960FB6F894DEBF0FBECDBF0B
:109CC000DF91CF911F910F91FF90EF90DF90CF9098
:109CD000BF90AF909F908F907F906F905F904F90CC
:109CE0000C941459CF92DF92EF92FF920F931F932F
:109CF0006B01FC01E080F18002811381EBEAF5E069
:109D0000248135814681578160817181828193816F
:109D10000DDF1F910F91FF90EF90DF90CF9008958E
:109D2000CF92DF92EF92FF920F931F936A01E09020
:109D3000B305F090B4050091B5051091B605FB018F
:109D40002081318142815381FC0160817181828156
:109D50009381ECDE1F910F91FF90EF90DF90CF90F9
:109D600008958823F9F08091480290914902A091CA
:109D70004A02B0914B028093670590936805A093C7
:109D80006905B0936A0580914602909147029093CD
:109D900066058093650584E690E090934702809382
:109DA000460208958091670590916805A091690524
:109DB000B0916A058093480290934902A0934A02A9
:109DC000B0934B0280916505909166059093470290
:109DD0008093460208958091480290914902A09193
:109DE0004A02B0914B028093670590936805A09357
:109DF0006905B0936A05809146029091470290935D
:109E000066058093650584E690E090934702809311
:109E10004602089580E0A5CFCF92DF92EF92FF92A5
:109E2000CF93DF9320914102222309F443C0EC0138
:109E3000C0902902D0902A02E0902B02F0902C02D0
:109E4000A7019601688179818A819B810E94C9AEB0
:109E5000181624F4C882D982EA82FB82C0902D02AF
:109E6000D0902E02E0902F02F0903002A7019601D0
:109E70006C817D818E819F810E94C9AE181624F469
:109E8000CC82DD82EE82FF82C0903102D09032021D
:109E9000E0903302F0903402A7019601688579853D
:109EA0008A859B850E94C9AE181624F4C886D98677
:109EB000EA86FB86DF91CF91FF90EF90DF90CF9005
:109EC000089524E0829FC0011124FC01EA51FB4E59
:109ED0004591559165917491FC01EB5CFD4F408378
:109EE000518362837383FC01E652FB4E4591559189
:109EF00065917491FC01E75DFD4F4083518362835E
:109F0000738308958F929F92AF92BF92CF92DF9208
:109F1000EF92FF928BE995E07FDF8091930383FDC1
:109F20007DC0C090A705D090A805E090A905F0904D
:109F3000AA052091B7053091B8054091B905509117
:109F4000BA05C701B6010E94C6AC882309F466C0F1
:109F50006091D3047091D4048091D5049091D6047B
:109F600020919C04211117C00E9435AD2091190247
:109F700030911A026217730774F4C092B705D09239
:109F8000B805E092B905F092BA050E9439168DE73E
:109F900094E10E942B168090A7059090A805A090B0
:109FA000A905B090AA052091B7053091B805409158
:109FB000B9055091BA05C501B4010E94ECAB6B0123
:109FC0007C0120E030E0A9010E94C9AE87FF04C0F7
:109FD000C701B601905802C0C701B60120914C02DA
:109FE00030914D0240914E0250914F020E9404AFB9
:109FF00020E030E048E453E40E94C9AE181674F43F
:10A000008092B7059092B805A092B905B092BA05B2
:10A010000E9439168EE594E10E942B16609146024B
:10A0200070914702072E000C880B990B0E9468ADB7
:10A03000209148023091490240914A0250914B02CE
:10A040000E9404AF2AE037ED43E25CE30E9404AFD4
:10A050003DDD80E1EBE9F5E0ABEAB5E001900D9282
:10A060008A95E1F7FF90EF90DF90CF90BF90AF908F
:10A070009F908F9008951F93CF93DF93882329F0AB
:10A08000D091BD05D095D17001C0D0E0662339F0E4
:10A090001091BD051695117081E0182701C010E0E0
:10A0A000442341F0C091BD05C2FBCC27C0F981E03B
:10A0B000C82701C0C0E0D11104C0111102C0CC23D7
:10A0C000E9F00E94391688E594E10E942B16DD2301
:10A0D00021F086E594E10E942B16112321F084E5FE
:10A0E00094E10E942B16CC2321F082E594E10E949A
:10A0F0002B168AE494E10E942B16C1E08C2FDF918D
:10A10000CF911F910895CF92DF92EF92FF92CF935C
:10A11000DF93C82FD0E0FE01E95BFB4E84918111F3
:10A1200007C00E94391685E294E10E942B168AE04E
:10A13000FE01EE0FFF1FEE0FFF1FE955FB4EC5900E
:10A14000D590E590F490682F70E080E090E00E9458
:10A1500068AD9B01AC01C701B6010E94CDACDF9197
:10A16000CF91FF90EF90DF90CF9008954F925F9244
:10A170006F927F928F929F92AF92BF92CF92DF9217
:10A18000EF92FF920F931F93CF93DF93CDB7DEB77C
:10A1900068970FB6F894DEBF0FBECDBF2A013B0112
:10A1A0006901E82EF12CF701ED54FB4EE491AA244D
:10A1B000A3941E160CF4A12CBB24B39420E030E031
:10A1C000A901C301B2010E94C9AE18160CF0B12C4E
:10A1D00080E00E94005969837A838B839C8381E0AD
:10A1E0000E9400596D837E838F83988782E00E944E
:10A1F000005969877A878B879C8783E00E94005982
:10A200006D877E878F87988BEE0CFF1CEE0CFF1CF2
:10A2100088248394912C8C0E9D1E8E0C9F1CF4011F
:10A2200010821182128213829E01235F3F4FAE0182
:10A23000475F5F4FBE016B5F7F4FCE0101960E946B
:10A240000768F4014082518262827382198A1A8AF5
:10A250001B8A1C8A20E030E0A901B801C6010E94D7
:10A26000C6AC811108C0F701E955FB4E8591959167
:10A27000A591B49102C0C801D6018D8B9E8BAF8B86
:10A28000B88FCE0141966C01E12C8E010B5E1F4F01
:10A290009E01235F3F4FAE01475F5F4FBE016B5F83
:10A2A0007F4F40970E94C366BFD7AB100E94C42D5A
:10A2B00068960FB6F894DEBF0FBECDBFDF91CF9189
:10A2C0001F910F91FF90EF90DF90CF90BF90AF90D4
:10A2D0009F908F907F906F905F904F900895CF9355
:10A2E000DF9324E0829FC0011124EC01C559DA4FAD
:10A2F000FC01E958FA4FDC01AD57BA4F2D913D9161
:10A300004D915C9160817181828193810E94EDAB5E
:10A31000688379838A839B83DF91CF910895CF935C
:10A32000DF9321E030E0082E01C0220F0A94EAF703
:10A330009091BC05922B9093BC059091BD05292B63
:10A340002093BD0594E0899FE0011124FE01ED57A3
:10A35000FA4F1082118212821382C1DFFE01E25392
:10A36000FB4E85919591A591B491C555DA4F88839F
:10A370009983AA83BB83DF91CF9108954F925F9217
:10A380006F927F928F929F92AF92BF92FF920F93A4
:10A390001F93CF93DF93833008F06AC0F82EC82F45
:10A3A000D0E0FE01ED54FB4E8491CC0FDD1FCC0FAD
:10A3B000DD1FFE01EE53FB4E459055906590749065
:10A3C000682F880F770B880B990B0E9468AD4B01A3
:10A3D0005C0120E030E040EC5FE3C301B2010E9489
:10A3E00004AFA50194010E9404AFAB01BC0100E0E1
:10A3F00010E098018F2DBADEFE01EA54FB4E259144
:10A40000359145915491C501B4010E9404AF4B01AF
:10A410005C0120E030E0A9010E94C6AC8823C1F0B5
:10A42000B501A401705800E010E098018F2D9EDE68
:10A430008F2D69DE2B013C01A5019401C501B401FA
:10A440000E94EDABAB01BC01930182018F2D8EDE2A
:10A450008F2D65DF85DAFE01E556FA4FC555DA4FD7
:10A4600088819981AA81BB8180839183A283B383F0
:10A47000DF91CF911F910F91FF90BF90AF909F9070
:10A480008F907F906F905F904F90089594E0899F98
:10A49000F0011124E958FA4F40835183628373839A
:10A4A0001ECF80E1E0E0F6E0DF01982F1D929A9543
:10A4B000E9F7E3EDF5E0DF01982F1D929A95E9F7B2
:10A4C000ECEEF5E0DF011D928A95E9F71092E805C0
:10A4D0001092E9051092EA051092EB058CE196E0E6
:10A4E0000E947FA51092BC061092BF061092BD0676
:10A4F0001092BE061092B90608954F925F926F9225
:10A500007F928F929F92AF92BF92CF92DF92EF9203
:10A51000FF920F931F93CF93DF93CDB7DEB768976A
:10A520000FB6F894DEBF0FBECDBF8C015B014A01B0
:10A53000FC01EF5BFF4F60817181828193810E94FA
:10A5400066AD6B017C01D5012D913D914D915C91E2
:10A550000E9404AF0E94B3AC0E943AAD69877A872B
:10A560008B879C87F4012081318142815381C7010F
:10A57000B6010E9404AF0E94B3AC0E943AAD6D8751
:10A580007E878F87988B29853A854B855C85283710
:10A5900031054105510540F488E790E0A0E0B0E0C6
:10A5A00089879A87AB87BC872D853E854F855889DB
:10A5B000283731054105510540F488E790E0A0E0D7
:10A5C000B0E08D879E87AF87B88B9801235B3F4FA4
:10A5D000D9018D919D910D90BC91A02D89839A8375
:10A5E000AB83BC83BC01CD010E9468AD2B013C0153
:10A5F00069857A858B859C850E9466AD698B7A8B8F
:10A600008B8B9C8B20E030E0A901C301B2010E943A
:10A61000C6AC882329F1A7019601C701B6010E94A3
:10A6200004AF4B015C0129893A894B895C89CA01D5
:10A63000B9010E9404AF9B01AC01C501B4010E94A5
:10A64000ECAB4B015C01A3019201C301B2010E947A
:10A65000EDAB9B01AC01C501B4010E94CDAC03C0C0
:10A6600060E070E0CB010E94B3AC0E943AAD6D8314
:10A670007E838F83988769817A818B819C81909575
:10A680008095709561957F4F8F4F9F4F0E9468AD69
:10A690004B015C016D857E858F8598890E9466AD32
:10A6A00069837A838B839C8320E030E0A901C50114
:10A6B000B4010E94C6AC882349F129813A814B81BB
:10A6C0005C81CA01B9010E9404AF6D8B7E8B8F8BB8
:10A6D000988FA7019601C701B6010E9404AF9B01A4
:10A6E000AC016D897E898F89988D0E94ECAB6B01DE
:10A6F0007C01A5019401C501B4010E94EDAB9B0151
:10A70000AC01C701B6010E94CDAC03C060E070E0AF
:10A71000CB010E94A3ADF80185A096A0A7A0B0A48C
:10A72000750164012D813E814F815885C21AD30A7B
:10A73000E40AF50A0E943AADC61AD70AE80AF90AED
:10A74000F7FE73C020E030E0A901C301B2010E940E
:10A75000C6AC882309F443C0A3019201C301B2012E
:10A760000E94EDAB6B017C01C501B4010E9466AD96
:10A770009B01AC01C701B6010E9404AF6B017C01D3
:10A7800029893A894B895C89CA01B9010E9404AFC1
:10A790009B01AC01C701B6010E94ECAB6B017C01CF
:10A7A00029813A814B815C81CA01B9010E9404AFC1
:10A7B0009B01AC01C701B6010E94EDAB6B017C01AE
:10A7C00020E030E040E850E4C301B2010E9404AF51
:10A7D0009B01AC01C701B6010E94CDAC03C060E093
:10A7E00070E0CB010E94B3AC7B016C0120E030E053
:10A7F000A9010E94C9AE181624F0E12CF12CC12C3D
:10A80000D12CB701C6010E943AAD6D837E838F8340
:10A81000988786169706A806B90620F48D829E8230
:10A82000AF82B886C12CD12C76018D819E81AF81FB
:10A83000B885F80181A792A7A3A7B4A7C80ED91E0F
:10A84000EA1EFB1EC5A6D6A6E7A6F0AAEB5BFF4F45
:10A8500029853A854B855C852083318342835383E8
:10A8600034968D859E85AF85B88980839183A28338
:10A87000B38368960FB6F894DEBF0FBECDBFDF91ED
:10A88000CF911F910F91FF90EF90DF90CF90BF90ED
:10A89000AF909F908F907F906F905F904F900895B2
:10A8A0002F923F924F925F926F927F928F929F92E0
:10A8B000AF92BF92CF92DF92EF92FF920F931F93CE
:10A8C000CF93DF93009709F471C08B01EC01D98419
:10A8D000CA847B846C848D809E80AF80B8842D2D4B
:10A8E0003C2D472D562DC501B4010E94C6AC8111E7
:10A8F00008C00115110509F459C0F801808180FFD5
:10A9000055C0888181FD34C00115110531F0F80171
:10A91000258036804780508408C08BE0282E87ED44
:10A92000382E83E2482E8BE3582E89899A89AB8989
:10A93000BC89BC01CD0190589B01AC010E94EDABDC
:10A940002D853E854F8558890E9404AF9B01AC013F
:10A95000C201B1010E94ECAB7B018C019B01AC01F7
:10A960006D2D7C2D872D962D0E94C6AC87FF04C0CF
:10A97000ED2CFC2C072D162D9701A801C501B40163
:10A980000E94C6AC882391F0888181608883CE01C3
:10A990000E94B932882321F088818E7F888306C087
:10A9A000A701B8014D835E836F837887DF91CF91D4
:10A9B0001F910F91FF90EF90DF90CF90BF90AF90DD
:10A9C0009F908F907F906F905F904F903F902F90CF
:10A9D0000895FF920F931F93CF93DF93C091BF060B
:10A9E000C150CF70D091BD068091BF06D817E9F055
:10A9F00060E070E086E5F82ECD17B9F0FC9E80018E
:10AA000011240054194FF801808183FD03C0C8014F
:10AA100047DFB801C150CF708091BD06D81761F3F0
:10AA2000CD1719F0DF5FDF70F7CFDF91CF911F9166
:10AA30000F91FF9008954F925F926F927F928F9245
:10AA40009F92AF92BF92FF920F931F93CF93DF938A
:10AA5000009709F459C0F42EEB018C01FC018081B0
:10AA600081FD3CC045805680678070848D809E80CB
:10AA7000AF80B884A5019401C301B2010E94C6ACA5
:10AA800087FF2CC0F80181899289A389B489BC0110
:10AA9000CD0190589B01AC010E94EDABF8012585DA
:10AAA0003685478550890E9404AF9B01AC01C301E4
:10AAB000B2010E94ECAB2B013C01A50194010E9464
:10AAC000C6AC87FF0BC0888181608883CE010E945D
:10AAD000B932882391F088818E7F888329853A85D1
:10AAE0004B855C856D817E818F8198850E94C6AC87
:10AAF00081110AC0F092BD0607C04D825E826F824E
:10AB00007886F092BD06EACFDF91CF911F910F9129
:10AB1000FF90BF90AF909F908F907F906F905F90CD
:10AB20004F900895CF92DF92EF92FF920F931F9371
:10AB3000CF93DF931091BD06C0E0D0E086E5C82E2C
:10AB40008091BF06181709F1C19EB0011124CB01F5
:10AB50008054994F7C01FC01808183FD0AC00E2D39
:10AB6000DF2C209769F0CE010E94B932882341F092
:10AB700002C00C2FDD2E1F5F1F70C02FDD2DE0CF18
:10AB8000412FB701CE0157DFF6CFDF91CF911F9153
:10AB90000F91FF90EF90DF90CF9008952F923F920A
:10ABA0004F925F926F927F928F929F92AF92BF92DD
:10ABB000CF92DF92EF92FF920F931F93CF93DF9389
:10ABC000CDB7DEB72E970FB6F894DEBF0FBECDBF60
:10ABD0002091BC0629873091BF063B8796E58B857F
:10ABE000E9858E1759F08B8581508F70989FF00101
:10ABF0001124E054F94F208123FD0DC0812C912CAC
:10AC0000A12CB12C1A861C861D861E86212C312C67
:10AC100000E010E01AC08B87E2CFF6E52985F29FAD
:10AC2000C0011124FC01E054F94F1F01808183FF12
:10AC300011C0FA84EC84DD84CE8489858F5F8F70A7
:10AC40008987FA86EC86DD86CE86F9852B85F21318
:10AC5000E4CF93C065817681878190850E9471AF32
:10AC6000F62EE72ED82EC92E0115110509F47FC046
:10AC7000F801808180FD04C0F101808180FF77C0F0
:10AC8000F801808181608083C8010E94B9328111FE
:10AC90006AC0F80161817281838194810E9471AFE1
:10ACA0002B013C019B01AC0160E070E080E89FE378
:10ACB0000E94CDAC4B015C019B01AC016F2D7E2D40
:10ACC0008D2D9C2D0E9404AF69837A838B839C8396
:10ACD000A50194016A857C858D859E850E9404AFBF
:10ACE0006D837E838F839887AE014F5F5F4FBE0178
:10ACF0006B5F7F4FC80101DCF80186A9882399F1B9
:10AD00002091E3053091E4054091E5055091E60579
:10AD1000FD9660817181828193810E9404AF2091B0
:10AD200091063091920640919306509194060E94AC
:10AD300004AF4B015C019B01AC01C301B2010E9455
:10AD400004AF0E943AADF80172AF61AFA501940162
:10AD50006F2D7E2D8D2D9C2D0E9404AF0E943AAD4B
:10AD6000F80174AF63AFF80180818E7F80838F2CF0
:10AD70009E2CAD2CBC2C810160CF2114310409F430
:10AD800073C0F101808181608083C8010E94B93263
:10AD9000811166C0F10161817281838194810E9479
:10ADA00071AF6B017C019B01AC0160E070E080E859
:10ADB0009FE30E94CDAC2B013C012DEC3CEC4CE41C
:10ADC0005DE30E9404AF69837A838B839C83A30134
:10ADD0009201B401C5010E9404AF6D837E838F830D
:10ADE0009887AE014F5F5F4FBE016B5F7F4FC10120
:10ADF00084DBF10186A9882399F12091E305309144
:10AE0000E4054091E5055091E605FD96608171816C
:10AE1000828193810E9404AF209191063091920625
:10AE200040919306509194060E9404AF4B015C013F
:10AE30009B01AC01C701B6010E9404AF0E943AAD6C
:10AE4000F10172AF61AF2DEC3CEC4CE45DE3C50168
:10AE5000B4010E9404AF0E943AADF10174AF63AF38
:10AE6000F10180818E7F80832E960FB6F894DEBF2D
:10AE70000FBECDBFDF91CF911F910F91FF90EF904B
:10AE8000DF90CF90BF90AF909F908F907F906F900A
:10AE90005F904F903F902F9008958091BF069091C2
:10AEA000BD0681508F70891711F093DD3BDE76CEA1
:10AEB000AF92BF92CF92DF92EF92FF920F931F93C8
:10AEC000CF939091BF068091BC06981791F0E091C6
:10AED000BC0686E5E89FF0011124EF5EF84FC081C3
:10AEE0008091BC069091BF06891729F08F5F8F7003
:10AEF000F9CFC091CE04CC2339F10E94A611009164
:10AF0000CF051091D0052091D1053091D205DC01FB
:10AF1000CB01011511052105310571F48C599F4FA5
:10AF2000AF4FBF4F8093CF059093D005A093D1052D
:10AF3000B093D205CFEF1EC0801B910BA20BB30BB9
:10AF4000B7FF18C0CFEF16C01092CF051092D005F2
:10AF50001092D1051092D20560E070E088E0CF91A8
:10AF60001F910F91FF90EF90DF90CF90BF90AF9027
:10AF70000C9472126C2F70E080E090E01F921F9290
:10AF80001F922FEF2F9326E4A22EB12CC12CD12C8F
:10AF9000E12CF12C8701EA9421E030E040E050E020
:10AFA0000E947C150F900F900F900F90D7CFCF92EB
:10AFB000DF92EF92FF920F931F93CF93DF93CDB762
:10AFC000DEB728970FB6F894DEBF0FBECDBF209135
:10AFD0004006222309F44AC06A018B017C0120E06B
:10AFE00030E040E450E4FC01608171818281938112
:10AFF0000E94EDAB6D837E838F83988720E030E0E5
:10B000004EE353E4F80160817181828193810E9453
:10B01000ECAB69837A838B839C839601AE014F5F8F
:10B020005F4FBE016B5F7F4F8CE196E00E94B7A43B
:10B0300020E030E040E450E46D817E818F8198858E
:10B040000E94ECABF701608371838283938320E0DD
:10B0500030E04EE353E469817A818B819C810E94C8
:10B06000EDABF801608371838283938328960FB6DA
:10B07000F894DEBF0FBECDBFDF91CF911F910F912E
:10B08000FF90EF90DF90CF9008950F931F93CF9391
:10B09000DF93CDB7DEB7AC970FB6F894DEBF0FBE27
:10B0A000CDBF20914006222309F450C08C016CE1F1
:10B0B00076E0CE0101960E943AA620E030E040E41E
:10B0C00050E4F80160817181828193810E94EDAB2F
:10B0D00069A77AA78BA79CA720E030E04EE353E452
:10B0E000F80164817581868197810E94ECAB6DA324
:10B0F0007EA38FA398A79801285F3F4FAE014B5DB9
:10B100005F4FBE01675D7F4FCE0101960E94B7A4DD
:10B1100020E030E040E450E469A57AA58BA59CA529
:10B120000E94ECABF801608371838283938320E0FB
:10B1300030E04EE353E46DA17EA18FA198A50E945B
:10B14000EDABF8016483758386839783AC960FB665
:10B15000F894DEBF0FBECDBFDF91CF911F910F914D
:10B16000089580916F0081FB992790F981FF05C0B8
:10B1700080916F008D7F80936F008091BC068093DB
:10B18000BF068093BD068093BE0684E68093B90611
:10B1900028EE33E03093BB062093BA06992329F0BA
:10B1A00080916F00826080936F0081E080934E05F4
:10B1B00008950C94E838CF93C82F0E9411390E944B
:10B1C00068AD24E0C29FF0011124EF5AF94F2081AD
:10B1D0003181428153810E9404AFCF9108959091B3
:10B1E000BF068091BC06981719F00E944BABF7CFB1
:10B1F0008091BA069091BB06892BB9F70C9422AACC
:10B20000CF93C82F0E94CA380E9468AD24E0C29F25
:10B21000F0011124EF5AF94F20813181428153818D
:10B220000E9404AFCF9108959091BF068091BC0613
:10B23000981719F00E944BABF7CF8091BA06909106
:10B24000BB06892BB9F708952F923F924F925F92D8
:10B250006F927F928F929F92AF92BF92CF92DF9226
:10B26000EF92FF920F931F93CF93DF93CDB7DEB78B
:10B2700066970FB6F894DEBF0FBECDBFB88AAF8613
:10B28000E091CE05DC2CDE26672B682B692B19F4A8
:10B290008D2D8E7FD82E232B242B252B19F49D2D1D
:10B2A0009D7FD92EEF28E02AE12A19F4AD2DAB7F3E
:10B2B000DA2E8D2D8E278093CE058091650C90918E
:10B2C000660CA091670CB091680C8D839E83AF8350
:10B2D000B88720E030E0A901BC01CD010E94C6ACD6
:10B2E000882309F420C18091530290915402A091C7
:10B2F0005502B091560289879A87AB87BC87A9E629
:10B30000BCE0BE87AD87EF85F889FA83E98382ECDC
:10B3100095E09E8B8D8BA1E7B6E0BC83AB83212C9F
:10B32000312C812C912C5401EC2DF0E0FA8BE98B1F
:10B330008D2D90E09C8B8B8BAD85BE85CD90DD9067
:10B34000ED90FD90BE87AD8720E030E0A901C701F8
:10B35000B6010E94C6AC882309F4CEC009891A89B7
:10B36000022C02C0159507950A94E2F70170112787
:10B370008B899C89022C02C0959587950A94E2F7E7
:10B3800080FF38C0ED89FE8960817181828193815F
:10B390000E9468AD2B013C010115110529F420E044
:10B3A00030E040E85FE304C020E030E040E85FEBDD
:10B3B0006D817E818F8198850E9404AFA7019601DF
:10B3C0000E9404AFAB81BC8154962D913D914D916B
:10B3D0005C9157970E9404AF9B01AC01C301B2017D
:10B3E0000E94EDAB0E9435ADED89FE8960837183CB
:10B3F00082839383AD89BE89CD90DD90ED90FC90E2
:10B40000C114D104E104F10409F476C020E030E075
:10B41000A90169857A858B859C850E94C6AC8823A5
:10B4200009F441C0D701C6018827B7FD8395992744
:10B43000AA27BB270817190709F05EC020E030E0F3
:10B44000A901C501B4010E94C6AC81111CC02985A7
:10B450003A854B855C85EF85F88965857685878596
:10B4600090890E94CDAC4B015C0120E030E040E8C7
:10B470005FE30E94C9AE181634F4812C912C80E849
:10B48000A82E8FE3B82EC701B6010E9468ADA501B2
:10B4900094010E9404AF0E9435AD611571058105CC
:10B4A000910519F429C0C701B6018B019C0197FFD2
:10B4B00007C0002711279801061B170B280B390B13
:10B4C000A981BA8155964D905D906D907C9058976A
:10B4D000040D151D261D371DFD01058B168B278BB1
:10B4E000308FC61AD70AE80AF90AAD89BE89CD920B
:10B4F000DD92ED92FC921397BFEF2B1A3B0AE98184
:10B50000FA813496FA83E9838D899E8904969E8B0D
:10B510008D8BAB81BC811496BC83AB83B3E02B16BF
:10B52000310409F009CF66960FB6F894DEBF0FBE5E
:10B53000CDBFDF91CF911F910F91FF90EF90DF90E2
:10B54000CF90BF90AF909F908F907F906F905F90C3
:10B550004F903F902F9008952F923F924F925F927D
:10B560006F927F928F929F92AF92BF92CF92DF9213
:10B57000EF92FF920F931F93CF93DF93CDB7DEB778
:10B58000C756D1090FB6F894DEBF0FBECDBF1C0160
:10B59000A4966FAFA4976F965FAF4EAF6F97699603
:10B5A0003FAF2EAF69972896EFAE2897FFAE609613
:10B5B0000FAF609764961FAF6497CFAAA196BFAEF6
:10B5C000AEAEA197DA014D915D916D917C91809124
:10B5D000000690910106A0910206B09103068A012F
:10B5E0009B01081B190B2A0B3B0B0BA31CA32DA3C0
:10B5F0003EA36F96AEADBFAD6F9714964D915D9122
:10B600006D917C9117978091040690910506A09109
:10B610000606B09107068A019B01081B190B2A0B2D
:10B620003B0B0FA318A729A73AA76F96AEADBFADE6
:10B630006F9718964D915D916D917C911B978091BC
:10B64000080690910906A0910A06B0910B068A019E
:10B650009B01081B190B2A0B3B0B0FA718AB29AB3F
:10B660003AAB6F96AEADBFAD6F971C96CD90DD90A7
:10B67000ED90FC901F9780910C0690910D06A09183
:10B680000E06B0910F0626013701481A590A6A0AB8
:10B690007B0A09F497C06091D3047091D40480911F
:10B6A000D5049091D60420919C0421112AC00E94B7
:10B6B00035AD2091190230911A02621773070CF50B
:10B6C000C0920C06D0920D06E0920E06F0920F0684
:10B6D0006996EEADFFAD699784859585A685B7859A
:10B6E0008093DF059093E005A093E105B093E20518
:10B6F0000E94391681E195E10E942B16412C512CB4
:10B700003201C301B2010E9468AD1FA904E0109F7D
:10B71000F0011124E45BFD4F20813181428153818E
:10B720000E9404AF6B017C0120E030E0A9010E947F
:10B73000C9AE87FF04C0F7FAF094F7F8F09460916F
:10B7400091067091920680919306909194060E94C2
:10B7500035AD9B01AC01A8ECB0E00E944CB00E945A
:10B7600068AD9B01AC01C701B6010E94C9AE1816B5
:10B770004CF56F96EEADFFAD6F9784859585A685E8
:10B78000B78580930C0690930D06A0930E06B09398
:10B790000F066996EEADFFAD699784859585A68500
:10B7A000B7858093DF059093E005A093E105B09302
:10B7B000E2050E94391682EF94E10E942B16412C7B
:10B7C000512C32018BA19CA1ADA1BEA18827B7FD50
:10B7D00083959927AA27BB27182F2FA138A549A5FC
:10B7E0005AA557FD12608FA598A9A9A9BAA9B7FDB6
:10B7F000146077FC1860C301B2010E9468ADBFA954
:10B80000A4E0BA9FF0011124E45BFD4F2081318157
:10B81000428153810E9404AF4B015C0120E030E083
:10B82000A9010E94C9AE87FF04C0C501B4019058A8
:10B8300002C0C501B40120E030E040E05FE30E94B7
:10B84000EDAB0E943AAD6BAF7CAF8DAF9EAFF10117
:10B85000108215AB2BA13CA14DA15EA12BA73CA74B
:10B860004DA75EA757FF0BC0509540953095219589
:10B870003F4F4F4F5F4F2BA73CA74DA75EA78BA510
:10B880009CA5ADA5BEA5F101858B968BA78BB08F2E
:10B890002FA138A549A55AA52BAB3CAB4DAB5EAB50
:10B8A00057FF0BC050954095309521953F4F4F4F16
:10B8B0005F4F2BAB3CAB4DAB5EAB8BA99CA9ADA94D
:10B8C000BEA9F101818F928FA38FB48F2FA538A9C4
:10B8D00049A95AA92F962CAF3DAF4EAF5FAF2F9716
:10B8E00057FF0DC050954095309521953F4F4F4FD4
:10B8F0005F4F2F962CAF3DAF4EAF5FAF2F972F9678
:10B900008CAD9DADAEADBFAD2F97F101858F968FFC
:10B91000A78FB0A36BA17CA18DA19EA10E9468AD51
:10B920002091510630915206409153065091540691
:10B930000E9404AF27966CAF7DAF8EAF9FAF279765
:10B94000698B7A8B8B8B9C8B6FA178A589A59AA527
:10B950000E9468AD209155063091560640915706D9
:10B96000509158060E9404AF6B017C016D8B7E8B59
:10B970008F8B988F6FA578A989A99AA90E9468AD25
:10B980002091590630915A0640915B0650915C0611
:10B990000E9404AF6D966CAF7DAF8EAF9FAF6D9779
:10B9A000698F7A8F8B8F9C8F20915D0630915E0618
:10B9B00040915F0650916006C501B4010E9404AF3A
:10B9C0004B015C016D8F7E8F8F8F98A32BA53CA5BB
:10B9D0004DA55EA5263031054105510544F58BA9DD
:10B9E0009CA9ADA9BEA90697A105B10504F52F969E
:10B9F0002CAD3DAD4EAD5FAD2F97263031054105E5
:10BA00005105ACF420E030E0A901C501B4010E9469
:10BA1000C9AE87FF04C0B7FAB094B7F8B094D101AB
:10BA20001D968D929D92AD92BC92509759C0A19651
:10BA3000EEADFFADA19780809180A280B38020E021
:10BA400030E0A901C501B4010E94C6AC882341F0D1
:10BA5000D1011D968D929D92AD92BC92509731C0AE
:10BA600027962CAD3DAD4EAD5FAD2797CA01B9010C
:10BA70000E9404AF4B015C01A7019601C701B6010A
:10BA80000E9404AF9B01AC01C501B4010E94EDAB63
:10BA90004B015C016D962CAD3DAD4EAD5FAD6D972C
:10BAA000CA01B9010E9404AF9B01AC01C501B401F8
:10BAB0000E94EDAB0E9471AFF101658776878787A1
:10BAC000908B5101C12EEFA4F8A809A91AA92FA1A2
:10BAD00038A549A55AA56BA17CA18DA19EA1B4DB77
:10BAE0000BAD1CAD2DAD3EADD10191960D931D93C7
:10BAF0002D933C93949755964D915D916D917C91CA
:10BB000058975D960D911D912D913C919097599666
:10BB10008D919D910D90BC91A02D80179107A2074A
:10BB2000B30710F4D901C80184179507A607B70712
:10BB300010F4DB01CA010BAD1CAD2DAD3EAD80177D
:10BB40009107A207B30710F4D901C801F10185A339
:10BB500096A3A7A3B0A70697A105B105A8F1809168
:10BB6000CE04EF5AFF4F8083452B462B472B09F01D
:10BB70001798F101818D928DA38DB48D892B8A2B1D
:10BB80008B2B09F01698F101858D968DA78DB0A1AC
:10BB9000892B8A2B8B2B09F015980BAD1CAD2DAD85
:10BBA0003EAD012B022B032BD1F08091E7058823BA
:10BBB00019F081508093E7051FA9111107C014984F
:10BBC00080E28093E70502C080E0FEC7E090B10606
:10BBD000F090B2060091B3061091B40608C0E09050
:10BBE000B506F090B6060091B7061091B806970119
:10BBF000A80128966FAD28977FAD60968FAD6097AE
:10BC000064969FAD64970E94C6AC87FFD2C7D101EE
:10BC10001D962D913D914D915C9150976D962CAF55
:10BC20003DAF4EAF5FAF6D9760E070E080E89FE39F
:10BC30000E94CDAC2B966CAF7DAF8EAF9FAF2B9794
:10BC40009B01AC01B701C8010E9404AF4B015C012C
:10BC50008091BF069091BE06891B8F7024968FAF8E
:10BC60002497A501940160E074E284E799E40E94BE
:10BC7000CDAC0E94D4AE6B017C0124968FAD24978D
:10BC800082508630C0F58091810690918206A09105
:10BC90008306B0918406C816D906EA06FB0658F555
:10BCA0008C199D09AE09BF09BC01CD01660F771F34
:10BCB000881F991F2496BFAD24970B2F10E020E01A
:10BCC00030E0A90198010E94F1AFCA01B9010E94B8
:10BCD00066AD0E94D4AE6C0D7D1D8E1D9F1D0E9411
:10BCE00066AD9B01AC0160E074E284E799E40E94D8
:10BCF000CDAC4B015C01A50194016D966CAD7DADA1
:10BD00008EAD9FAD6D970E9404AF9B01AC010E9468
:10BD100004AF23966CAF7DAF8EAF9FAF2397F10139
:10BD2000618372838383948305A116A127A130A523
:10BD30000FA718AB29AB3AABC901B8010E9466AD99
:10BD40006FAB78AF89AF9AAFA50194010E9404AFA1
:10BD50000E94B3AC0E943AAD63966CAF7DAF8EAFDC
:10BD60009FAF6397F101EF5BFF4F60837183828325
:10BD700093838E010F5E1F4F1CA70BA70051110963
:10BD80002D961FAF0EAF2D9705E916E0A1961FAFB8
:10BD90000EAFA1978E010F5D1F4F1AA309A32D9619
:10BDA0000EAD1FAD2D971CAB0BAB1BA21FA200E865
:10BDB0001FE3ABA5BCA56D917D918D919D91BCA715
:10BDC000ABA7A50194010E9404AF6B017C01EBA914
:10BDD000FCA96193719381939193FCABEBAB20E051
:10BDE00030E0A9010E94C9AE87FF04C0F7FAF094C1
:10BDF000F7F8F094A196AEADBFADA1972D913D910E
:10BE00004D915D91A196BFAFAEAFA19767962CAF54
:10BE10003DAF4EAF5FAF6797C701B6010E94C9AE95
:10BE20001816C4F4A701960167966CAD7DAD8EAD72
:10BE30009FAD67970E94CDAC6B017C019B01AC016B
:10BE40006BA17FA1C8010E94C9AE18161CF4CBA239
:10BE5000DFA28701EBA5FCA529A13AA1E217F30710
:10BE600009F0A7CF20E030E040E85FE36BA17FA1BD
:10BE7000C8010E94C6AC87FF4BC06E0131E1C30E02
:10BE8000D11C2D96EEACFFAC2D972BA13FA1A801A4
:10BE9000D7016D917D918D919C910E9404AFF70126
:10BEA00061937193819391937F01EC15FD0569F77F
:10BEB0007101F1E4EF0EF11C63966CAD7DAD8EADBA
:10BEC0009FAD63970E9466AD2BA13FA1A8010E9480
:10BED00004AF0E943AADD7016D937D938D939C93EF
:10BEE00013972BA13FA1A8016BA17FA1C8010E94BC
:10BEF00004AF9B01AC0123966CAD7DAD8EAD9FADC3
:10BF000023970E9404AFF10161837283838394833A
:10BF10002B962CAD3DAD4EAD5FAD2B976FA978AD97
:10BF200089AD9AAD0E9404AF6BAB7CAB8DAB9EAB81
:10BF3000D10155960D911D912D913C9158970BA3D0
:10BF40001CA32DA33EA35D960D911D912D913C91B7
:10BF500090970FA318A729A73AA759960D911D915D
:10BF60002D913C915C970BA71CA72DA73EA70BA179
:10BF70001CA12DA13EA1012B022B032B41F52BA5CA
:10BF80003CA54DA55EA5232B242B252B01F58FA1C8
:10BF900098A5A9A5BAA5892B8A2B8B2BC1F4209132
:10BFA000A9063091AA064091AB065091AC066BA948
:10BFB0007CA98DA99EA90E9404AF0E94B3AC0E94E7
:10BFC0003AAD4B015C01D101D6961C92F0C20BAD8B
:10BFD0001CAD2DAD3EAD012B022B032B49F0609122
:10BFE000A5067091A6068091A7069091A80608C0A4
:10BFF0006091AD067091AE068091AF069091B0064B
:10C000002BA93CA94DA95EA90E9404AF0E94B3AC24
:10C010000E943AAD4B015C012BAD3CAD4DAD5EAD28
:10C02000232B242B252BA9F020E030E0A9016091DF
:10C03000E3057091E4058091E5059091E6050E9485
:10C04000C6AC882331F081E01414150416041704DB
:10C050000CF080E0D101D6968C93882309F4BAC005
:10C060002091D3053091D4054091D5055091D60546
:10C070006996EEADFFAD6997608171818281938190
:10C080000E94ECAB2B013C012091D7053091D805E3
:10C090004091D9055091DA056996AEADBFAD69976B
:10C0A00014966D917D918D919C9117970E94ECABA8
:10C0B0006BAF7CAF8DAF9EAF2091DB053091DC057F
:10C0C0004091DD055091DE056996EEADFFAD6997B3
:10C0D00060857185828593850E94ECAB6B017C0144
:10C0E000A3019201C301B2010E9404AF2B013C01E4
:10C0F0002BAD3CAD4DAD5EADCA01B9010E9404AFA0
:10C100009B01AC01C301B2010E94EDAB2B013C01CC
:10C11000A7019601C701B6010E9404AF9B01AC01C3
:10C12000C301B2010E94EDAB0E9471AF6B017C01B3
:10C130002091DF053091E0054091E1055091E20545
:10C140006996AEADBFAD69971C966D917D918D914D
:10C150009C911F970E94ECABA70196010E94CDAC69
:10C160006B017C01F101FD9660837183828393836F
:10C1700020E030E040E450E40E94C9AE18161CF400
:10C18000F10116AA27C02091E3053091E405409102
:10C19000E5055091E605C701B6010E9404AF9B0179
:10C1A000AC0160914D0670914E0680914F069091C2
:10C1B00050060E94CDAC2BA93CA94DA95EA90E94B6
:10C1C00004AF0E943AAD681579058A059B0510F405
:10C1D0004B015C018091FC059091FD05A091FE054D
:10C1E000B091FF05F10141A052A063A074A00FA57A
:10C1F00018A929A93AA980179107A207B30708F43B
:10C20000CDC02BA13CA14DA15EA1232B242B252B1E
:10C2100061F1209161063091620640916306509170
:10C220006406281539054A055B05F8F46FA578A959
:10C2300089A99AA90E94CEAF6B017C01A501940146
:10C240006BA17CA18DA19EA10E94CEAFC616D70680
:10C25000E806F90650F4C701B6012BA13CA14DA197
:10C260005EA10E94F1AF49015A018BA59CA5ADA525
:10C27000BEA5892B8A2B8B2B61F12091650630910D
:10C2800066064091670650916806281539054A05EB
:10C290005B05F8F46FA578A989A99AA90E94CEAF89
:10C2A0006B017C01A50194016BA57CA58DA59EA5C4
:10C2B0000E94CEAFC616D706E806F90650F4C701AD
:10C2C000B6012BA53CA54DA55EA50E94F1AF490185
:10C2D0005A010FA118A529A53AA5012B022B032B62
:10C2E00061F12091690630916A0640916B06509188
:10C2F0006C06281539054A055B05F8F46FA578A981
:10C3000089A99AA90E94CEAF6B017C01A501940175
:10C310006FA178A589A59AA50E94CEAFC616D706AB
:10C32000E806F90650F4C701B6012FA138A549A5C2
:10C330005AA50E94F1AF49015A0141145104610408
:10C34000710409F434C120916D0630916E0640915C
:10C350006F0650917006281539054A055B0508F0EF
:10C3600026C16FA578A989A99AA90E94CEAF6B01B1
:10C370007C01A5019401C301B2010E94CEAFC61693
:10C38000D706E806F90608F012C1C701B601A301F5
:10C3900092010E94F1AF49015A0109C12BA13CA1B0
:10C3A0004DA15EA1232B242B252BE9F16091610681
:10C3B0007091620680916306909164066815790514
:10C3C0008A059B0580F50E9466AD2FA938AD49AD61
:10C3D0005AAD0E9404AF6B017C016BA17CA18DA1C1
:10C3E0009EA10E9466AD6BA37CA38DA39EA3C501F5
:10C3F000B4010E9466AD2BA13CA14DA15EA10E949B
:10C4000004AFA70196010E94C9AE181664F42BA1CF
:10C410003CA14DA15EA1C701B6010E94CDAC0E9416
:10C420003AAD4B015C018BA59CA5ADA5BEA5892BA2
:10C430008A2B8B2BE9F160916506709166068091DD
:10C44000670690916806681579058A059B0580F551
:10C450000E9466AD2FA938AD49AD5AAD0E9404AF18
:10C460006B017C016BA57CA58DA59EA50E9466AD88
:10C470006BA37CA38DA39EA3C501B4010E9466ADEE
:10C480002BA13CA14DA15EA10E9404AFA701960182
:10C490000E94C9AE181664F42BA13CA14DA15EA167
:10C4A000C701B6010E94CDAC0E943AAD4B015C01C0
:10C4B0000FA118A529A53AA5012B022B032BE9F101
:10C4C0006091690670916A0680916B0690916C0686
:10C4D000681579058A059B0580F50E9466AD2FA930
:10C4E00038AD49AD5AAD0E9404AF6B017C016FA11C
:10C4F00078A589A59AA50E9466AD6BA37CA38DA3A0
:10C500009EA3C501B4010E9466AD2BA13CA14DA123
:10C510005EA10E9404AFA70196010E94C9AE181641
:10C5200064F42BA13CA14DA15EA1C701B6010E94FC
:10C53000CDAC0E943AAD4B015C0141145104610441
:10C540007104A9F160916D0670916E0680916F067D
:10C5500090917006681579058A059B0540F50E9443
:10C5600066AD2FA938AD49AD5AAD0E9404AF6B013D
:10C570007C01C301B2010E9466AD2B013C01C501E3
:10C58000B4010E9466ADA30192010E9404AFA7010D
:10C5900096010E94C9AE181654F4A3019201C70176
:10C5A000B6010E94CDAC0E943AAD4B015C01F10195
:10C5B000E35BFF4F80829182A282B382C501B40106
:10C5C0000E9466AD6B017C012BA93CA94DA95EA917
:10C5D0000E94CDAC2B966CAF7DAF8EAF9FAF2B97EB
:10C5E000D10151966D937D938D939C9354972DEB30
:10C5F00037E346E051E4C701B6010E9404AF0E9450
:10C600003AADF10161AB72AB83AB94AB86A98823E1
:10C6100081F1FD9620813181428153816091E30552
:10C620007091E4058091E5059091E6050E9404AFC4
:10C630002B962CAD3DAD4EAD5FAD2B970E9404AF58
:10C640002091910630919206409193065091940664
:10C650000E9404AF9B01AC0160E074E284EF99E4B6
:10C660000E94CDAC0E943AADD101D8967C936E93D6
:10C67000D797D10111960D911D912D913C91149751
:10C6800063960CAF1DAF2EAF3FAF6397C901B801E2
:10C690000E9471AF6FA77BAF8FAB9BA701E416E041
:10C6A00065961FAF0EAF65973E0111E1610E711CDB
:10C6B00001E416E021961FAF0EAF21972D964EACE8
:10C6C0005FAC2D976BA37FA3182F092F1BAAD20154
:10C6D000CD90DD90ED90FD902D0120E030E0A9019E
:10C6E000C701B6010E94C9AE87FF04C0F7FAF094F3
:10C6F000F7F8F0942196EEADFFAD219781909190DF
:10C70000A190B1902196FFAFEEAF2197A5019401C2
:10C71000C701B6010E94C9AE18160CF03FC0FBA9B4
:10C72000FF2329F1A50194016FA57BAD8FA99BA5DE
:10C730000E9404AF4B015C012BA13FA1412F502F60
:10C74000C701B6010E9404AFA50194010E94C9AEC1
:10C75000181614F5A7019601C501B4010E94CDACCD
:10C760006BA37FA3182F092F21E02BAB17C0A701C4
:10C770009601C501B4010E94CDAC9B01AC016BA137
:10C780007FA1812F902F0E9404AF6BA37FA3182F4E
:10C79000092F31E03BAB02C041E04BAB46145704DC
:10C7A00009F095CF5BA1A5965FAFA5978FA1A6963F
:10C7B0008FAFA697A7961FAFA797A8960FAFA8977A
:10C7C00024969FAD2497992309F44CC1C090E805A5
:10C7D000D090E905E090EA05F090EB052DEB37E30A
:10C7E00046E855E3C701B6010E94C6AC87FD3AC1D1
:10C7F000C701B6010E9471AF6B017C019B01AC01C6
:10C800006FA57BAD8FA99BA50E94C6AC87FD04C018
:10C81000CFA6DBAEEFAAFBA69601A7016FA57BAD65
:10C820008FA99BA50E94CDACA3966CAF7DAF8EAFB8
:10C830009FAFA397ACEEB5E02196BFAFAEAF219707
:10C8400020E030E040E85FE32BAB3CAB4DAB5EABB0
:10C8500024961FAE24972196AEADBFAD21976D9162
:10C860007D918D919D912196BFAFAEAF2197A396FB
:10C870002CAD3DAD4EAD5FADA3970E9404AF6B01F3
:10C880007C012D96EEADFFAD2D9781909190A190FA
:10C89000B1902D96FFAFEEAF2D972496FFAD249764
:10C8A000FF2391F02BA93CA94DA95EA90E9404AFDA
:10C8B0006B017C012BA93CA94DA95EA9C501B4015E
:10C8C0000E9404AF4B015C01A5019401C701B601B0
:10C8D0000E94C9AE20E030E0A90118164CF5C50150
:10C8E000B4010E94C9AE18164CF020E030E0A90156
:10C8F000C701B6010E94C6AC87FF09C0A50194011B
:10C90000C701B6010E94ECAB2B013C0139C02401E8
:10C91000350177FA709477F87094A3019201C701FA
:10C92000B6010E94C9AE18165CF52601370128C071
:10C93000C501B4010E94C6AC87FD09C020E030E00B
:10C94000A901C701B6010E94C9AE18164CF4A7018F
:10C950009601C501B4010E94ECAB2B013C0110C053
:10C960002601370177FA709477F87094A501940145
:10C97000C301B2010E94C9AE181614F0240135019A
:10C980006596AEADBFAD6597CD90DD90ED90FD9015
:10C990006596BFAFAEAF6597A7019601C301B2011F
:10C9A0000E94C9AE1816CCF4A3019201C701B601CA
:10C9B0000E94CDAC9B01AC016BA97CA98DA99EA95D
:10C9C0000E9404AF6BAB7CAB8DAB9EAB2496BFAD2E
:10C9D0002497BF5F2496BFAF24972196EEADFFAD9D
:10C9E0002197EC5FF54009F036CF24963FAD2497B0
:10C9F000332371F02BA93CA94DA95EA96FA57BAD8E
:10CA00008FA99BA50E9404AF6FA77BAF8FAB9BA79D
:10CA100024EA30E74DE75FE36FA57BAD8FA99BA5C7
:10CA20000E9404AF6B017C019B01AC016091BE05CB
:10CA30007091BF058091C0059091C1050E94C9AE5B
:10CA4000181654F4A70196016BA17FA1812F902F96
:10CA50000E94C9AE181634F00FA50BA31BAD1FA37F
:10CA60001FA90BA5A5968FADA597A6969FADA697D6
:10CA7000A796AFADA797A896BFADA8978093BE0520
:10CA80009093BF05A093C005B093C1052BA13FA112
:10CA9000412F502F6BA17FA1812F902F0E9404AFB7
:10CAA0007B018C01CB01D801F10181879287A3879B
:10CAB000B4872B966CAD7DAD8EAD9FAD2B97905806
:10CAC0009B01AC010E94EDAB6D962CAD3DAD4EAD22
:10CAD0005FAD6D970E9404AF9B01AC016BE077EDF9
:10CAE00083E29BE30E94ECAB5B016C01A496FFAD7B
:10CAF000A497FF2361F09B01AC01B701C8010E941C
:10CB0000C6AC87FD09C09A2D8B2D860107C09BE01E
:10CB100087ED03E21BE302C09E2D8F2D492F582F76
:10CB2000B801D10115964D935D936D937C93189741
:10CB30001C919501A60163966CAD7DAD8EAD9FAD48
:10CB400063970E94C6AC181614F481E001C083E01C
:10CB5000182BF101108380E1FE013196ACEEB5E0B7
:10CB600001900D928A95E1F7F10181819281A38173
:10CB7000B4818093E8059093E905A093EA05B0930A
:10CB8000EB0580E16F96EEADFFAD6F97A0E0B6E0EC
:10CB900001900D928A95E1F780E16996EEADFFADC7
:10CBA0006997A3EDB5E001900D928A95E1F781E0D8
:10CBB0000BC02896EFAC2897FFAC60960FAD60973E
:10CBC00064961FAD649723C8C959DF4F0FB6F89418
:10CBD000DEBF0FBECDBFDF91CF911F910F91FF90B0
:10CBE000EF90DF90CF90BF90AF909F908F907F900D
:10CBF0006F905F904F903F902F9008956F927F922B
:10CC00008F929F92AF92BF92CF92DF92EF92FF925C
:10CC10000F931F93CF93DF9300D01F92CDB7DEB752
:10CC20004C013B018091BA069091BB06892BD9F546
:10CC30009091BF068091BC06981B9F709F3059F45D
:10CC400029833A834B835C830E944BAB5C814B818D
:10CC50003A812981EDCFD090BF068091BF0666E56D
:10CC6000869FC00111245701C02E79018A019301CA
:10CC7000A40160E08054994F0E94AC5A8823A9F027
:10CC80002091BF069091BC06291303C094E69093AF
:10CC9000B90691E09D0D9F709093BF0689830E9415
:10CCA0004D57898103C080E001C081E00F900F9053
:10CCB0000F900F90DF91CF911F910F91FF90EF9008
:10CCC000DF90CF90BF90AF909F908F907F906F90AC
:10CCD00008958091BF069091BC06891B8F708F309C
:10CCE00019F40E944BABF5CF8091BF068F5F8F7018
:10CCF000E091BF0696E59E9FF0011124E054F94FA4
:10CD0000DF011D929A95E9F798E090834091000623
:10CD1000509101066091020670910306458B568B77
:10CD2000678B708F4091040650910506609106064E
:10CD300070910706418F528F638F748F4091080660
:10CD40005091090660910A0670910B06458F568F27
:10CD5000678F70A340910C0650910D0660910E06EE
:10CD600070910F0641A352A363A374A32091BF0641
:10CD70009091BC06291303C094E69093B906809362
:10CD8000BF060C949D2F2F923F924F925F926F920D
:10CD90007F928F929F92AF92BF92CF92DF92EF924B
:10CDA000FF920F931F93CF93DF93CDB7DEB7A99771
:10CDB0000FB6F894DEBF0FBECDBFF801A091BA0642
:10CDC000B091BB06AB2B09F0A7C016010E2DF8A73A
:10CDD000EFA33EA32DA36A017B01FC01408051809B
:10CDE0006280738020918506309186064091870687
:10CDF00050918806C301B2010E9404AF0E94D4AED4
:10CE0000698B7A8B8B8B9C8BD7018D909D90AD908D
:10CE1000BC902091890630918A0640918B065091F2
:10CE20008C06C501B4010E9404AF0E94D4AE6D8B84
:10CE30007E8B8F8B988FD6012D913D914D915C917A
:10CE400029A33AA34BA35CA320918D0630918E06B3
:10CE500040918F065091900669A17AA18BA19CA167
:10CE60000E9404AF0E94D4AE698F7A8F8B8F9C8F03
:10CE7000EDA1FEA1C080D180E280F38020919106D7
:10CE8000309192064091930650919406C701B601E5
:10CE90000E9404AF0E94D4AE6D8F7E8F8F8F98A3B7
:10CEA00049825A826B827C828D829E82AF82B88652
:10CEB00029A13AA14BA15CA129873A874B875C87BE
:10CEC000CD86DE86EF86F88A2091930323FF10C07B
:10CED00060930C0670930D0680930E0690930F06D8
:10CEE000C092DF05D092E005E092E105F092E20504
:10CEF000AFA1B8A52D913D914D915C917101BE01FD
:10CF00006F5F7F4FCE01419679DE882331F089A78C
:10CF10000E949D2F89A501C080E0A9960FB6F894C4
:10CF2000DEBF0FBECDBFDF91CF911F910F91FF905C
:10CF3000EF90DF90CF90BF90AF909F908F907F90B9
:10CF40006F905F904F903F902F900895AF92BF9257
:10CF5000CF92DF92EF920F931F93CF93DF93CDB7D2
:10CF6000DEB764970FB6F894DEBF0FBECDBFA98AB7
:10CF7000BA8ACB8ADC8AFC0180819181A281B3814B
:10CF800089839A83AB83BC83FB0180819181A281D9
:10CF9000B3818D839E83AF83B887FA0180819181AD
:10CFA000A281B38189879A87AB87BC87F901808189
:10CFB0009181A281B3818D879E87AF87B88BAE01A7
:10CFC000475F5F4FBE016B5F7F4FCE0101960E94AE
:10CFD000D757CE0141966C019E01235F3F4FAE01B2
:10CFE000475F5F4FBE016B5F7F4F4097CCDE64961B
:10CFF0000FB6F894DEBF0FBECDBFDF91CF911F916A
:10D000000F91EF90DF90CF90BF90AF9008958F92E7
:10D010009F92AF92BF92EF92FF920F931F93CF9385
:10D02000DF937B018A01E901FC0180809180A2806D
:10D03000B3802091850630918606409187065091F5
:10D040008806C501B4010E9404AF0E94D4AE60936B
:10D0500000067093010680930206909303062091C8
:10D06000890630918A0640918B0650918C06F70113
:10D0700060817181828193810E9404AF0E94D4AE4D
:10D080006093040670930506809306069093070646
:10D0900020918D0630918E0640918F06509190061A
:10D0A000F80160817181828193810E9404AF0E94A6
:10D0B000D4AE609308067093090680930A06909395
:10D0C0000B06209191063091920640919306509163
:10D0D0009406688179818A819B810E9404AF0E94B5
:10D0E000D4AE60930C0670930D0680930E06909359
:10D0F0000F068092D3059092D405A092D505B092E8
:10D10000D605F70180819181A281B3818093D705F3
:10D110009093D805A093D905B093DA05F8018081E2
:10D120009181A281B3818093DB059093DC05A0936C
:10D13000DD05B093DE0588819981AA81BB8180934A
:10D14000DF059093E005A093E105B093E20590918F
:10D15000BF068091BC06981759F0DF91CF911F91BF
:10D160000F91FF90EF90BF90AF909F908F90B1CDB7
:10D170000E94145980916F0081FBCC27C0F981FF78
:10D1800005C080916F008D7F80936F002CE036E0AA
:10D1900048E056E064E076E080E096E00E94CD3220
:10D1A000CC2329F080916F00826080936F00DF9123
:10D1B000CF911F910F91FF90EF90BF90AF909F90F4
:10D1C0008F900895CF93DF93CDB7DEB760970FB6FA
:10D1D000F894DEBF0FBECDBFFC0180819181A2819A
:10D1E000B38189839A83AB83BC83FB018081918166
:10D1F000A281B3818D839E83AF83B887FA0180813A
:10D200009181A281B38189879A87AB87BC87F90115
:10D2100080819181A281B3818D879E87AF87B88BF2
:10D22000AE01475F5F4FBE016B5F7F4FCE0101963E
:10D230000E94D7579E01235F3F4FAE01475F5F4F6C
:10D24000BE016B5F7F4FCE010196E1DE60960FB6A7
:10D25000F894DEBF0FBECDBFDF91CF910895CF927E
:10D26000DF92EF92FF92FC01C080D180E280F380D8
:10D270002091910630919206409193065091940628
:10D28000C701B6010E9404AF0E94D4AE60930C06A1
:10D2900070930D0680930E0690930F06C092DF05E3
:10D2A000D092E005E092E105F092E2059091BF0690
:10D2B0008091BC06981729F0FF90EF90DF90CF90F7
:10D2C00008CD0E94145980916F0081FB992790F935
:10D2D00081FF05C080916F008D7F80936F0040912A
:10D2E0000C0650910D0660910E0670910F0640934A
:10D2F000F1045093F2046093F3047093F4049923BF
:10D3000029F080916F00826080936F00FF90EF9012
:10D31000DF90CF900895CF92DF92EF92FF920F931C
:10D320001F93CF93DF93C1E7D6E001E616E0C12C4F
:10D33000D12C7601C39469917991899199910E9438
:10D3400066AD288939894A895B890E9404AF0E94A9
:10D350003AADF80161937193819391938F01C61651
:10D36000D706E806F90610F46B017C01F6E0C13837
:10D37000DF0709F76FEF7FEFCB01A70196010E944E
:10D38000F1AF2093FC053093FD054093FE055093CB
:10D39000FF05DF91CF911F910F91FF90EF90DF90EC
:10D3A000CF9008950F931F93CF93DF9305E816E076
:10D3B000C1E5D6E0F80121913191419151918F0160
:10D3C00060E070E080E89FE30E94CDAC69937993C0
:10D3D00089939993F6E0C136DF0761F727EB35E0D3
:10D3E00043EB55E06FEA75E08BEA95E0EBDEDF9109
:10D3F000CF911F910F918FCF80E29CE00C945152FE
:10D4000081548A3108F041C0A82FB0E04091490C06
:10D4100050914A0C60914B0C70914C0C04C0769565
:10D420006795579547958A95D2F740FF2EC0E091B2
:10D43000540CF091550CA15DB34F8C918823E9F009
:10D44000E80FF11D808190ED980F9A3098F08E32A0
:10D4500011F481810CC08D3211F08B3271F4818115
:10D4600090ED980F9A3030F08E3239F482818053EB
:10D470008A3018F49E2F8F2F02C090E080E09093A6
:10D48000500C8093510C81E0089580E00895B8DF3E
:10D49000882341F081E02091500C3091510C232BD6
:10D4A00009F480E008950F931F93CF938091500C5F
:10D4B0009091510C009711F1FC018F01C1912C2F1B
:10D4C0002F7DA9F0C53411F0C536B9F7F8011082E7
:10D4D00060E070E08091500C9091510C0E9456B029
:10D4E000F801C083562F472F382F292F0BC060E03B
:10D4F00070E0CF911F910F910C9456B050E040E036
:10D5000030E020E0652F742F832F922FCF911F9151
:10D510000F9108958091500C9091510C009731F02B
:10D520004AE050E060E070E00C94BCB160E070E074
:10D53000CB010895CF9384E5AADF882359F1EADF70
:10D5400097FD24C0E7DF6F3F71058105910509F064
:10D55000FCF4E0DFC62F1616FCF40E9439168DE4A9
:10D560000E94BB186AE070E080914D0C90914E0CC7
:10D570000E94AE196C2FCC0F770B84E895E10E94C6
:10D580005C168AE00E94BB188FEF07C0C0E004C0A1
:10D59000CFEF02C080E001C08C2FCF910895AF92F1
:10D5A000BF92CF92DF92EF92FF920F931F93CF9390
:10D5B000DF9389E2A82E83E0B82E9BE9E92E95E05F
:10D5C000F92E0BEA15E02BE6C22E25E0D22EC0E0A4
:10D5D000D0E0F50181915F0113DF882319F163DF4A
:10D5E000FE01EA5DF34F2081211104C02091BB05AB
:10D5F000222341F0F80120813181428153810E9430
:10D60000EDAB0AC0C330D10539F0F601208131817C
:10D61000428153810E94ECABF70160837183828366
:10D6200093830AC0F80180819181A281B381F701BF
:10D6300080839183A283B3832196F4E0EF0EF11CE3
:10D640000C5F1F4F84E0C80ED11CC430D10509F017
:10D65000C0CF86E41CDF8823B9F025DF20E030E06E
:10D66000A9010E94C9AE18167CF41DDF20E030E04D
:10D6700040E752E40E94CDAC6093480270934902A7
:10D6800080934A0290934B02DF91CF911F910F91AB
:10D69000FF90EF90DF90CF90BF90AF900895CF9222
:10D6A000DF92EF92FF926B017C010E94A611C60EE1
:10D6B000D71EE81EF91E0E94A611DC01CB018C19B1
:10D6C0009D09AE09BF09B7FF03C00E944BABF3CF62
:10D6D000FF90EF90DF90CF9008956F927F928F929E
:10D6E0009F92AF92BF92CF92DF92EF92FF920F93F1
:10D6F0001F93CF93DF93CDB7DEB73C01A090540CBE
:10D70000B090550CCDB6DEB66AE070E0C3010E9461
:10D7100029B47C01009721F08C010619170904C077
:10D72000C3010E9434B48C01C80101962DB73EB7E5
:10D73000281B390B0FB6F8943EBF0FBE2DBF8DB717
:10D740009EB701964C01A801B3010E9455B4F401A3
:10D75000E00FF11F1082C40157D581E034D0E114ED
:10D76000F10451F037019FEF691A790A0FB6F89466
:10D77000DEBE0FBECDBEC6CF0FB6F894DEBE0FBE66
:10D78000CDBEC501DF91CF911F910F91FF90EF901A
:10D79000DF90CF90BF90AF909F908F907F906F90D1
:10D7A00033C5CF93C3E00E94C287882341F0C150A4
:10D7B00019F00E9435AAF7CFCF910C9462AA8DE69A
:10D7C00095E1CF918ACFCF93C82F41E04093250CAC
:10D7D00090914F0C9D3409F459C0943509F406C258
:10D7E000973409F007C220914D0C30914E0C2B312B
:10D7F0003105D1F1ACF42430310544F42230310547
:10D8000044F537FDF7C10E949097F7C124303105E8
:10D8100041F12C30310509F0EDC10E94AA92EDC111
:10D820002A35310551F154F42D31310521F1FCF047
:10D830002E31310509F0DEC165D2DFC12C3531054D
:10D8400011F1F4F0293A314009F0D4C10E947885F1
:10D85000D4C181E02230310509F080E00E94C19BF3
:10D86000CCC10E949997C9C10E94AE92C6C180E006
:10D870000E94767BC2C195DFC0C11092BB05BDC1BD
:10D880004093BB05BAC10E948479B7C120914D0C69
:10D8900030914E0C2C38310509F44AC10CF08BC084
:10D8A0002836310509F439C10CF044C02C34310557
:10D8B00009F430C104F52231310509F44DC164F495
:10D8C00037FD98C1223031050CF41CC121313105DE
:10D8D00009F090C1B6D791C12A32310509F414C1BB
:10D8E0002B34310509F413C12F31310509F082C100
:10D8F0000E94347782C12335310509F42AC16CF4C2
:10D900002135310509F420C10CF020C12D34310539
:10D9100009F070C10E94727670C12535310509F495
:10D920001DC10CF419C12C35310509F063C10E94E9
:10D93000379463C12037310509F45FC1CCF42C362C
:10D94000310509F45AC15CF42A36310509F4F6C0F0
:10D950000CF0F7C00E9404A21092250C55C12E367F
:10D96000310509F4DDC00CF0DEC00E9491A145C173
:10D970002537310509F4F7C06CF42237310509F475
:10D98000EFC00CF4D2C02337310509F033C10E9437
:10D99000ED7733C12737310509F4EAC00CF4E5C04F
:10D9A0002837310509F4E7C02937310509F022C1CC
:10D9B0000E94437522C12F3581E0380709F414C154
:10D9C0000CF04DC0233D310509F4E3C00CF52B3CB0
:10D9D000310509F4D5C07CF42E3B310509F4ABC008
:10D9E000293C310509F4C9C02B39310509F002C1C0
:10D9F0000E9427A102C12D3C310509F4C7C00CF4D7
:10DA0000C2C02E3C310509F0F5C00E945378F5C024
:10DA10002D3281E0380709F4C3C07CF42D3D310577
:10DA200009F4B9C0223E310509F4B8C02C3D3105D6
:10DA300009F0E0C00E94E693E0C02F3281E0380791
:10DA400009F4B7C00CF4B2C0203381E0380709F400
:10DA5000AAC02E35314009F0CDC09DD5CEC0243F9F
:10DA600081E0380709F4B2C03CF52A3981E0380773
:10DA700009F4C3C084F4213981E0380709F49CC05B
:10DA8000223981E0380709F499C02039314009F082
:10DA9000B1C0FCD7B2C0293A81E0380709F490C080
:10DAA0002C3A81E0380709F48EC0243A314009F05D
:10DAB000A1C00E94A886A1C0283F81E0380709F4D0
:10DAC0008BC04CF4263F81E0380709F481C00CF08C
:10DAD00081C017D592C0243883E0380709F47EC08E
:10DAE00034F42335334009F085C045D286C02B3845
:10DAF00083E0380709F475C0273E334009F07AC047
:10DB000099D77BC0B1D279C00E940F7676C00E94AF
:10DB10006E7673C00E94707670C00E946EA16DC058
:10DB20000E9439786AC013D768C00E945F7765C0C9
:10DB30000E94E8A062C00E9401A15FC00E94E7A10C
:10DB40005CC00E94FDA159C067D757C00E94899749
:10DB500054C00E948C9751C076D64FC021D64DC07C
:10DB60000E949D774AC07FD248C00E94A17745C0DD
:10DB70000E94957742C084D740C00E94A2953DC0C4
:10DB80000E94D1953AC00E94F69537C00E946C96CB
:10DB900034C07ED732C00E9419932FC0C5D52DC086
:10DBA0000E94F2962AC00E94749327C00E940B958F
:10DBB00024C00E9433A021C09BD01FC09ED01DC096
:10DBC0000E94317A1AC00E949A7817C098D415C062
:10DBD0009AD413C09AD411C0BFD40FC00E94299206
:10DBE0000CC00E94FA9209C00BD507C080914D0C61
:10DBF00022D603C08EE29CE072D41092250CC11193
:10DC000003C0CF910C944D9ECF910895CF93DF9395
:10DC1000C091F00E80E6C89FE0011124C15FD24F91
:10DC20008091930380FF05C00E943916CE010E94A7
:10DC30001219CE01E9D280E0DF91CF91C4CDCF920D
:10DC4000DF92EF92FF920F931F930E94A6116B0138
:10DC50007C018091100F81112FC080915202882386
:10DC600059F18091250C882339F14091210C509174
:10DC7000220C6091230C7091240C97018601041BE7
:10DC8000150B260B370B37FD2CC0833079F03CF495
:10DC9000813094F00E9439168BE595E10BC08430F9
:10DCA00059F40E9439168CE295E104C00E9439169D
:10DCB00084E495E10E942B162091520230E0A8EEF8
:10DCC000B3E00E9437B0DC01CB018C0D9D1DAE1D71
:10DCD000BF1D8093210C9093220CA093230CB09332
:10DCE000240C1F910F91FF90EF90DF90CF9008953B
:10DCF00081E00E940F490C94674C80E00E940F491C
:10DD00000C94674C8F929F92AF92BF92CF92DF920A
:10DD1000EF92FF920F931F93CF93DF93CDB7DEB7B0
:10DD200028970FB6F894DEBF0FBECDBFC090AB05ED
:10DD3000D090AC05E090AD05F090AE0588E5A7DB8E
:10DD4000811108C020E030E0A901C701B6010E949E
:10DD5000EDAB01C0A8DB6D837E838F839887C09075
:10DD6000AF05D090B005E090B105F090B20589E51F
:10DD70008EDB811108C020E030E0A901C701B601A7
:10DD80000E94EDAB01C08FDB6B017C0169837A835C
:10DD90008B839C838D809E80AF80B88422ED30E0A1
:10DDA00040EE50EC0E94C9AE87FDD2C027E030E0C3
:10DDB0004EE353E4C701B6010E94C6AC18160CF43A
:10DDC000C7C023EA31E040E450ECC501B4010E9431
:10DDD000C9AE87FDBDC027E030E042E253E4C50193
:10DDE000B4010E94C6AC18160CF4B2C027E030E0B3
:10DDF00041E253E4C501B4010E94C6AC18160CF40C
:10DE0000A7C027E030E041E253E4C701B6010E9419
:10DE1000C6AC18160CF49CC080E00E94AF1A0E9499
:10DE2000EB4E85E434DB182F8823B1F08091500C41
:10DE30009091510C892B09F489C06CDB97FD0FC0C0
:10DE400069DB6F3F71058105910509F04CF462DBD8
:10DE500061117CC040E005C085E4D2DA77C010E0F3
:10DE6000412F01E021E0BE016F5F7F4FCE0105969B
:10DE70000E94B0496B017C019B01AC010E94B2AFD2
:10DE800081115FC08D809E80AF80B88420E030E03B
:10DE9000A901C501B4010E94C6AC87FD05C027E1F8
:10DEA00037EB41E558E304C027E137EB41E558EB98
:10DEB000C501B4010E94EDABAB01BC0181EA95E163
:10DEC0000E94761689809A80AB80BC8020E030E08A
:10DED000A901C501B4010E94C6AC87FD05C027E1B8
:10DEE00037EB41E558E304C027E137EB41E558EB58
:10DEF000C501B4010E94EDABAB01BC018CE995E119
:10DF00000E94761620E030E0A901C701B6010E9408
:10DF1000C6AC87FD05C027E137EB41E558E304C0F7
:10DF200027E137EB41E558EBC701B6010E94EDABA5
:10DF3000AB01BC0187E995E10E9476168AE00E9458
:10DF4000BB180E940A4F0E94674C02C041E089CF73
:10DF500028960FB6F894DEBF0FBECDBFDF91CF91EC
:10DF60001F910F91FF90EF90DF90CF90BF90AF90F7
:10DF70009F908F900895EF92FF920F931F93CF93EE
:10DF8000DF938AE53DDA882309F456C08091500C6E
:10DF90009091510C009709F44FC0FC017F01C19191
:10DFA0002C2F2F7D89F0C53411F0C536B9F7F70154
:10DFB000108260E070E08091500C9091510C0E94B2
:10DFC00056B0F701C08304C060E070E00E9456B014
:10DFD0008B01D82FC92F20E030E040E050EC0E94A8
:10DFE000C9AE87FD1DC020E030E040EA50E4B80132
:10DFF0008D2F9C2F0E94C6AC181694F0C801AD2F2F
:10E00000BC2F8093610590936205A0936305B09344
:10E010006405DF91CF911F910F91FF90EF900895CC
:10E020000E943C168AEB95E1DF91CF911F910F91F1
:10E03000FF90EF900C942B160E94391640916105C9
:10E0400050916205609163057091640589EA95E1DC
:10E050000E9476168AE0DF91CF911F910F91FF9079
:10E06000EF900C94BB180895CF92DF92EF92FF923D
:10E070000F931F93CF93DF93C091520CD091530C09
:10E0800080E505DA8823D1F08091500C9091510CF5
:10E09000009749F04AE050E060E070E00E94E4B28E
:10E0A0006B017C0103C0C12CD12C760111E0C1149D
:10E0B000D104E104F10431F410E004C010E0C12CFB
:10E0C000D12C760183E5E3D9882309F486C08091B9
:10E0D000500C9091510C009701F1FC017F010191CE
:10E0E000202F2F7D89F0053411F00536B9F7F7019F
:10E0F000108260E070E08091500C9091510C0E9471
:10E1000056B0F701008304C060E070E00E9456B092
:10E11000B62FA72FF82FE92F04C0B0E0A0E0F0E061
:10E12000E0E020E030E04AE754E46B2F7A2F8F2FB5
:10E130009E2F0E9404AF0E943AAD6B017C01111129
:10E1400009C0672B682B692B29F4209719F0888167
:10E15000811102C010E001C011E00E941459112386
:10E1600029F00E943916CE010E94121983E0809393
:10E17000250C81E08093110FC114D104E104F10456
:10E1800029F10E94A611C60ED71EE81EF91E0E9494
:10E19000A611DC01CB018C199D09AE09BF09B7FDA1
:10E1A0000EC01092110F81E08093250CDF91CF916A
:10E1B0001F910F91FF90EF90DF90CF900895809185
:10E1C000110F882371F30E944BABE1CF8091110FA7
:10E1D000882339F30E944BABF9CF1111BBCFB5CFD8
:10E1E0001092530C1092520C8FE380934F0C1092AC
:10E1F0004E0C10924D0C1092490C10924A0C109239
:10E200004B0C10924C0C08953F924F925F926F927C
:10E210007F928F929F92AF92BF92CF92DF92EF92B6
:10E22000FF920F931F93CF93DF931F921F92CDB74F
:10E23000DEB789839A83D4DF8981282F9A81392F89
:10E24000F90180812F5F3F4F8032D1F38E34B1F4DA
:10E25000818190ED980F9A3020F08D3211F08B3241
:10E2600069F43296DF0131962C9120532A30D0F395
:10E27000CD01FC01019620812032D9F3F093550C99
:10E28000E093540C8F010F5F1F4F30806AE270E003
:10E29000C8010E948BB4009731F0FC013197808156
:10E2A0008032E1F311828DE4381631F0E4E53E1658
:10E2B00019F0F7E43F12FFC0F80180810F5F1F4F94
:10E2C0008032D1F380538A3008F0F5C030924F0C81
:10E2D00010924E0C10924D0C4AE020914D0C309152
:10E2E0004E0C429FC001439F900D112490934E0C01
:10E2F00080934D0C3196DF0111972C91022E000C6A
:10E30000330B20533109280F391F30934E0C2093C3
:10E310004D0C808180538A3000F3DF0131968C915F
:10E320008032D9F38DE438121AC02E31310591F0C4
:10E330003CF42731310571F02C31310581F40AC0EC
:10E340002537310564F02737310524F0203AE3E022
:10E350003E0729F4B093530CA093520CACC010921A
:10E36000530C1092520C5091540CC12CD12C7601AC
:10E37000C394FD0131964C91442309F49CC0413271
:10E38000A9F48DE4381212C02032310579F4F093EB
:10E39000530CE093520C63E270E0CF010E948BB407
:10E3A000009709F488C0FC01108285C041544A31AD
:10E3B00008F055C0BF01FB0180816F5F7F4F803245
:10E3C000D1F390ED980F9A3008F18E3211F48181DB
:10E3D0000CC08D3211F08B3259F4818190ED980F81
:10E3E0009A30A0F08E3221F4828180538A3070F00E
:10E3F0008091520C9091530C892B09F059C0CF0198
:10E4000001979093530C8093520C52C0CF01A42FCC
:10E41000B0E04601570104C0880C991CAA1CBB1C23
:10E420004A95D2F74090490C50904A0C60904B0CA2
:10E4300070904C0C84289528A628B7288092490C07
:10E4400090924A0CA0924B0CB0924C0C009711F099
:10E45000851B01C080E0A15DB34F8C930AC0809101
:10E46000520C9091530C892B21F4B093530CA09330
:10E47000520C808181548A3130F4DF017ACF80EDF3
:10E48000890F8A3040F44E2F6F2F91919111F7CF61
:10E49000842F962F07C083ED890F8230A0F39B3223
:10E4A00091F3F6CFFC01019640814032D9F3E5CFDC
:10E4B00080E090E0ACCF0F900F90DF91CF911F9153
:10E4C0000F91FF90EF90DF90CF90BF90AF909F9013
:10E4D0008F907F906F905F904F903F9008950E9433
:10E4E00039166091540C7091550C85ED95E10E94A0
:10E4F0003F1682E20E94BB188AE00C94BB180C9471
:10E50000D93B0C9408490C94623FCF9383E50E9459
:10E51000006AC82F8823D1F08091500C9091510C43
:10E52000892BC1F00E948A6A97FD0DC00E948A6AF9
:10E530006F3F71058105910509F034F40E948A6AE4
:10E54000611108C003C0C0E081E0C8278C2FCF91C3
:10E550000C94AC40C0E0FACF0E940149882331F00E
:10E560000E94391688EE95E10C942B1608950E94AE
:10E570008A6A97FD0CC00E948A6A6F3F7105810507
:10E58000910509F034F40E948A6A862F089580E08C
:10E5900008958FEF08950F931F93CF9383E50E9403
:10E5A000006A811104C00DE213E0C0E00DC0C0E0BC
:10E5B000DEDF682F8C2F0E94503ACF5FC530C1F745
:10E5C000F2CFCF5FC43069F0F80181918F010E94D2
:10E5D000006A8823B1F3CBDF682F8C2F0E94503A5A
:10E5E000F0CF82E40E94006A882329F0C0DF682F00
:10E5F00084E00E94503ACF911F910F910C94FA3A07
:10E600000F931F93CF9383E50E94476A882309F4F1
:10E6100065C0ADDF823029F1833009F43FC081301D
:10E6200009F05CC00DE213E0C0E0F80181918F01B8
:10E630000E94476A882339F09ADF2FEF4FEF682F47
:10E640008C2F0E94F939CF5FC43079F782E40E94A1
:10E65000476A882309F442C08ADF2FEF4FEF682F03
:10E660003AC00DE213E0C0E0F80181918F010E94F1
:10E67000476A882339F07BDF2FEF482F6FEF8C2F0D
:10E680000E94F939CF5FC43079F782E40E94476A6B
:10E69000882321F16CDF2FEF482F1CC00DE213E01F
:10E6A000C0E0F80181918F010E94476A882339F008
:10E6B0005EDF282F4FEF6FEF8C2F0E94F939CF5F6D
:10E6C000C43079F782E40E94476A882339F04FDF2B
:10E6D000282F4FEF6FEF84E00E94F939CF911F91FF
:10E6E0000F910C94FA3ACF93DF931F921F92CDB7FC
:10E6F000DEB769837A830E94006A69817A81882300
:10E7000061F08091500C9091510C009731F04AE0EB
:10E7100050E060E070E00E94BCB1972F862F0F9010
:10E720000F90DF91CF9108951F93CF93DF9380E5F2
:10E730000E94006A882381F160E070E080E5D3DF09
:10E74000182F6FEF7FEF83E5CEDFEC010196039783
:10E7500018F517FD21C00E941459CF3F8FEFD8073D
:10E7600029F0219771F4C1E0D0E00DC0812F0E9403
:10E77000FA1331E020E0892B09F030E0C32FD22FCB
:10E7800002C0C0E0D0E0812F0E94FA138C179D07D1
:10E7900019F00E944BABF7CFDF91CF911F910895F5
:10E7A0000F931F93CF9383E50E94006A882309F497
:10E7B0003EC08091500C9091510C009701F1FC01EA
:10E7C0008F01C1912C2F2F7D89F0C53411F0C536F2
:10E7D000B9F7F801108260E070E08091500C9091E0
:10E7E000510C0E9456B0F801C08304C060E070E094
:10E7F0000E9456B0B62FA72FF82FE92F04C0B0E023
:10E80000A0E0F0E0E0E020E030E04AE754E46B2FE5
:10E810007A2F8F2F9E2F0E9404AF0E943AAD6093F3
:10E820000C0F70930D0F80930E0F90930F0FCF91DD
:10E830001F910F91089520E040E050E0BA010C9440
:10E840004C2F0C941BAA0F931F93CF9383E50E9428
:10E85000006A882391F18091500C9091510C00979F
:10E8600061F1FC018F01C1912C2F2F7D89F0C534FE
:10E8700011F0C536B9F7F801108260E070E08091C0
:10E88000500C9091510C0E9456B0F801C08304C006
:10E8900060E070E00E9456B020E030E04AE754E4C7
:10E8A0000E9404AF0E943AAD6093570270935802E1
:10E8B0008093590290935A0246C088E50E94006AEC
:10E8C000811114C089E50E94006A81110FC08AE598
:10E8D0000E94006A81110AC085E40E94006A8111C9
:10E8E00005C0CF911F910F910C94EF580E941459BD
:10E8F00088E50E94006A882331F0179A8091BC0550
:10E900008E7F8093BC0589E50E94006A882331F0E0
:10E91000169A8091BC058D7F8093BC058AE50E9484
:10E92000006A882331F0159A8091BC058B7F809313
:10E93000BC0585E40E94006A882329F0CF911F91CD
:10E940000F910C9420AACF911F910F910895FF92DF
:10E950000F931F93CF93DF9383E50E94006A882370
:10E96000F1F083E50E94006A811102C060E015C0E9
:10E970008091500C9091510C892BC1F30E948A6AAE
:10E9800097FDF4CF0E948A6A6F3F7105810591055A
:10E9900011F00CF03FC00E948A6A609393030E94BA
:10E9A000391687E296E10E942B1680919303882303
:10E9B00029F10DE116E1C0E0D0E020E08091930361
:10E9C00090E00C2E02C0959587950A94E2F780FF9F
:10E9D0000EC0FF24F394F20E222319F08CE20E9461
:10E9E000BB18F801859194910E942B162F2D21962A
:10E9F0000E5F1F4FC530D10509F704C089E196E1CC
:10EA00000E942B168AE0DF91CF911F910F91FF900A
:10EA10000C94BB186FEFC1CF0E94D2200E946BA74D
:10EA20000E94EF581092CE0468EE73E080E090E010
:10EA30000C94E91581E080935C0283E50E94006AF2
:10EA4000882331F08091500C9091510C892B39F42E
:10EA500083E50E94006A811112C00C94AC9E0E9452
:10EA60008A6A97FDFACF0E948A6A6F3F7105810515
:10EA7000910509F024F40E948A6A662371F30895CF
:10EA800081E00C94EA2D80E00C94EA2D0C9414594A
:10EA9000CF930E9439168EE496E10E942B1683E5EF
:10EAA0000E94006AC82F8823D1F08091500C909169
:10EAB000510C892B91F00E948A6A97FD0DC00E942B
:10EAC0008A6A6F3F71058105910509F034F40E944F
:10EAD0008A6AC1E0611101C0C0E0C0934102809127
:10EAE00041020E94B01686E496E10E942B16209106
:10EAF0006B0530916C0540916D0550916E056091EC
:10EB000035027091360280913702909138020E944E
:10EB1000EDABAB01BC0184E496E10E947616209136
:10EB20006F053091700540917105509172056091AB
:10EB3000390270913A0280913B0290913C020E940E
:10EB4000EDABAB01BC0181E496E10E947616209109
:10EB5000730530917405409175055091760560916B
:10EB60003D0270913E0280913F02909140020E94CE
:10EB7000EDABAB01BC018EE396E10E94761686E315
:10EB800096E10E942B1620916B0530916C05409107
:10EB90006D0550916E056091290270912A02809155
:10EBA0002B0290912C020E94EDABAB01BC0184E3DF
:10EBB00096E10E94761620916F0530917005409184
:10EBC00071055091720560912D0270912E02809115
:10EBD0002F02909130020E94EDABAB01BC0181E3AA
:10EBE00096E10E947616209173053091740540914C
:10EBF00075055091760560913102709132028091D5
:10EC00003302909134020E94EDABAB01BC018EE265
:10EC100096E10E9476168AE0CF910C94BB180F9370
:10EC20001F93CF93DF9383E50E94476A882309F4FB
:10EC300050C09DDC182F80E50E94476A81110AC0F0
:10EC400081E0111101C080E0DF91CF911F910F9100
:10EC50000C94D31580E50E94476A882331F00E9406
:10EC60008A6AEB0177FD35C002C0CDE0D0E00C2F01
:10EC700089E40E94476A882351F08091500C90915A
:10EC8000510C892B49F073DC811106C017C089E44F
:10EC90000E94006A882391F061E08C2F0E948F13FC
:10ECA000612F8C2F0E94CB13612F70E08C2F0E945C
:10ECB0007212083071F41093CE040BC0802F0E94A2
:10ECC000E4A9882349F3DF91CF911F910F910C9410
:10ECD0000CAADF91CF911F910F9108950C94E4A796
:10ECE0000C9480A70C946BA74F925F926F927F92C7
:10ECF000AF92BF92CF92DF92EF92FF92CF93DF93CA
:10ED0000EB01FC0160817181828193812CE3C22E31
:10ED1000D12CE12CF12CA70196010E94F1AFB62E67
:10ED2000A72ECA01B901A70196010E94F1AF6B019C
:10ED30007C01CA01B90128E130E040E050E00E94C6
:10ED4000F1AF2B013C01C9016DE671E00E94DDAF1E
:10ED500061157105D9F0AF92BF92DF92CF925F92A9
:10ED60004F929F938F937F936F9386E896E19F9343
:10ED70008F93DF93CF930E94B6B48DB79EB70E9654
:10ED80000FB6F8949EBF0FBE8DBF61C00097C9F04B
:10ED9000AF92BF92DF92CF925F924F929F938F93E9
:10EDA00086E796E19F938F93DF93CF930E94B6B44B
:10EDB000EDB7FEB73C960FB6F894FEBF0FBEEDBFA1
:10EDC00046C04114510461047104B9F0AF92BF927E
:10EDD000DF92CF925F924F928AE696E19F938F9354
:10EDE000DF93CF930E94B6B48DB79EB70A960FB645
:10EDF000F8949EBF0FBE8DBF2AC0C114D104E10498
:10EE0000F104A9F0AF92BF92DF92CF9282E696E131
:10EE10009F938F93DF93CF930E94B6B4EDB7FEB765
:10EE200038960FB6F894FEBF0FBEEDBF10C0AF927C
:10EE3000BF928EE596E19F938F93DF93CF930E94CD
:10EE4000B6B40F900F900F900F900F900F90DF912E
:10EE5000CF91FF90EF90DF90CF90BF90AF907F90D9
:10EE60006F905F904F900895CF93DF93CDB7DEB74B
:10EE700069970FB6F894DEBF0FBECDBF0E94B0A752
:10EE80006E8B7F8B888F998FBE016F5F7F4FCE0116
:10EE900046962ADF0E943916BE016F5F7F4F8AE9CE
:10EEA00096E10E943F168AE00E94BB1869960FB651
:10EEB000F894DEBF0FBECDBFDF91CF91089583E5FB
:10EEC0000E94006A882331F08091500C9091510C7F
:10EED000892B71F40E9439164091520250E060E093
:10EEE00070E087EA96E10E94A0168AE00C94BB18B5
:10EEF0000E948A6A97FD17C00E948A6A6F3F710557
:10EF00008105910509F01CF40E948A6A01C06FEF27
:10EF1000862F90E0CD971CF46093520208958CE305
:10EF200080935202089560E0F3CF81E00E94D315F0
:10EF30000E94512E80E00C94D3150E9414590C9419
:10EF4000674C1F93CF93DF93C091520CD091530C19
:10EF500083E010E040E08150C9F09881292F2B7F99
:10EF60002134C9F729812133B1F7913421F0953447
:10EF700019F441E001C011E09E012E5F3F4FE9010D
:10EF80002F5F3F4F98819032D1F3E5CF41110E941E
:10EF90003916112321F08EEA96E10E942B16CE013C
:10EFA000DF91CF911F910C9412190F931F93CF9360
:10EFB0008C01C62F82EB96E10E942B16C8010E949D
:10EFC0002B168AE30E94BB186AE070E08C2F90E059
:10EFD000CF911F910F910C94B41982EB97E10E948D
:10EFE0002B1660E082EA97E1E0DF61E08BE997E1D0
:10EFF000DCDF60E080E997E1D8DF61E080E897E15D
:10F00000D4DF60E087E797E1D0DF61E08DE697E14C
:10F01000CCDF61E083E697E1C8DF61E08BE597E153
:10F02000C4DF61E08DE497E1C0DF60E08FE397E14A
:10F03000BCDF60E080E397E1B8DF60E082E297E167
:10F04000B4DF60E08CE097E1B0DF61E08BEF96E148
:10F05000ACDF60E08CEE96E1A8DF60E087ED96E142
:10F06000A4DF61E084EC96E1A0DF60E087EB96E14D
:10F070009CCF8EE40E94006A8823A1F08091500CFE
:10F080009091510C009771F04AE050E060E070E020
:10F090000E94BCB16093F20E7093F30E8093F40E55
:10F0A0009093F50E0895EF92FF920F931F93CF93D5
:10F0B000DF93C1E3D3E010E089910E94006A8823C6
:10F0C00071F18091500C9091510C0097F1F0FC017E
:10F0D0007F010191202F2F7D89F0053411F0053635
:10F0E000B9F7F701108260E070E08091500C9091C8
:10F0F000510C0E9456B0F701008304C060E070E03C
:10F100000E9456B0362F272F04C030E020E080E068
:10F1100090E0432F522FBC01812F0E9446521F5F67
:10F12000133051F6DF91CF911F910F91FF90EF9027
:10F130000C94674C2F923F924F925F926F927F9206
:10F140008F929F92AF92BF92CF92DF92EF92FF92F7
:10F150000F931F93CF93DF93CDB7DEB72F970FB6E3
:10F16000F894DEBF0FBECDBF41E061E081E00E94B8
:10F170003B508111B0C08EEC882E84E1982E8BEA32
:10F1800095E09E878D87FE0131965F0103EB14E1C8
:10F190001F01F3E0F00FFF87F401659175918591F0
:10F1A0009491ED85FE85C190D190E190F190FE871C
:10F1B000ED87A70196010E94ECAB2B013C0120E0FA
:10F1C00030E040EA51EC0E94C9AE87FD10C020E05B
:10F1D00030E040EA51E4C301B2010E94C6AC181607
:10F1E00034F0F10140825182628273820DC0F801D5
:10F1F00084911816B4F7F7FAF094F7F8F094F10147
:10F20000C082D182E282F382F101C190D190E1907B
:10F21000F1901F0120E030E040EA51ECC701B60157
:10F220000E94C9AE87FD0AC020E030E040EA51E408
:10F23000C701B6010E94C6AC1816F4F40E943C1631
:10F2400088EA98E12F960FB6F894DEBF0FBECDBFC7
:10F25000DF91CF911F910F91FF90EF90DF90CF90B2
:10F26000BF90AF909F908F907F906F905F904F90E6
:10F270003F902F900C942B16F4E08F0E911C0F5F93
:10F280001F4F8F85801388CF10E0F5014191519178
:10F29000619171915F01812F0E9446521F5F13306F
:10F2A000A1F72F960FB6F894DEBF0FBECDBFDF914A
:10F2B000CF911F910F91FF90EF90DF90CF90BF9073
:10F2C000AF909F908F907F906F905F904F903F9006
:10F2D0002F900C94674C2F960FB6F894DEBF0FBE9C
:10F2E000CDBFDF91CF911F910F91FF90EF90DF90F5
:10F2F000CF90BF90AF909F908F907F906F905F90D6
:10F300004F903F902F9008953F924F925F926F924F
:10F310007F928F929F92AF92BF92CF92DF92EF92A5
:10F32000FF920F931F93CF93DF9385E3A82E83E083
:10F33000B82E9BEAE92E95E0F92E2BE6C22E25E0A9
:10F34000D22E912C312C812CF50181915F010E94EC
:10F35000006A882309F460C08091500C9091510C90
:10F36000009709F459C0FC013F01C1912C2F2F7D5A
:10F3700089F0C53411F0C536B9F7F301108260E0A9
:10F3800070E08091500C9091510C0E9456B0F301A6
:10F39000C08304C060E070E00E9456B08B01D82F9B
:10F3A000C92FF3E09F1651F0F6012081318142818F
:10F3B00053810E94ECAB8B01D82FC92FF70120811C
:10F3C000318142815381B8018D2F9C2F0E94ECAB7B
:10F3D0002B013C012DEB37E346E855EB0E94C9AE0B
:10F3E00087FD0AC02DEB37E346E855E3C301B201C0
:10F3F0000E94C6AC181684F4F3E09F1619F033246B
:10F40000339402C088248394C801AD2FBC2FF70128
:10F4100080839183A283B3839394F4E0EF0EF11C75
:10F4200084E0C80ED11CE4E09E128ECF332019F088
:10F430000E94B04C03C081100E94BA4CDF91CF9162
:10F440001F910F91FF90EF90DF90CF90BF90AF9002
:10F450009F908F907F906F905F904F903F900C9413
:10F46000674CBF92CF92DF92EF92FF920F931F9360
:10F47000CF93DF9329E3E22E23E0F22E06E51CE092
:10F480006701C0E0D0E0BB24B394F60181916F0125
:10F490000E94006A882351F10E941459F80160818A
:10F4A000662389F070E080E090E00E9468AD9B01E7
:10F4B000AC01FE01E75AF34F608171818281938133
:10F4C0000E94CDAC03C060E070E0CB012091500CF5
:10F4D0003091510C232B11F00E94536AFE01E75921
:10F4E000F34F6083718382839383B12C24960F5FE3
:10F4F0001F4FCC30D10549F686E40E94006A88236C
:10F5000071F10E9414590E94536A8B01D82FC92FA0
:10F5100020E030E040E85FE30E94C9AE18167CF0BE
:10F5200020E030E0A901B8018D2F9C2F0E94C6ACCD
:10F5300087FF09C000E010E0D0E0C0E004C000E0B8
:10F5400010E0D0E8CFE3C801AD2FBC2F8093650C4D
:10F550009093660CA093670CB093680CB12C83E574
:10F560000E94006A882369F00E9414590E94536A1D
:10F570006093530270935402809355029093560205
:10F58000ABC0BB2009F4A8C083E999E10E942B1607
:10F5900020E030E0A9016091650C7091660C8091CB
:10F5A000670C9091680C0E94C6AC811104C080E980
:10F5B00099E10E942B1687E899E10E942B16409151
:10F5C000650C5091660C6091670C7091680C83E635
:10F5D00099E10E94761682E499E10E942B1680E25E
:10F5E00099E10E942B1609E61CE0C9E3D3E093E001
:10F5F000D92EDE0C80E20E94BB1889910E94BB18B4
:10F60000F80161917191819191918F0142E050E0F7
:10F610000E94391A8AE00E94BB18DC12EBCF40919D
:10F6200053025091540260915502709156028CEF32
:10F6300098E10E9476168AE00E94BB188AED98E154
:10F640000E942B1689E5C82E8CE0D82EC6E5DCE09A
:10F6500013E01C0F88818823D1F080E20E94BB1840
:10F66000F70180810E94BB18688170E080E090E023
:10F670000E9468AD9B01AC01F601608171818281BD
:10F6800093810E94CDAC42E050E00E94391A21964D
:10F69000FFEFEF1AFF0A84E0C80ED11C1C13DACF6B
:10F6A0008091560C81110CC08091570C811108C0BB
:10F6B0008091580C811104C086EC98E10E942B16B1
:10F6C0008AE0DF91CF911F910F91FF90EF90DF9033
:10F6D000CF90BF900C94BB18DF91CF911F910F91E9
:10F6E000FF90EF90DF90CF90BF9008952F923F92C0
:10F6F0004F925F926F927F928F929F92AF92BF9242
:10F70000CF92DF92EF92FF920F931F93CF93DF93ED
:10F71000CDB7DEB76A970FB6F894DEBF0FBECDBF88
:10F72000182F81E00E94D3158FE40E94476A882336
:10F73000B9F08091500C9091510C892BB1F00E943E
:10F740008A6A97FD18C00E948A6A6F3F7105810519
:10F75000910509F054F40E948A6A611106C00BC039
:10F760008FE40E94006A882331F09091BD05977064
:10F77000973009F40FC20E94145920914006288F37
:10F7800080E00E94AF1A0E94EB4E81E00E94FD2DA6
:10F79000111119C088E50E94006A382E89E50E947F
:10F7A000006A182F8AE50E94006A282E311006C0D0
:10F7B000111110C081110EC0312E0AC0112351F059
:10F7C000312E082F08C011E03324339422242394CF
:10F7D00001E001C000E080E1EBEAF5E0ABE9B5E073
:10F7E00001900D928A95E1F7011102C0222019F0D3
:10F7F00082E00E94BE5182E50E94476A882371F12F
:10F800008091500C9091510C009709F457C0FC0165
:10F810005F012191322F3F7D99F0253411F025367B
:10F82000B9F7D5011C9260E070E08091500C909186
:10F83000510C2A8F0E9456B02A8DF501208304C0F6
:10F8400060E070E00E9456B06B017C0120E030E087
:10F85000A9010E94C6AC882389F106C0C12CD12C15
:10F8600020E8E22E30E4F32E011105C0311003C070
:10F87000112309F410C1C601D7018093A305909309
:10F88000A405A093A505B093A6052091B3053091DA
:10F89000B4054091B5055091B605B601C7010E9467
:10F8A000C9AE18165CF419821A821B821C82BE0132
:10F8B0006F5F7F4F83EA95E00E94724E01110CC08A
:10F8C000332009F4FCC0111107C080E00E94BE5132
:10F8D000002309F47EC1DCC01092AF051092B00580
:10F8E0001092B1051092B2051092AB051092AC05C2
:10F8F0001092AD051092AE050E94B04CE3EBF4E11E
:10F900002491298FE2ECF4E185909590A590B49034
:10F91000E6ECF4E14590559065907490A301920156
:10F92000C501B4010E94C9AE18162CF4A5019401BA
:10F93000C301B20104C0A3019201C501B4010E9438
:10F94000CDAC6B017C01EBEAF4E185919591A59139
:10F95000B4918D879E87AF87B88BE7EAF4E18591F4
:10F960009591A591B491898B9A8BAB8BBC8B2D858E
:10F970003E854F855889BC01CD010E94C6AC87FDEC
:10F9800009C09D859D8BAE85AE8BBF85BF8BE889F9
:10F99000ED8708C0F989FD8B2A892E8B8B898F8B87
:10F9A0009C899D87A7019601C701B6010E9404AFFB
:10F9B00020E030E040E85FE30E94EDAB0E9471AFD1
:10F9C0009B01AC016D897E898F899D850E9404AF62
:10F9D00069877A878B879C87E4EBF4E1F49020E0D9
:10F9E00030E040EC5FE3C301B2010E9404AF2B01A1
:10F9F0003C016F2DFF0C770B880B990B0E9468ADB3
:10FA00009B01AC01C301B2010E9404AF69837A83F8
:10FA10008B839C8320E030E040EC5FE3C501B401C0
:10FA20000E9404AF6B017C01A98D6A2FAA0F770B8E
:10FA3000880B990B0E9468AD9B01AC01C701B60110
:10FA40000E9404AF6D837E838F839887AE01475FEA
:10FA50005F4FBE016F5F7F4FCE0105960E94904EB3
:10FA60000E94C42D1092AF051092B0051092B105FE
:10FA70001092B2051092AB051092AC051092AD0534
:10FA80001092AE05011121CF3110A0C0112319F041
:10FA900081E00E94BE510E94B04CF090DF0480E0F3
:10FAA0000E94EA2D812C912C90EAA92E90E4B92E87
:10FAB00089829A82AB82BC82011115C0A8C0111143
:10FAC000E7CF0E94B04CF090DF0480E00E94EA2D66
:10FAD00080E090E0A0EAB0E489839A83AB83BC83A2
:10FAE000222009F48BC080E090E0ADE1B3E48D8387
:10FAF0009E83AF83B887BE016F5F7F4FCE010596AF
:10FB00000E94724E80E090E0A0EAB0E489839A837C
:10FB1000AB83BC8301110BC0111109C08091AF05EB
:10FB20009091B005A091B105B091B20504C080E0FC
:10FB300090E0A9E3B3E48D839E83AF83B88701117E
:10FB40000BC0311009C08091AB059091AC05A0911C
:10FB5000AD05B091AE0504C080E090E0A0EAB0E44D
:10FB600089879A87AB87BC87AE014F5F5F4FBE0125
:10FB70006B5F7F4FCE0109960E94904E8F2D0E94A1
:10FB8000EA2D0E94BF2D888D0E94AF1A0E940A4F55
:10FB90000E94674C80E00E94D3156A960FB6F894D5
:10FBA000DEBF0FBECDBFDF91CF911F910F91FF90B0
:10FBB000EF90DF90CF90BF90AF909F908F907F900D
:10FBC0006F905F904F903F902F90089580E00E943B
:10FBD000BE5111115DCF0E94B04CF090DF0480E067
:10FBE0000E94EA2D812C912C80EAA82E80E4B82E68
:10FBF00089829A82AB82BC8221101FC08091B3059A
:10FC00009091B405A091B505B091B60570CF2220B2
:10FC1000A9F380E090E0ADE1B3E48D839E83AF83F0
:10FC2000B887BE016F5F7F4FCE0105960E94724E6E
:10FC300089829A82AB82BC826FCF80E090E0ADE196
:10FC4000B3E48D839E83AF83B887BE016F5F7F4F20
:10FC5000CE0105960E94724E89829A82AB82BC8246
:10FC60005DCF80E1EBEAF5E0ABE9B5E001900D9204
:10FC70008A95E1F708954F925F926F927F928F92EB
:10FC80009F92AF92BF92CF92DF92EF92FF920F932B
:10FC90001F93CF93DF93CDB7DEB72E970FB6F894AF
:10FCA000DEBF0FBECDBF270138012E874A875B8795
:10FCB0006C877D878987D5DF89852E854A855B8519
:10FCC0006C857D858F3F51F094E0899FF001112470
:10FCD000E556FA4F40835183628373832F3F51F07F
:10FCE000A4E02A9FF0011124E556FA4F4082518288
:10FCF00062827382BFEFCB1651F084E0C89EF001A0
:10FD00001124E556FA4F80829182A282B3828090BC
:10FD10009B0590909C05A0909D05B0909E0520E0CD
:10FD200030E042E253E4C501B4010E94C6AC87FF53
:10FD300011C020E030E040E450ECC501B4010E9465
:10FD4000C9AE18166CF0812C912C30E4A32E30EC47
:10FD5000B32E06C0812C912C22E2A22E23E4B22ED7
:10FD600080929B0590929C05A0929D05B0929E0565
:10FD700040909F055090A0056090A1057090A2054D
:10FD800020E030E04EE353E4C301B2010E94C6AC70
:10FD900087FF11C020E030E040EE50ECC301B2011B
:10FDA0000E94C9AE18166CF0412C512C90EE692EB1
:10FDB00090EC792E06C0412C512C8EE3682E83E402
:10FDC000782E40929F055092A0056092A1057092F6
:10FDD000A2058091A3059091A405A091A505B091DD
:10FDE000A6058D839E83AF83B88720E030E04FE186
:10FDF00053E4BC01CD010E94C6AC87FF11C020E0D6
:10FE000030E040E050EC6D817E818F8198850E94CA
:10FE1000C9AE18166CF080E090E0A0E0B0EC04C031
:10FE200080E090E0AFE1B3E48D839E83AF83B88739
:10FE30008D819E81AF81B8858093A3059093A405A1
:10FE4000A093A505B093A60580E090E0A8E4B2E4F5
:10FE500089839A83AB83BC83DE0111966D01ED80AB
:10FE6000FE800F811885A3019201C501B4010E9493
:10FE7000964D2E960FB6F894DEBF0FBECDBFDF9124
:10FE8000CF911F910F91FF90EF90DF90CF90BF9097
:10FE9000AF909F908F907F906F905F904F9008955C
:10FEA0008F929F92AF92BF92CF92DF92EF92FF928A
:10FEB0000F931F93CF93DF93EC016A017B0120E046
:10FEC00030E040E45FE3688579858A859B850E9400
:10FED000EDABA70196010E94EDABAB01BC01812CFB
:10FEE000912C5401CC24CA94850174012FEF82E037
:10FEF000C2DEEC80FD800E811F81488159816A81BC
:10FF00007B8121E080E0B7DEDF91CF911F910F91DF
:10FF1000FF90EF90DF90CF90BF90AF909F908F9029
:10FF200008952F923F924F925F926F927F928F929D
:10FF30009F92AF92BF92CF92DF92EF92FF920F9378
:10FF40001F93CF93DF93CDB7DEB72E970FB6F894FC
:10FF5000DEBF0FBECDBF89878B014A87222359F0B0
:10FF6000812C912C90E8A92E9EE3B92E80E090E0A0
:10FF7000A0EAB1E40CC08AE0882E87ED982E83E2D7
:10FF8000A82E8CE3B82E80E090E0A0E8BFE3898340
:10FF90009A83AB83BC83211105C080E090E0A0EA86
:10FFA000B0E404C080E090E0A8E4B2E48D839E83D6
:10FFB000AF83B88756DE412C512C3201B985A4E0BD
:10FFC000BA9FC0011124FC01E556FA4F1F01C80178
:10FFD000110FAA0BBB0B8B879C87AD87BE872D812A
:10FFE0003E814F815885C301B2010E94C6AC87FF94
:10FFF0003FC06B857C858D859E850E9468ADA5017F
:020000021000EC
:1000000094010E9404AF9B01AC01D1016D917D91DF
:100010008D919C910E94EDABF1016083718382838D
:100020009383E090A305F090A4050091A50510919D
:10003000A60520919F053091A0054091A105509102
:10004000A20560919B0570919C0580919D05909102
:100050009E05DE0111966D010E94964D0E94145975
:1000600083B182958170B1E08B27EA858E1324C01D
:10007000398524E0329FF0011124E556FA4F608162
:100080007181828193812E960FB6F894DEBF0FBEE8
:10009000CDBFDF91CF911F910F91FF90EF90DF9037
:1000A000CF90BF90AF909F908F907F906F905F9018
:1000B0004F903F902F900895A5019401C301B20184
:1000C0000E94EDAB2B013C018ACF4F925F926F9261
:1000D0007F928F929F92AF92BF92CF92DF92EF92D8
:1000E000FF920F931F93CF93DF93CDB7DEB728977F
:1000F0000FB6F894DEBF0FBECDBFB82E6B01A42E95
:100100004901C801B701FF24F39420E030E040EA40
:1001100050E40E94C6AC8111F12CA3DD84E0B89EAE
:1001200080011124F801E556FA4F80819181A28166
:10013000B3818D839E83AF83B8872F2D4A2DB6015F
:100140008B2DEFDE2B013C018114910411F1F11094
:1001500020C041E04A25662777276C197D0920E0F9
:100160008B2DDFDEA30192010E94ECAB6B017C01C1
:1001700020E030E0A9010E94C9AE87FF04C0F7FA71
:10018000F094F7F8F094D401CD92DD92ED92FC92C8
:100190001397F801E556FA4F8D819E81AF81B8859E
:1001A00080839183A283B38380E090E0A8E4B2E4EB
:1001B00089839A83AB83BC83E090A305F090A40568
:1001C0000091A5051091A60520919F053091A005ED
:1001D0004091A1055091A20560919B0570919C05ED
:1001E00080919D0590919E05DE0111966D010E9402
:1001F000964DC301B20128960FB6F894DEBF0FBE2C
:10020000CDBFDF91CF911F910F91FF90EF90DF90C5
:10021000CF90BF90AF909F908F907F906F905F90A6
:100220004F9008952F923F924F925F926F927F92DC
:100230008F929F92AF92BF92CF92DF92EF92FF92F6
:100240000F931F93CF93DF93CDB7DEB769970FB6A8
:10025000F894DEBF0FBECDBF3C014C8B5D8B6E8B27
:100260007F8B2D878CE0EDEEF2E0DE0111960190A0
:100270000D928A95E1F74C895D896E897F89C3016A
:100280000FDE2D852230D1F060F42223F1F02130F1
:1002900009F073C1212C312C60E8462E6FEB562EED
:1002A00046C03D853330C9F1343009F066C1212C98
:1002B000312C70E8472E7FEB572E36C0212C312C85
:1002C000F0E84F2EFFE35F2E2FC09301205E3F4FDB
:1002D000EC88FD880E891F8941E06FEF7FEF82E097
:1002E000F4DE6B017C0120E030E040E05FE36985F3
:1002F0007A858B859C850E9404AF9B01AC01C70168
:10030000B6010E94ECABF301608771878287938707
:10031000C486D586E686F78630C1212C312CE0E8EC
:100320004E2EEFE35E2E03C0DD24D39401C0D12C0A
:100330002D2D30E03F872E87002309F463C0C901CB
:10034000880F991F880F991F7301E80EF91EE1E0CD
:10035000F0E0EC0FFD1FE80FF91F20E030E040E077
:100360005FE360817181828193810E9404AFF70114
:10037000E05CFF4F20813181428153810E94ECABD0
:100380009B01AC01C201B10190580E9404AFF7017A
:1003900020813181428153810E94EDABAB01BC01D0
:1003A000812C912C5401CC24CA94850174012FEF27
:1003B0008D2D61DCEC88FD880E891F899301205EFC
:1003C0003F4F41E06FEF7FEF82E07FDE4B015C014A
:1003D000F301648775878687978720E030E040E0E7
:1003E0005FE369857A858B859C850E9404AF9B01BC
:1003F000AC01C501B4010E94ECABF30160877187C9
:10040000828793878E859F85880F991F880F991FF4
:100410009301280F391F3F872E87E1E0F0E0EC0FB2
:10042000FD1FE80FF91F20E030E040E05FE360814E
:100430007181828193810E9404AF688B798B8A8B52
:100440009B8B52014101B7FAB094B7F8B0948E85F6
:100450009F85805C9F4F998F888F20E030E040E03F
:100460005FE3FC0160817181828193810E9404AF0E
:100470009B01AC01688979898A899B890E94EDABCF
:100480002C893D894E895F890E94EDAB9B01AC01AF
:10049000C501B4010E9404AFEE85FF852081318142
:1004A000428153810E94EDABAB01BC01812C912CA8
:1004B0005401CC24CA94850174012FEF8D2DDBDB10
:1004C00023E333E343E35FE3F301648575858685C6
:1004D00097850E94ECABAB01BC012FEF82E0CBDB38
:1004E000FD85AF2EB12C450128E0820E911C880CB1
:1004F000991C880C991C860C971CC201B1010E94A2
:1005000035ADEC88FD880E891F89940141E08D2D61
:10051000DCDD6B017C0120E030E040E05FE3E88D52
:10052000F98D60817181828193810E9404AF9B016A
:10053000AC01688979898A899B890E94EDAB9B010E
:10054000AC01C201B1010E9404AF9B01AC01C70123
:10055000B6010E94EDABEE85FF85608371838283D7
:100560009383F5013396EE0FFF1FEE0FFF1FE60D8D
:10057000F71DC082D182E282F38269960FB6F894A9
:10058000DEBF0FBECDBFDF91CF911F910F91FF90C6
:10059000EF90DF90CF90BF90AF909F908F907F9023
:1005A0006F905F904F903F902F900895CF92DF9281
:1005B000EF92FF920F93CF93DF93EC016A017B01DF
:1005C00000E020E02FDE22E0B701A601CE012ADE06
:1005D00023E0B701A601CE0125DEB701A601CE01B9
:1005E0005FDC1CAA1DAA1EAA1FAA18AE19AE1AAE5D
:1005F0001BAE288539854A855B8560E070E0CB01BC
:100600000E94ECAB6CAF7DAF8EAF9FAFDF91CF910F
:100610000F91FF90EF90DF90CF9008958F929F926F
:10062000AF92BF92CF92DF92EF92FF920F931F9300
:10063000CF93DF93EC01C090650CD090660CE090F6
:10064000670CF090680C80E090E0A0E8BFE3809336
:10065000650C9093660CA093670CB093680C809027
:10066000530290905402A0905502B09056021092FE
:100670005302109254021092550210925602CE016B
:1006800095DF0E9414590BEA15E02CAD3DAD4EAD3F
:100690005FADF80160857185828593850E94EDAB21
:1006A000F8016087718782879387188619861A8672
:1006B0001B861CAE1DAE1EAE1FAE0E94B04C8092BB
:1006C000530290925402A0925502B0925602C092E8
:1006D000650CD092660CE092670CF092680CDF918A
:1006E000CF911F910F91FF90EF90DF90CF90BF902F
:1006F000AF909F908F9008952F923F924F925F926C
:100700006F927F928F929F92AF92BF92CF92EF9211
:10071000FF920F931F93CF93DF93CDB7DEB7289748
:100720000FB6F894DEBF0FBECDBF5C018091650CA3
:100730009091660CA091670CB091680C8D839E839C
:10074000AF83B8871092650C1092660C1092670CFC
:100750001092680C8091530290915402A09155021E
:10076000B091560289839A83AB83BC831092530263
:10077000109254021092550210925602C50116DFD3
:10078000E9E6FCE0D5019C964D915D916D917C91DF
:100790009F97408351836283738398964D915D91B7
:1007A0006D917C919B974483558366837783909664
:1007B0004D915D916D917C919397408751876287B0
:1007C000738780E090E0A0E8BFE38093650C90938E
:1007D000660CA093670CB093680C109253021092B1
:1007E000540210925502109256028BEA282E85E090
:1007F000382E20E030E040E450E4F101608571855E
:10080000828593850E94EDAB4B015C0120E030E0D6
:1008100040E450E4D10114966D917D918D919C91AD
:1008200017970E94EDAB2B013C0120E030E040E443
:1008300050E4F10160817181828193810E94EDAB6E
:10084000AB01BC0192E0C92E8301720121E080E07E
:1008500012DA20E030E040E450E4D10118966D91C6
:100860007D918D919C911B970E94ECAB4B015C019B
:1008700020E030E040E450E4F1016481758186813C
:1008800097810E94ECAB2B013C0120E030E040E47A
:1008900050E4D1016D917D918D919C910E94ECABC2
:1008A000AB01BC018301720121E080E0E4D98981C0
:1008B0009A81AB81BC818093530290935402A093A0
:1008C0005502B09356028D819E81AF81B885809389
:1008D000650C9093660CA093670CB093680C2896F7
:1008E0000FB6F894DEBF0FBECDBFDF91CF911F9141
:1008F0000F91FF90EF90CF90BF90AF909F908F900F
:100900007F906F905F904F903F902F9008958F92BF
:100910009F92AF92BF92CF92DF92EF92FF92C090E0
:10092000650CD090660CE090670CF090680C812C00
:10093000912C20E8A22E2FE3B22E8092650C90928B
:10094000660CA092670CB092680C80905302909055
:100950005402A0905502B090560210925302109289
:100960005402109255021092560258DE80925302A1
:1009700090925402A0925502B0925602C092650C19
:10098000D092660CE092670CF092680CFF90EF90AA
:10099000DF90CF90BF90AF909F908F9008959C0173
:1009A0008CE0E9EFF2E0D90101900D928A95E1F730
:1009B00098E0E5E0F3E0D901A05CBF4F01900D9213
:1009C0009A95E1F708954F925F926F927F928F927E
:1009D0009F92AF92BF92CF92EF92FF920F931F938D
:1009E000CF93DF93CDB7DEB7CC54D1090FB6F894CF
:1009F000DEBF0FBECDBFCE010196D1DF4090650CAA
:100A00005090660C6090670C7090680C80E090E0ED
:100A1000A0E8BFE38093650C9093660CA093670CED
:100A2000B093680C8091530290915402A0915502AA
:100A3000B09156022D968CAF9DAFAEAFBFAF2D9744
:100A400010925302109254021092550210925602C4
:100A500040E050E060EA70E4CE01019658DF40E0EB
:100A600050E060E87FE3CE01019646DE40E050E0D2
:100A700060E87FE3CE0101964ADF812C912C54017E
:100A8000CC24CA94850174012FEF40E050E066E168
:100A900073E480E0F0D82D968CAD9DADAEADBFADCA
:100AA0002D978093530290935402A0935502B093D4
:100AB00056024092650C5092660C6092670C7092E0
:100AC000680CC45BDF4F0FB6F894DEBF0FBECDBF1E
:100AD000DF91CF911F910F91FF90EF90CF90BF903A
:100AE000AF909F908F907F906F905F904F90089500
:100AF0009F92AF92BF92CF92DF92EF92FF920F93AD
:100B00001F93CF93DF93CDB7DEB7C854D1090FB68B
:100B1000F894DEBF0FBECDBF81E00E94D3150091D7
:100B20004102109241029090400680E00E94AF1A6C
:100B300041E061E081E00E943B508111EEC0CE01B6
:100B400001962DDF85E50E94006A882341F12091FE
:100B5000500C3091510C2115310509F1F9015F015B
:100B60001191812F8F7D99F0153411F01536B9F759
:100B7000F501108260E070E08091500C9091510C72
:100B80000E9456B06B017C01F50110830EC060E03D
:100B900070E0C9010E9456B06B017C0106C0C12CF7
:100BA000D12C80E8E82E8FE3F82E82E40E94006AC0
:100BB000882331F0B701A601CE0101969DDDADC0BD
:100BC00084E50E94006A882391F08091500C9091F6
:100BD000510C009731F04AE050E060E070E00E9474
:100BE000BCB1B701A601CE01019618DD96C086E51D
:100BF0000E94006A882309F48FC0B701A601CE01C4
:100C00000196D4DC8AE00E94BB188DE29AE10E9432
:100C10002B164D855E856F85788985E29AE10E9465
:100C200076168AE00E94BB18498D5A8D6B8D7C8D9B
:100C30008CE19AE10E9476168AE00E94BB184D89E9
:100C40005E896F89788D82E19AE10E9476168AE04A
:100C50000E94BB188AE00E94BB1889E09AE10E94BA
:100C60002B1649855A856B857C8586E09AE10E9422
:100C700076168AE00E94BB188AE00E94BB188BEFB0
:100C800099E10E942B164DA55EA56FA578A982EF6C
:100C900099E10E9476168AE00E94BB1849A55AA5E0
:100CA0006BA57CA588EE99E10E9476168AE00E94E9
:100CB000BB1849A15AA16BA17CA180EE99E10E94C9
:100CC00076168AE00E94BB188AE00E94BB1882EC6C
:100CD00099E10E942B168AE00E94BB1884E50E94CD
:100CE000BB186AE070E080E090E00E94AE198EEAE6
:100CF00099E10E942B1621964CAD5DAD6EAD7FAD96
:100D000021978BEA99E10E9476168AE00E94BB182F
:100D10008AE00E94BB1801C056DE892D0E94AF1ADE
:100D20000093410280E00E94D315C85BDF4F0FB6ED
:100D3000F894DEBF0FBECDBFDF91CF911F910F9111
:100D4000FF90EF90DF90CF90BF90AF909F9008956D
:100D50001F93CF93DF93CDB7DEB72C970FB6F894E0
:100D6000DEBF0FBECDBF83E50E94006A8823B9F0C5
:100D70008091500C9091510C892BC9F00E948A6A85
:100D800097FD10C00E948A6A6F3F71058105910529
:100D900009F06CF40E948A6A611109C003C01091C5
:100DA000400606C080E00E94AF1A10E001C011E0CA
:100DB0008091AB059091AC05A091AD05B091AE05C9
:100DC00089839A83AB83BC838091AF059091B005F2
:100DD000A091B105B091B2058D839E83AF83B88792
:100DE0008091B3059091B405A091B505B091B60579
:100DF00089879A87AB87BC8786E50E94006A88232B
:100E000031F062E67AE18CE196E00E9497A6812FAC
:100E10000E94AF1A112351F080914006811106C043
:100E20000E943C1683E49AE10E942B160E94391618
:100E300085E39AE10E942B16809140060E94B81625
:100E40004CE050E06BEA75E0CE0101960E947EB462
:100E5000892B59F02C960FB6F894DEBF0FBECDBF8C
:100E6000DF91CF911F910C94674C2C960FB6F8949C
:100E7000DEBF0FBECDBFDF91CF911F9108958F923E
:100E80009F92AF92BF92CF92DF92EF92FF92CF9359
:100E90004B015C0169017A0122ED30E040EE50EC3B
:100EA000C701B6010E94C9AE87FD33C027E030E01C
:100EB0004EE353E4C701B6010E94C6AC18164CF1CC
:100EC00023EA31E040E450ECC501B4010E94C9AE10
:100ED00087FD1FC027E030E042E253E4C501B401C2
:100EE0000E94C6AC1816ACF027E030E041E253E4B3
:100EF000C501B4010E94C6AC18165CF0C1E027E041
:100F000030E041E253E4C701B6010E94C6AC1816B6
:100F10000CF4C0E08C2FCF91FF90EF90DF90CF903A
:100F2000BF90AF909F908F900895CF93DF93D82F6D
:100F3000C62F0E94476A8823D1F08091500C90916F
:100F4000510C892B11F481E01AC00E948A6A97FD26
:100F500015C00E948A6A6F3F71058105910509F0ED
:100F600094F70E948A6A81E0611109C007C08D2F41
:100F70000E94006A8111E7CF8C2F01C080E0DF91D1
:100F8000CF9108952F923F924F925F926F927F92EE
:100F90008F929F92AF92BF92CF92DF92EF92FF9289
:100FA0000F931F93CF93DF93CDB7DEB7CB51D140D3
:100FB0000FB6F894DEBF0FBECDBF81E00E94D315FF
:100FC00041E061E081E00E943B5081111AC08091B4
:100FD0004006882329F060E08FE4A7DF811111C06B
:100FE000FE0131968CE3DF011D928A95E9F730907E
:100FF00040068AE40E94006A982E882329F00E9405
:10100000CE1A912C0C94FC9160E070E086E50E9471
:101010007373C351DF4F99838883CD5ED0400597AA
:1010200018F085E49CE15FC160E084E47EDFC95094
:10103000DF4F8883C75FD040C351DF4F288139819C
:10104000CD5ED040233031054CF460E084E56DDFA7
:10105000C450DF4F8883CC5FD04006C031E0C4501D
:10106000DF4F3883CC5FD04062E070E088E50E94BB
:101070007373182F62E070E089E50E947373082F84
:1010800080E50E94476A811103C0612F802F03C051
:101090000E948A6A862F623019F08CE19CE123C19C
:1010A000823019F083EF9BE11EC183E50E94476AFD
:1010B000882319F00E94536A04C060E070E88BEB4B
:1010C00095E420E030E040E752E40E94CDAC60932C
:1010D000420270934302809344029093450288E455
:1010E0000E94006A882399F10E94536A0E9435ADDC
:1010F0008B0177FF02C00F5F1F4F15950795119564
:1011000001951109035B1F4F0E3F4FEF14072CF49D
:101110004DEFA42EBB24BA9401C058016501C60E40
:10112000D71E51EAC516D1041CF031EAC32ED12CCA
:101130000A3FAFEF1A0714F409EF1FEF7801E60E2C
:10114000F71EB1EAEB16F1040CF461C05DC08CE44B
:101150000E94476A882381F00E94536A20916B05A0
:1011600030916C0540916D0550916E050E94ECAB7D
:101170000E9435AD5B0104C02DEFA22EBB24BA94B2
:1011800082E50E94476A882381F00E94536A209179
:101190006B0530916C0540916D0550916E050E9474
:1011A000ECAB0E9435AD6B0103C091EAC92ED12C86
:1011B00086E40E94476A882381F00E94536A209146
:1011C0006F053091700540917105509172050E9434
:1011D000ECAB0E9435AD8B0102C009EF1FEF82E43A
:1011E0000E94476A882381F00E94536A20916F050C
:1011F0003091700540917105509172050E94ECABE1
:101200000E9435AD7B0103C081EAE82EF12CB801C4
:10121000012E000C880B990B0E9468ADC250DF4F65
:10122000688379838A839B83CE5FD040B5010B2C82
:10123000000C880B990B0E9468ADCE5FDE4F68836F
:1012400079838A839B83C250D140C250DF4F28816B
:1012500039814A815B81CE5FD04011DE882309F459
:1012600040C0B7010F2C000C880B990B0E9468AD91
:101270009B01AC01B6010D2C000C880B990BC85ECC
:10128000DE4F2883C851D140C75EDE4F3883C95135
:10129000D140C65EDE4F4883CA51D140C55EDE4FA5
:1012A0005883CB51D1400E9468ADC85EDE4F288183
:1012B000C851D140C75EDE4F3881C951D140C65EAA
:1012C000DE4F4881CA51D140C55EDE4F5881CB51B7
:1012D000D140D5DDCA50DF4F8883C65FD040811131
:1012E00006C087ED9BE10E942B160C94FC91B60181
:1012F0006A197B09072E000C880B990B0E9468ADB8
:10130000C65FDE4F688379838A839B83CA50D1404E
:10131000B701601B710B072E000C880B990B0E9404
:1013200068ADC25FDE4F688379838A839B83CE502A
:10133000D140C351DF4FE881F981CD5ED040EF2B22
:1013400091F081EC9BE10E942B16C950DF4FE881A0
:10135000C75FD040EE2321F087EB9BE10E942B1664
:101360008AE00E94BB180E94145980E00E94AF1AC4
:1013700081E00E940F49882329F0832D0E94AF1A33
:101380000C94FC910E94EB4E60E085E4CEDD81116F
:1013900007C0F2E0C350DF4FF883CD5FD04006C0F6
:1013A00021E0C350DF4F2883CD5FD040C151DF4FD4
:1013B00019821882CF5ED040C752DF4F188219823F
:1013C0001A821B82C95DD040C850DF4F1882198233
:1013D0001A821B82C85FD040C751DF4F1882C95E96
:1013E000D0404FEF5FEFC352DF4F59834883CD5D4D
:1013F000D0405FEFCB50DF4F5883C55FD0408FEFB9
:10140000CD50DF4F8883C35FD04091E0CB52DF4F98
:101410009883C55DD040C352DF4F88819981CD5DEF
:10142000D0400196880F991F880F991F4DE350E017
:101430004C0F5D1F480F591FCB51DF4F5983488315
:10144000C55ED040DC011497C85FDE4FB983A88326
:10145000C850D1408CE0C352DF4F28813981CD5D27
:10146000D040829FF001839FF00D1124CA5FDE4FB0
:10147000F983E883C650D140CF51DF4F19821882DB
:10148000C15ED040C151DF4F88819981CF5ED0408D
:10149000092E000CAA0BBB0BCE5EDE4F888399830E
:1014A000AA83BB83C251D140C151DF4FA881B9810A
:1014B000CF5ED040AA0FBB1FCA5EDE4FB983A883A0
:1014C000C651D140CB52DF4F5881C55DD040CD5081
:1014D000DF4F8881C35FD040581709F497C2CE5EB2
:1014E000DE4F688179818A819B81C251D1400E94FF
:1014F00068AD9B01AC01C65FDE4F688179818A814E
:101500009B81CA50D1400E9404AF9B01AC01CE5FC9
:10151000DE4F688179818A819B81C250D1400E94CF
:10152000EDAB4B015C01CB52DF4FB881C55DD040C4
:101530006B2FBB0F770B880B990B0E9468AD9B013B
:10154000AC01C25FDE4F688179818A819B81CE5078
:10155000D1400E9404AF9B01AC01C250DF4F6881B3
:1015600079818A819B81CE5FD0400E94EDAB6B0177
:101570007C0120E030E0A901C501B4010E94C6ACA5
:1015800087FD05C020E030E040E05FE303C020E0DD
:1015900030E0A901C501B4010E94EDAB0E94A3ADEA
:1015A000C355DF4F688379838A839B83CD5AD040AC
:1015B00020E030E0A901C701B6010E94C6AC87FD5A
:1015C00005C020E030E040E05FE303C020E030E011
:1015D000A901C701B6010E94EDAB0E94A3ADC7559A
:1015E000DF4F688379838A839B83C95AD040C35273
:1015F000DF4FE881F981CD5DD0403196C352DF4F96
:10160000F983E883CD5DD040CA5EDE4FE881F98181
:10161000C651D140CB52DF4F2881C55DD040E20F8B
:10162000F11D27FDFA95EE0FFF1F41EA50E04C0F28
:101630005D1FE40FF51FC352DF4F88819981CD5D97
:10164000D0409183808301E0C351DF4F2881CD5E7C
:10165000D040C350DF4F4881CD5FD040BE016755B9
:101660007F4FCE0183559F4F0E94B049C752DF4F35
:10167000688379838A839B83C95DD0409B01AC01D9
:101680000E94B2AF882321F0832D0E94AF1AD5C1EA
:10169000C752DF4F288139814A815B81C95DD040C3
:1016A000C850DF4F688179818A819B81C85FD040B3
:1016B0000E94EDABC850DF4F688379838A839B8398
:1016C000C85FD040CF51DF4FE881F981C15ED04083
:1016D000C85FDE4FA881B981C850D140EA0FFB1F17
:1016E0002DE630E02C0F3D1FE20FF31FC752DF4FF6
:1016F00088819981AA81BB81C95DD040848395830B
:10170000A683B783C355DF4F488059806A807B80AA
:10171000CD5AD040CB51DF4FA881B981C55ED040B2
:101720004D925D926D927D92CB51DF4FB983A8832C
:10173000C55ED040CF51DF4FE881F981C15ED04016
:101740003496CF51DF4FF983E883C15ED040C7554F
:10175000DF4F88809980AA80BB80C95AD0401C96F0
:101760008D929D92AD92BC921F9720E030E040E8B0
:101770005FE35C962D933D934D935C935F97A3013C
:10178000920169817A818B819C810E94EDAB698392
:101790007A838B839C83A50194016D817E818F81E7
:1017A00098850E94EDAB6D837E838F839887C752A7
:1017B000DF4F288139814A815B81C95DD0406985CD
:1017C0007A858B859C850E94EDAB69877A878B87AC
:1017D0009C87A3019201C301B2010E9404AF9B0147
:1017E000AC016D857E858F8598890E94EDAB6D87F4
:1017F0007E878F87988BA5019401C501B4010E9453
:1018000004AF9B01AC0169897A898B899C890E940C
:10181000EDAB698B7A8B8B8B9C8BC752DF4F28810A
:1018200039814A815B81C95DD040CA01B9010E94FA
:1018300004AF9B01AC016D897E898F89988D0E94D0
:10184000EDAB6D8B7E8B8F8B988FA5019401C301BF
:10185000B2010E9404AF9B01AC01698D7A8D8B8D22
:101860009C8D0E94EDAB698F7A8F8B8F9C8FC752B6
:10187000DF4F288139814A815B81C95DD040C30136
:10188000B2010E9404AF9B01AC016D8D7E8D8F8DE6
:1018900098A10E94EDAB6D8F7E8F8F8F98A3C7525A
:1018A000DF4F288139814A815B81C95DD040C50104
:1018B000B4010E9404AF9B01AC0169A17AA18BA184
:1018C0009CA10E94EDAB69A37AA38BA39CA31DA14D
:1018D0000EA13FA028A420E030E0A901C301B2017D
:1018E0000E94C9AE7301620187FF04C0F7FAF09449
:1018F000F7F8F094212F302F432D522DC701B60158
:101900000E94C9AE181624F0C12ED02EE32CF22C62
:10191000CDA2DEA2EFA2F8A619A50AA53BA42CA48D
:1019200020E030E0A901C501B4010E94C9AE7501F3
:10193000640187FF04C0F7FAF094F7F8F094212FC0
:10194000302F432D522DC701B6010E94C9AE181683
:1019500024F0C12ED02EE32CF22CC9A6DAA6EBA6D9
:10196000FCA620E030E040E85FE369AD7AAD8BADE6
:101970009CAD0E94EDAB69AF7AAF8BAF9CAFC75205
:10198000DF4FC880D980EA80FB80C95DD0409501D7
:101990008401B301A201CE0183589F4F0E9425A26A
:1019A000CF51DF4FA881B981C15ED040AA0FBB1FC4
:1019B000CF51DF4FE881F981C15ED040AE0FBF1F2C
:1019C000CA5FDE4F28813981C650D140A20FB31FB4
:1019D000AB58B34FFE01E358FF4F8CE001900D92DE
:1019E0008A95E1F70E944BABCB52DF4F3881C55D42
:1019F000D040CB50DF4F4881C55FD040340FCB5231
:101A0000DF4F3883C55DD040312C5CCDC151DF4FF5
:101A1000A881B981CF5ED040119779F0C752DF4FCE
:101A2000288139814A815B81C95DD040CA01B901F1
:101A30000E94B2AF882309F4A4C480E00E940F4939
:101A4000882381F0832D0E94AF1A20E030E040EC23
:101A50005FE7C752DF4F288339834A835B83C95DC1
:101A6000D04071C4C752DF4F288139814A815B81E0
:101A7000C95DD040CA01B9010E94B2AF811163C4EF
:101A8000CE0101960E9406A88DA59EA5AFA5B8A976
:101A9000C352DF4F88839983AA83BB83CD5DD04037
:101AA00029A93AA94BA95CA9CF51DF4F28833983D3
:101AB0004A835B83C15ED0408DA99EA9AFA9B8AD12
:101AC000CB51DF4F88839983AA83BB83C55ED04007
:101AD00020E030E040E85EE3C850DF4F6881798164
:101AE0008A819B81C85FD0400E9404AFC151DF4F03
:101AF000688379838A839B83CF5ED040C351DF4F55
:101B0000A881B981CD5ED040AB2B09F480C14DE8EE
:101B10005CE061E87CE0CE0183589F4F0E94F7A211
:101B200041E85CE065E77CE0CE0187579F4F0E946B
:101B3000F7A2AE0143585F4FBE0167577F4FCE01FA
:101B40008B569F4F0E943FA2CB56DF4F4880598053
:101B50006A807B80C559D040C756DF4F8880998006
:101B6000AA80BB80C959D040C356DF4F2881398134
:101B70004A815B81CD59D040CB52DF4F28833983D6
:101B80004A835B83C55DD0402091990C30919A0CBB
:101B900040919B0C50919C0CC301B2010E9404AF78
:101BA0006B017C0120919D0C30919E0C40919F0C0B
:101BB0005091A00CC501B4010E9404AF9B01AC017F
:101BC000C701B6010E94EDAB6B017C012091A10C15
:101BD0003091A20C4091A30C5091A40CCB52DF4F3A
:101BE000688179818A819B81C55DD0400E9404AF64
:101BF0009B01AC01C701B6010E94EDAB6B017C01FA
:101C00008091750C9091760CA091770CB091780C26
